:1000000000800020BD0100000DDE0000C5DD000005
:10001000C5DD0000C5DD0000C5DD0000C5DD000058
:10002000C5DD0000C5DD0000C5DD00000DDE0000FF
:100030000DDE0000C5DD00008DD4000091D500006C
:100040000DDE00000DDE00000DDE00000DDE000004
:100050000DDE00000DDE00000DDE00000DDE0000F4
:100060000DDE00000DDE00000DDE00000DDE0000E4
:100070000DDE00000DDE00000DDE00000DDE0000D4
:100080000DDE00000DDE00000DDE00000DDE0000C4
:100090000DDE00000DDE00000DDE00000DDE0000B4
:1000A000C9B90000D5B900000DDE00000DDE00006A
:1000B0000DDE00000DDE00000DDE00000DDE000094
:1000C0000DDE00000DDE00000DDE00000DDE000084
:1000D0000DDE00000DDE00000DDE00000DDE000074
:1000E0000DDE00000DDE00000DDE00000DDE000064
:1000F0000DDE0000290201000DDE0000F9E800001D
:100100000DDE000095EB00000DDE00000DDE0000AE
:100110000DDE00000DDE00000DDE00000DDE000033
:100120000DDE00000DDE00000DDE00000DDE000023
:100130000DDE00000DDE00000DDE00000DDE000013
:100140000DDE00000DDE00000DDE00000DDE000003
:100150007DD6000091D60000A5D60000B9D60000DB
:100160000DDE0000B1EE00000DDE00000DDE00002F
:100170000DDE00000DDE00000DDE00000DDE0000D3
:100180000DDE00000DDE00000DDE00000DDE0000C3
:100190000DDE00000DDE00000DDE00000DDE0000B3
:1001A0000DDE00000DDE00000DDE00000DDE0000A3
:1001B0000DDE00000DDE00000DDE0000564B4CF29F
:1001C000205210B51A804DF628121A8000BF00BFC9
:1001D0000DF020FE514B4FF010621A60504A9A60A9
:1001E000504ADA60504A136813F4807304D14F49BF
:1001F0000B604FF4A85313604D4B1A78110703D5C9
:100200001A7842F008021A704A4B4B492A221A7097
:100210004A4A4B4B8B4204D252F8040F43F8040B6A
:10022000F8E7484B484900228B4202D243F8042B9E
:10023000FAE74649464A002352F8230041F82300D2
:1002400001336F2BF8D1434B434A802103F8011B44
:100250009342FBD1414B3D4A1A60414B8A221A70AE
:10026000A3F5805324225A70A0221A709A7992071B
:10027000FCD59A79D406FCD43A4A937903F00C035E
:10028000082B384BF9D103221A7140225A719A79FE
:100290009006FCD5334A9179324B4906FBD5324A58
:1002A000324911600221516020221A709A7902F0BD
:1002B0000C020C2AFAD12E4B2E4A1A602E4B2F4AD2
:1002C0001A6000225A60072243F8042C2C4AC3F813
:1002D0000C2D62B60EF04EF9144B1B68DA0705D5EB
:1002E00028480DF01BFF284B284A1A60284B1B7822
:1002F0005B0609D5244C254B22689A4204D121483B
:100300000DF00CFF0023236011F046FA0DF088FD7C
:100310000DF0B6FCFEE700BF0E2005403080044023
:10032000823F04000100002B10D0034014D0034092
:1003300002D0074000E00740E49CFF1FA4530100E7
:100340004088FF1FE49CFF1F28A5FF1F0082FF1F9E
:100350000000000000E400E05FE400E008ED00E0E1
:100360000050064000400640448004400000030165
:1003700004800440C010050014E000E0FF76010096
:10038000000020202CE050601CE00340A5C3945ADC
:1003900000F00740FFFFFFFFFFFFFFFFFFFFFFFF32
:1003A000FFFFFFFFFFFFFFFFFFFFFFFFFFFFFFFF5D
:1003B000FFFFFFFFFFFFFFFFFFFFFFFFFFFFFFFF4D
:1003C000FFFFFFFFFFFFFFFFFFFFFFFFFFFFFFFF3D
:1003D000FFFFFFFFFFFFFFFFFFFFFFFFFFFFFFFF2D
:1003E000FFFFFFFFFFFFFFFFFFFFFFFFFFFFFFFF1D
:1003F000FFFFFFFFFFFFFFFFFFFFFFFFFFFFFFFF0D
:10040000FFFFFFFFFFFFFFFFFFFFFFFFDEF9FFFF23
:1004100010B5054C237833B9044B13B10448AFF33E
:1004200000800123237010BDE49CFF1F000000002A
:10043000A8530100084B10B51BB108490848AFF399
:1004400000800848036803B910BD074B002BFBD0A0
:10045000BDE81040184700BF00000000E89CFF1FE7
:10046000A8530100E49CFF1F0000000038B50446BB
:10047000104621700A491D4610F070FF01464FF0EA
:100480007E5011F01FF8074910F068FFE5606060CA
:10049000256165610DF0FEFFE061204638BD00BFBB
:1004A000DB0FC9400024744938B50446104621705A
:1004B00009491D4610F052FF01464FF07E5011F0E1
:1004C00001F8064910F04AFFE5606060256165614A
:1004D0000DF0E0FFE06138BDDB0FC9400024744936
:1004E00038B503780446032B20D8DFE803F01A1848
:1004F0001002C168406910F027FE0D49054660688A
:1005000010F0E0FF0146284610F0DCFF38BD084936
:10051000406810F0D7FFE16810F020FF38BDC068D8
:1005200038BDC168406910F00FFE38BD002038BDED
:100530000024744970B504460E460DF0ABFF054625
:10054000E069281A10F0B6FEE3682361E561666190
:10055000A0610146606810F0B5FF0146A060104838
:1005600010F0B0FF10F086FA0FF026FF10F098FDA3
:10057000054601464FF07E5010F0E6FD616910F02F
:10058000EDFE21690646284610F0E8FE0146304699
:1005900010F0DCFDE0602046BDE87040FFF7A0BF32
:1005A000000080BF38B50E201C4C0DF043FA2188A6
:1005B0001B4B884205461A881DDA0023511AB1F5F3
:1005C000805FAABF1B03C3EB03330131142093FBED
:1005D000F1F10DF0B5FD134B1988F1B923889D4257
:1005E00010DAC3F57F630F33282091FBF3F1BDE8E8
:1005F00038400DF0A5BD9042D4BFC1EB0003C1EB64
:100600000203DBE740F6FF718D42D4BFC3EB050167
:10061000C3EB0101C1EB0131E3E738BDE89DFF1FEA
:10062000B29FFF1F509FFF1F10B504460DF004F846
:10063000204610BD70B44C88A04220D9012301335C
:10064000DBB21CB2660031F8144084421D46F6D37A
:10065000A04211D005F10045013D965B31F815101F
:1006600032F81530401AF21A00FB02F0641A90FBBF
:10067000F4F4E01870BC7047905B70BC70470226C1
:100680000125E5E700280CDA064A434282FB0320F5
:10069000DA17C2EB600000EB4000A3EB8000C0F172
:1006A0000C007047ABAAAA2A38B5234B1B78002B45
:1006B0002CD015200DF0BEF9204B1860204B1B8864
:1006C000984203DA1F4C237863BB38BD1E4A148856
:1006D000A042A4EB0302A8BF20467F2A1CDDC01A5B
:1006E000C001541C90FBF4F4002CEBD0154B1A788D
:1006F0000AB901221A70154D2B689C4204D0144B84
:10070000E1B2187809F024FA2C6038BD11200EF0FF
:10071000ADFA0A4B1860D1E7C01AC0EBC01090FBCD
:10072000F2F4E1E70A4B0021187809F011FA0023EE
:10073000064A2370136038BD049FFF1F109DFF1FE2
:100740008E9DFF1FE49FFF1F7C9FFF1FDC9FFF1FED
:10075000689DFF1F38B50F200EF088FA1B4A1C4B0E
:1007600012881860C0F53B600830904220DB194BBE
:100770001B889842A3EB0204A8BF1846801A7F2C5E
:10078000C6BFC0010134C0EBC01090FBF4F47CB1D3
:10079000114B1A780AB901221A70104D2B689C422D
:1007A00004D00F4BE1B2187809F0D2F92C6038BDB3
:1007B000094C237803B938BD094B0021187809F09A
:1007C000C7F90023054A2370136038BDEC9DFF1F55
:1007D000289DFF1F689FFF1F8C9FFF1F9C9DFF1F71
:1007E000869DFF1FF0B40E8886420DD203F10043B0
:1007F000013B31F81350854202D9F0BCFFF71ABF14
:1008000032F81300F0BC70471088F0BC704700BF8E
:10081000094B1B880C2B09D8084A80B252F82320B8
:1008200028B143F6FE73984203D9108C70471088A4
:1008300070470349FFF7FEBE3E9DFF1FA42D010038
:10084000402F01004B4B4C4A2DE9F0471E8814689D
:100850004A4BB442B3F80080494B33DB4445A8BF50
:100860004446A6421C60C8BF00202DDDC6EB080729
:10087000B7F5804F33DB80037B1C90FBF3F0FFF771
:10088000C7FF404A404B15881B88C0F3C61909FBB7
:1008900005F57F2D8246A8BF7F252BB3A64253DCEA
:1008A0004445D4BFC6EB0404C6EB08049F42CCBF4A
:1008B00003FB04445C43354BC8BF013794FBF7F797
:1008C0001F6013E034461E60C6EB0807A045D4BF86
:1008D000C6EB0800C6EB0400B7F5804FCBDAC0EBDF
:1008E000803090FBF7F0CAE7284A1360284C236851
:1008F000994508D0274B1B88002B34D1264B1B88E9
:100900006BBBC4F80090254C23689A4506D0214B58
:100910001B885A1F032A19D9C4F800A0204C236849
:100920009D420FD01F4B188848B11A4B1E4A1B8896
:10093000D35C834203D0C0B2E9B209F009F9256063
:10094000BDE8F087BDE8F0870024AFE7164AD05C29
:100950002030C0B20AF07F0109F0FAF8DCE748461F
:1009600009F096F9CDE7104A4946D05C09F0F0F855
:10097000C4E700BFE89DFF1F4C9FFF1FB29FFF1FF2
:10098000089DFF1F189DFF1F1A9DFF1FB89FFF1F87
:10099000809DFF1F349FFF1FDA9DFF1F389DFF1FA3
:1009A000DC9DFF1F429FFF1F0C8AFF1F2DE9F04FA8
:1009B00001208BB00EF05AF9DFF870B3DFF870A3A6
:1009C000CBF8000000200EF051F9BA4BCAF8000035
:1009D0001B880C2B00F05E82B74EB84A3188B84BAA
:1009E00052F8214000221A70B64BB74A1B88B7490B
:1009F0001288013B012A31F91330059300F0AE81D2
:100A0000B34B0193B34B0293B34FDFF8288300231A
:100A10000093B24B1B88012B00F0F481DFF8189390
:100A2000AF4B0393D9F80050AE4B04930023AE4A6A
:100A30001288013A032A00F24982DFE812F0A50089
:100A4000ED000400C9002846059310F033FCA749C7
:100A500010F084FC059B0546184610F02BFCA449B9
:100A600010F07CFC0146284610F070FB10F03CFEB4
:100A70000546C9F80050386810F01CFC9B4910F07E
:100A80006DFC8146009810F015FC994910F066FC49
:100A90000146484610F05AFB10F026FE3860954A91
:100AA000954B17881988954BDBF800201B88DFF8D9
:100AB0008CE2C7EB050C3D44039FC7F800C0471A02
:100AC000084404990D6001990F600299BEF8007006
:100AD00008609A4280F2E7800025C3EB070E744558
:100AE000DAF8000080F2D380611C984205FB01F522
:100AF0000EF1010E95FBFEF5C0F25F838742A8BFA1
:100B00000746FF1A01FB07F494FBFEF49A4200F338
:100B1000A780984200F3A480794C206810F0CAFBAB
:100B2000784910F01BFC784910F010FB10F0DCFD48
:100B3000A0F5FF531C3B082B98BF4FF40050D8F88A
:100B40000030184400282060C0F29F80B0F5804F2C
:100B500080F2F6806D4B1B781BB1B0F5005F40F062
:100B6000F7806B4D2B78002B40F0AB81694D2068EE
:100B70002B68634C984204D080B208F0B9FF236818
:100B80002B600BB0BDE8F08F2846059310F092FB68
:100B9000614910F0E3FB059B0546184610F08AFBFF
:100BA0005E4910F0DBFB0146284610F0CFFA10F04A
:100BB0009BFD0546C9F80050386810F07BFB56498C
:100BC00010F0CCFB8146009810F074FB53495DE7B0
:100BD0002846059310F06EFB4A4910F0BFFB059BB9
:100BE0000546184610F066FB4D4910F0B7FB01466C
:100BF000284610F0ABFA10F077FD0546C9F8005012
:100C0000386810F057FB3F4910F0A8FB8146009868
:100C100010F050FB424939E72846059310F04AFB93
:100C2000404910F09BFB059B0546184610F042FB1F
:100C30003D4910F093FB0146284610F087FA10F06A
:100C400053FD0546C9F80050386810F033FB3549AC
:100C500010F084FB8146009810F02CFB324915E718
:100C60003388002B3FF458AF2B1B002BB8BF5B42DF
:100C7000092B00F32D81D8F80030214C4FF400509F
:100C8000184400282060BFF661AF00225AE0984265
:100C900005FB04F5B8BF002195FBFEF580F28482C8
:100CA00091FBFEF432E7BA42D4BFC3EB0205C3EBBB
:100CB000070512E77E9FFF1F769DFF1F8889FF1F94
:100CC0000E9DFF1F2089FF1F529FFF1FA4320100AE
:100CD000E09FFF1FAC9DFF1F009DFF1FE49EFF1FB5
:100CE000709FFF1FE89EFF1F5E89FF1FCDCC4C3F0A
:100CF000CDCC4C3E188AFF1F5C89FF1F489FFF1F09
:100D0000C089FF1F9A99193FCDCC4C4596A0FF1F73
:100D1000D89DFF1F2489FF1F3333733FCDCC4C3D3B
:100D2000CDCCCC3E6666663FCDCCCC3D709DFF1FE2
:100D3000349DFF1F889FFF1F6C9FFF1F549DFF1F47
:100D400043F6FF72C04B22601B78002B3FF409AFC3
:100D500005F0A4FFBD4B01221A7007E7BC4BBD4A4A
:100D60001B88BD491278013B31F91350002A40F02D
:100D7000C78011200DF07AFF0090B84B0193D3F893
:100D80000080009B984540F3C080B54BB54F1B8851
:100D9000B54A012B3B68B2F80090B44A0292204653
:100DA000A3EB050500F0E28010F084FA029A52F8F5
:100DB000291010F0D3FA0146002010F0C5F910F008
:100DC00093FC009BC8EB05029D42B8BF1D469042B4
:100DD000C8EB050580F2DE8000FB0555013295FB6E
:100DE000F2F5A34BDFF8B4820293D8F800302B441D
:100DF00003EBD3735B10C8F800309E4B1B88012BAC
:100E00007FF40CAE9C4B03931D460F200DF02EFF7C
:100E10002A6804929042034680F2CC80904A12885D
:100E2000012A00F03F81904A079012888F4D069268
:100E3000204610F03FFA069ADFF8649255F8221027
:100E4000D9F8005010F08AFA0146002010F07CF921
:100E5000059BEA1A059210F047FC059A079B049936
:100E60009A42C1EB020EB8BF1A46704580F2448127
:100E7000521A00FB02220EF1010192FBF1F2D8F8A6
:100E800000107E4804900A4402EBD2725210C8F857
:100E90000020CCE57A4B1B78002B3FF49DAD794EBA
:100EA000794A3188794B52F8210001221A7010F0EA
:100EB00001FA4FF07C5110F051FA10F015FC044685
:100EC00092E505F0E7FE00232B704FE63868E6E573
:100ED00005F500500130001B10F0ECF96C496D4C29
:100EE00010F03CFA0546206810F0E4F96A4910F069
:100EF00035FA0146284610F029F910F0F5FB1EE6F8
:100F000015200CF097FD009037E7594B0293D3F86A
:100F10000080009B984542DA514B524F1B88524A41
:100F2000012B3B68B2F80090504A039220461D44C2
:100F300000F0E98010F0BEF9039A52F8291010F081
:100F40000DFA10F0D1FB009B9D42C8EB0502A8BF33
:100F50001D46C8EB05059042BABF00FB055501329E
:100F6000454395FBF2F5DFF834813EE710F0A2F936
:100F7000029A52F8291010F0F1F910F0B5FB009B1D
:100F8000C8EB05029D42B8BF1D468242C8EB05056D
:100F90003FF722AF00FB05F595FBF2F521E7DFF8FF
:100FA000FC80304FD8F8003003EBD3735B10C8F8E7
:100FB00000302EE5314A049212680692904237DDE5
:100FC000274A1288012A00F0BC80274A099011881C
:100FD000264A08912046079210F06CF9079A089962
:100FE000DFF8BC9052F82110D9F8005010F0B6F993
:100FF000059B2B44059310F077FB0599099B069AF6
:101000009942C2EB010EA8BF1946704580F2BE801E
:10101000891A00FB01110EF1010291FBF2F2D8F8DE
:1010200000100A4402EBD2725210C8F80020FEE40D
:10103000D8F80020DFF8689002EBD2725210D9F88D
:101040000050C8F80020F2E496A0FF1FD89DFF1FB3
:10105000648AFF1F049FFF1FF82E0100E09FFF1FFF
:10106000BE9DFF1F009DFF1F5C9DFF1FBC32010046
:10107000AC9DFF1FE49EFF1F709FFF1FE89EFF1F98
:10108000269DFF1F769DFF1F8889FF1F0E9DFF1F56
:10109000CDCCCC3EC089FF1F9A99193F889FFF1F76
:1010A0006C9FFF1F464A08901188464A07912046C8
:1010B000069210F0FFF8069A0799DFF80C9152F8A3
:1010C0002110D9F8005010F049F9059BE91A059153
:1010D00010F00AFB0599089B049A9942C2EB010E95
:1010E000B8BF1946704558DA891A00FB01110EF194
:1010F000010291FBF2F2C2E60499521A00FB02F2DD
:1011000092FBFEF2BBE610F0D5F8039A52F82910D4
:1011100010F024F90146002010F016F810F0E4FA5F
:10112000009A9542C8EB0503A8BF1546C8EB050514
:101130009842BABF00FB05550133454395FBF3F5D3
:1011400011E71F491F4A089020460D88079210F0AA
:10115000B1F8079ADFF8709052F82510D9F80050CE
:1011600010F0FCF8014600200FF0EEFF059B2B4429
:10117000059310F0B9FA0599089B069A9942C2EBBB
:10118000010EA8BF19467045FFF642AF069A891AAC
:1011900000FB01F191FBFEF241E7049A891A00FB82
:1011A00001F191FBFEF26AE6B842D4BFC3EB000145
:1011B000C3EB070104FB01F172E51F46A1E400BF88
:1011C0005C9DFF1FBC3201006C9FFF1F08B5244BC4
:1011D0001B88FBB1234B1B78FBB1234B1B78E3B17E
:1011E000224B1B78CBB1224B1B78B3B1214B224849
:1011F0001A78C2B9214A2249008812880968024433
:10120000B1EB620F09DD01221A706420BDE80840CD
:1012100005F058BD174A117801B908BD1370BDE833
:10122000084008F009BD154A164900881288096867
:101230000244B1EB620FF0DD00221A7008F0FCFCF2
:10124000642005F03FFD642005F03CFD642005F0BE
:1012500039FD4FF41670BDE808400DF03DB900BFF0
:10126000F69EFF1FAE9FFF1FAF9FFF1FB09FFF1F88
:10127000B19FFF1F3C9DFF1F549DFF1F489FFF1FF5
:10128000709DFF1F349DFF1F38B5114C232025781A
:101290000CF0D0FB0F4A42F82500131F02F1C400E6
:1012A000002253F8041F83420A44FAD123780A49E2
:1012B00007480A4C0133DBB2322B81FB025108BFD5
:1012C0000023D217C2EB21120370226038BD00BF89
:1012D0001C9DFF1FF89DFF1F1F85EB51449FFF1FA3
:1012E0002DE9F04FB84CB94D2068B94F83B00FF0DD
:1012F000E1FFB84910F032F8064610200DF0B6FCB8
:101300000FF0D8FFB44910F029F831460FF01EFF56
:1013100010F0EAF92988206088423B8843DA9E462B
:101320005B1A7F2B4FF0000247DDD2015E1C92FB5F
:10133000F6F2AA4EDFF8C882B6F800C0C8F800205E
:10134000BCF1190F00F0DF80BCF11A0F00F018811A
:10135000BCF11E0F00F021810126B146A04A12887F
:10136000002A00F09D808842C0F208817045D4BFF9
:10137000C1EB0000C1EB0E009A42BABF02FB0000B5
:101380000133504390FBF3F3964A1360964B188851
:10139000C0B9964A1288AAB9954B197801B11A704A
:1013A00003B0BDE8F08F9842D4BFC1EB0002C1EB9F
:1013B00003029E465B1A7F2BB7DCC2EBC21292FB84
:1013C000F3F2B6E72988D4F800E0DFF80082DFF80E
:1013D000F8A171456CDCDFF818C29CF80020002AE7
:1013E0002ED14FF0010B04288CF800B028D1002E2C
:1013F00040F095817D4B18880028D1D0B9F1000FBD
:10140000CED023682C883A88A34280F266810023DC
:10141000141B7E2C774DD5BFC3EB8313C3EBC313D3
:101420005B00013493FBF4F42B680134A34203D036
:10143000C0B2E1B208F08CFB2C6003B0BDE8F08FC5
:10144000012800F0F780022800F0EC800328D1D1B9
:10145000694B1B88092BCDD0002ECBD023682E885A
:101460003A88B34280F27C810023961B7E2EDFF8FF
:101470008CA1D5BFC3EB8313C3EBC3135B00013651
:1014800093FBF6F6DAF800300136B34203D0F1B23E
:101490004A2008F05DFBCAF80060ABE791460126E0
:1014A000BCF11E0F7FF472AF0022DFF858817FE09D
:1014B0004F4B1A78002A3FF473AF002401281C70A8
:1014C00000F0A480022840F00F81002E00F0A380DD
:1014D0004A4D2B68002B00F09E800420214608F026
:1014E00037FB424B2C60188800283FF459AFB9F104
:1014F000000F3FF455AFC0B2002108F029FB3D4B6F
:1015000000221A604CE7DFF8FC8098F80020C2B196
:10151000DFF8D890B9F800A0BAF1000F11D0DFF8C9
:10152000E89099F800B0934578D05FFA8AF07F216F
:1015300008F00EFB98F80030B6F800C089F80030CB
:1015400010E0DFF8C49099F800A0924566D0274BD0
:101550000021187808F0FCFA98F80030B6F800C0BE
:1015600089F800301E4B1A88002A97D0BCF11E0F54
:1015700040F0078101264FF0000919E00020FBE64A
:10158000DFF8808098F80020002A0BBF0126002693
:101590004FF000094FF00109E0E6DFF86880104BDA
:1015A00098F800601A88B6FA86F676094FF00009B6
:1015B00098F80030002B3FF4E7AE2988B7F800E038
:1015C0002068C1EB0E03CEE6649DFF1FFC9EFF1F4B
:1015D000F89EFF1F9A99193FCDCCCC3E7E9FFF1FEE
:1015E000BC9FFF1FF09DFF1F6C9DFF1F909FFF1F63
:1015F000849FFF1F489DFF1F349FFF1FF49DFF1F07
:10160000649FFF1F269DFF1F229DFF1F1EB1624D7D
:101610002B68002B7CD1614B188865E701264FF0C1
:1016200000099BE6002E3FF4E5AEDFF86CA1DAF886
:1016300000202EE0002E3FF4DDAEB7F80080F0452C
:10164000D4BFC1EB0802C1EB0E02C1EB0808B8F130
:101650007E0FDFF844A1D5BFC2EB8212C2EBC212EB
:10166000520008F1010892FBF8F8DAF8002008F1BE
:101670000108424506D05FFA88F10120009308F086
:1016800067FA009B1888CAF8008002287FF4DEAE53
:1016900042462168B5F800803888414559DA002172
:1016A000C8EB0008B8F17E0FD3BFC1EB8111C1EBCD
:1016B000C11108F10108490091FBF8F808F101088F
:1016C000904506D05FFA88F10420009308F040FAB4
:1016D000009B1888CAF80080B8E69342D4BFC4EBD8
:1016E0000303C4EB020393E6032827D12C4B1B888A
:1016F000092B90D0002E8ED0274D2B68002B8AD03E
:101700004A20214608F024FA244B2C601888EBE686
:10171000214608F01DFA214B2C601888E4E6402091
:101720007F218DE80C0008F013FA019B009A1888BD
:1017300058451CD002287FF489AE76E704287FF450
:101740006AAF002E3FF467AF2146402008F000FA50
:1017500061E78142D4BFC8EB0101C8EB00019FE7FC
:101760009342D4BFC6EB0303C6EB02037DE6B8F891
:101770000010DAF800E0B7F800808E45FFF665AF9C
:101780005DE72988B7F800E02068C1EB0E03012669
:101790004FF00009E7E500BFF49DFF1F909FFF1F7A
:1017A000349FFF1F08B5114B1B88022B09D0052B56
:1017B00007D0032B15D0042B0BD00D4B01221A7030
:1017C00008BD7F21412008F0C3F9094B01221A709E
:1017D00008BD7F21092008F0BBF9054B01221A70D2
:1017E00008BD4021092008F0B3F9E6E7EE9DFF1F90
:1017F000929DFF1F38B5074B074D1B88052B0446EC
:1018000006D02B68834203D0C1B2052008F0A0F9AE
:101810002C6038BDEE9DFF1F989FFF1F38B5124DFD
:10182000124C2B88052B12D022684AB9022B0ED0FD
:10183000033B012B13D90E4A00231370236038BDDC
:101840000021052008F084F92B88022B04D1002107
:10185000412008F07DF9EEE7052BE9D1F7E70021FB
:10186000092008F075F9E6E7EE9DFF1F989FFF1F1E
:10187000929DFF1F464B1B881D2B70B541D0454DD7
:101880000024454B1B88022B16D0444B1B88022B8F
:1018900054D02888424B002C1B780ADB8442A8BF16
:1018A000044634B1002B3AD02046BDE87040FFF723
:1018B000A1BF002B2FD170BD3A4B1B78002B37D026
:1018C00015200CF0B7F8384B1860384A1288002AF7
:1018D000DBD0374A186811888142D6DC354B2A881C
:1018E0001B888342A3EB0106A8BF03465B1AB242E2
:1018F000BABF02FB03330136534393FBF6F31C4498
:10190000C3E72A4B1C888CB12B4B224D1C78002C32
:10191000B7D02C88B5E7BDE87040FFF77FBFFFF771
:1019200041FF2046BDE87040FFF764BF194DA8E7AE
:1019300011200DF09BF91C4B1860C6E70F200DF02D
:1019400095F91A4B1D4A1B881060002BA1D01C4A28
:10195000C0F53B63118808338B429ADB194A28880B
:1019600012889342A2EB0105A8BF1346A842A3EB3D
:10197000010306DA00FB0333013593FBF5F31C4446
:1019800088E700FB03F292FBF5F31C4482E700BFFB
:101990007E9FFF1F869FFF1F529FFF1FE49EFF1F1A
:1019A000929DFF1F049FFF1F109DFF1FEE9DFF1FB5
:1019B0008E9DFF1F7C9FFF1F269DFF1F289DFF1FE1
:1019C000EC9DFF1F689FFF1FF8B510200DF04EF92A
:1019D000C830B0F5FA7FC0F29680B0F57A6F014654
:1019E000A8BF4FF47A6101F51673B3F57A6FA8BFFB
:1019F0004FF47A639BB289B2914A924C11802220B3
:101A0000238008F0FFF921888F4D904C242008F0A6
:101A1000F9F90E200CF00EF840F6FF71C83088423C
:101A2000A8BF084620EAE07000F2DC5283B28A4286
:101A3000A8BF0A460220194622802B8008F0E2F94E
:101A40002188042008F0DEF901200DF00FF904468A
:101A500000200DF00BF9A042B8BF204600F1C801EC
:101A6000B1F5FA7FC0F2D180B1F57A6FA8BF4FF41B
:101A70007A6101F54873B3F57A6FA8BF4FF47A63C2
:101A80009BB289B2724A734C11800A20238008F0FD
:101A9000B9F921880C2008F0B5F90F200DF0E6F80F
:101AA000C0F53F610431B1F5AF6FC0F2AB80B1F565
:101AB000FA6FA8BF4FF4FA6189B2674BC0F5436073
:101AC000B0F5AF6F1980C0F29A80B0F5FA6FA8BF79
:101AD0004FF4FA6083B2614CA420238008F092F99D
:101AE0002188A62008F08EF915200BF0A3FF00F541
:101AF0009671B1F52F7F0BDB41F25C23994240F3E5
:101B00008980194608E040F24C434FF4FA7173E7BC
:101B100040F214534FF42F71514A1180514C524DE1
:101B20002380062008F06EF92188504E082008F026
:101B300069F900274FF4AF74F9B24D4809F0B8FFC6
:101B400055F8043BC3F5967300FB03F086FB0023B6
:101B5000C017C0EB6310844207F10107A8BF044619
:101B6000062FE9D1434F414E0025E9B2424809F022
:101B70009FFF57F8043BC3F5967300FB03F086FB09
:101B80000023C017C0EB6310844205F10105A8BF14
:101B900004460C2DE9D1394F344E0025E9B23848BE
:101BA00009F086FF57F8043B304AC3F5967300FBF3
:101BB00003F086FB0013C017C0EB6310844205F1ED
:101BC0000105A8BF04460C2DE8D1A4F11401312968
:101BD00031DD40F23A73A4F5B97403FB04F482FBDF
:101BE0000432E417A4EB621289B232322548264B44
:101BF00001801A602A20BDE8F84008F003B94FF4CC
:101C0000AF6368E74FF4AF6157E740F214534FF406
:101C1000FA7137E7124A00F5617089B2B0F52F7F8B
:101C20001180B8BF4FF42F73FFF678AF8342A8BF7F
:101C300003469BB272E740F26C723221D6E700BFD6
:101C4000FC9EFF1FF89EFF1FE89DFF1FB29FFF1F16
:101C5000489FFF1F549DFF1FEC9DFF1F689FFF1FA4
:101C60008E9DFF1F7C9FFF1F4C8AFF1FB5814E1B5F
:101C7000409DFF1F1C8AFF1F749DFF1F2C89FF1FA3
:101C8000E09DFF1FAC9FFF1F088AFF1F2DE9F84F43
:101C90000C200BF09BFE0C200CF050FBCB49DFF826
:101CA000B4A314200CF05AFBC949CA4809F092FBAE
:101CB000022103200CF0E8FB022104200CF0E4FBDD
:101CC000022105200CF0E0FB022106200CF0DCFBD9
:101CD00001210A200CF0D8FB012109200CF0D4FBD3
:101CE00001210D200CF0D0FB012128200CF0CCFBB1
:101CF000012114200CF0C8FB012116200CF0C4FBBC
:101D0000012117200CF0C0FB012121200CF0BCFBAD
:101D100002211C200CF0B8FB01211B200CF0B4FBAD
:101D200000211B200CF09CFB1C200CF09FFBB0FA48
:101D300080F35B091A208AF800300CF03BFD1F206D
:101D400000210CF0FDFC04200CF090FB002800F0BA
:101D5000318105200CF08AFB002800F0A6810023C9
:101D60009D4C062023700CF081FBB0FA80F35B09D8
:101D70004FF0000B994A137006F0CCFB2478002C2E
:101D800040F01481584608F067F8954B954A1B8837
:101D900015889549954840F23A72A3F5AF7302FB56
:101DA00003F381FB0312DB17A3EB621332330360EF
:101DB0008F4B01210D201D700CF052FB64200CF0A4
:101DC0008BFB4FF416710A200CF0BAF95D2189489B
:101DD00009F0AAFE002800F0A58164200CF07CFB2D
:101DE00021460A200CF0ACF94FF4967109200CF052
:101DF000A7F95C21804809F097FE002800F07F8158
:101E000064200CF069FB214609200CF099F94FF48D
:101E1000967116200CF094F95B21784809F084FE45
:101E2000002800F0498164200CF056FB2146162062
:101E30000CF086F94FF4967117200CF081F96420AC
:101E40000CF04AFB214617200CF07AF964200CF0C4
:101E500043FB21460D200CF003FB694A69481268D8
:101E6000DFF8F491684F694D694EDFF8F081002387
:101E70000121FEF719FB01233C602C60346089F8D6
:101E8000003004240F200CF0F1FE336803440E20D0
:101E900033600BF0CFFD3B6899F8002018443860A0
:101EA000002A7CD015200BF0C5FD2B681844286053
:101EB00004F0010080F0010004F0F4FEB8F80030F6
:101EC000002B14BF4B20DC200CF006FB013CD9D1C9
:101ED000336839684C4A28684E4F002BB8BF03332B
:101EE0000029B8BF0331891011604B494B4A09885A
:101EF00014889B1000283360B8BF0330484E82100E
:101F0000581A19442A6031603860464D464847499E
:101F1000161B22442E6002600B60BBF1000F40F0E4
:101F2000AC80B8F80030002B00F09A80404B0124C0
:101F300004201C600CF09AFA18B93E4B2C4A1C7015
:101F400010703D4B1B881C2B00F09F803B4C04F114
:101F5000C80523200BF06EFD44F8040F01200CF09F
:101F6000BBFAA542F5D19AF8003023B1344B1B7867
:101F7000002B40F09580002121200CF071FA314AAD
:101F8000314B1078187007F06FFD04F083FE45F6B2
:101F9000BF522E492E48BDE8F84F0BF003BB11206D
:101FA0000CF064FE2B681844286081E7BDE8F84F08
:101FB00009F020B906200CF059FA00287FF4C9AEC8
:101FC000054C034620704FF0010BD3E6001B37464B
:101FD00040420F00EC91FF1F449DFF1FEC9EFF1F2E
:101FE000AC9FFF1F809FFF1FB5814E1B088AFF1FFC
:101FF000A89DFF1F409DFF1FE09DFF1F749DFF1FB9
:102000002889FF1F109FFF1F149DFF1F009DFF1FAA
:102010006C9FFF1F709FFF1F188AFF1F5C89FF1FA7
:10202000E89EFF1FE09FFF1FAC9DFF1FC49FFF1F87
:10203000789FFF1F2C9DFF1F7E9FFF1FF49DFF1F9A
:10204000FE9EFF1F009FFF1FE39EFF1FA5050000D0
:10205000A09FFF1FE69EFF1F049FFF1F3E9FFF1FC5
:102060004FF4FA7004F02EFE04F018FE06F09CFD0A
:102070004FF4AF600CF030FA58E7FFF7A5FCB8F862
:102080000030002B7FF452AFEAE7294B1888002874
:102090003FF45CAF274BC0B2197807F059FD55E704
:1020A000012121200CF0DCF969E703200CF0DEF9B6
:1020B000B0FA80F35B0953E603200CF0D7F900284F
:1020C000FAD104200CF0D2F90028F5D105200CF04B
:1020D000CDF90028F0D106200CF0C8F90028EBD18A
:1020E0000CF0E4FE04200CF0C1F940B905200CF01E
:1020F000BDF920B906200CF0B9F90028F0D0032072
:102100000CF0B4F90028FAD1ECE704200CF0AEF999
:1021100040B905200CF0AAF920B906200CF0A6F968
:102120000028DDD003200CF0A1F90028FAD1ECE75B
:10213000B09DFF1F609DFF1F2DE9F04FAD4C26782D
:10214000012E95B000F05582C0F00B82022E00F0F7
:10215000D880A949A94A91F800801178A84ADFF8E7
:102160003CE3A84DA84FA948A94B0292A94A009266
:10217000A94A9EF800B001922D78A84A3F7890F8BD
:1021800000E01B78DFF818A3DFF818C3DFF8189316
:102190000392012E84BF00222270A14AA14813702D
:1021A000A14A80F800B01570A048A14A077082F8D3
:1021B0000080A048A04A03709CBF013626701170B1
:1021C000BEF1000F40F074819C4A10880D2800F089
:1021D000B9819B4C00202070024604462DB19748DF
:1021E0000088002840F0BA810546964806882544B4
:1021F000002E40F067819448944C019E0078367818
:1022000024780130A0EB4600002C40F05682039C5D
:1022100094F800E0CEEB0004BEF1000F40F07682AF
:102220000026DFF874E202989EF800E00078A41B14
:10223000A4EB4E043C44CBEB040410B1B7FA87F096
:1022400040099CF800602718BC1B1EB11EF1000657
:1022500018BF0126009F99F8000097F800909AF89F
:1022600000C07B4FC6EB040EC0EB0E00A0EB490094
:102270008044C3EB0803A3EB41010C2313FB0C11B7
:102280003960744B744F754C75481B880088D7F8BB
:1022900000C0744E2788744C3688D4F800E0033BA5
:1022A000C0EBC00403EB4303C7EBC70001EB8303A0
:1022B00064446E4F334470446D4E57F8244056F8D2
:1022C00020000C3B1D44254405440AB1694B1960AC
:1022D000694A13689D4200F03181684B684819686B
:1022E0000791079901601B6808936648089B00885E
:1022F00015605B1A834284BF634B1D6015B0BDE857
:10230000F08FDFF8A881614E08AF0025E9B2604880
:1023100009F0CEFB58F8043BC3F5967300FB03F0BD
:1023200086FB00230135C017C0EB63100C2D47F866
:10233000040BEBD1574B384D0195384DB3F800C025
:102340000395109D09980F99404EDFF8C0A0DFF863
:10235000B490DFF8BC80654511AA8CCAAE46ACBF0C
:102360004FF0000E4FF0010E8445D4BF0020012035
:1023700030708C4528480B9D1F4E8AF800E0D4BF72
:1023800000210121017094452449DFF814A1D4BF34
:10239000002201220A709C453F4AD4BF002301233A
:1023A000BC45AB46D4BF002701271370AC45164B84
:1023B0000C9D1F70D4BF4FF0000B4FF0010B374B3B
:1023C0000F4A0292AC45DFF834C0124A83F800B0DD
:1023D000D4BF0025012589F8005098F800309CF8FA
:1023E000001096F80080DFF8BCC02678DFF8B890BF
:1023F0000092CEE6E29EFF1F309FFF1F329FFF1F1D
:10240000C09DFF1F379FFF1F909DFF1FEC9FFF1F69
:10241000319FFF1F829FFF1F959FFF1F969FFF1FEA
:10242000E69FFF1FE79FFF1FE89FFF1FE99FFF1F1A
:10243000EA9FFF1FEB9FFF1F839FFF1FEE9FFF1F62
:10244000269DFF1F0C9DFF1F1A8AFF1FD09FFF1F95
:10245000389FFF1F569FFF1FF09DFF1F949DFF1F7A
:10246000749FFF1F1E9DFF1FB89FFF1FB830010004
:10247000402A0100C89FFF1F889DFF1FD4A0FF1F97
:10248000789DFF1F8E9FFF1FD49FFF1FB5814E1B9E
:10249000E09DFF1FAC9FFF1F979FFF1F919DFF1F98
:1024A000ED9EFF1FE59FFF1FAA9FFF1F2C89FF1FA7
:1024B000AF4AB04814880122182C027040F20581FE
:1024C00000248BE6012E00F08F81022E00F0EE81B9
:1024D000032EA94B00F01F811E78009B9CF800E0A2
:1024E0001C78019B99F800C01878029B93F8008033
:1024F000039B1F78A6EB4E03A4EB8404CCEB030CE8
:10250000C0EB80760CEB0403C0EB8600034403EBC6
:10251000480303EB810327B198490978002940F06B
:10252000608201269AF800109548C1F1060101EB7E
:102530004101334403EB81010160A2E69149924BD2
:102540000968D0E6002D3FF444AE894A894E1488CC
:102550000122182C327040F2B8807446A0F10D05AB
:1025600043E6DFF87092894F0DF120080025E9B2AB
:10257000874809F09DFA59F8043BC3F5967300FBB0
:1025800003F087FB00230135C017C0EB6310062D55
:1025900048F8040BEBD17F4BDFF83CA219880D9B68
:1025A00000228B428AF8002080F2A2807A4B8AF8BF
:1025B00000507A497A4A7B4891F8008011787A4A2B
:1025C0001D7002920378794ADFF810C2DFF810928A
:1025D0000092774A774E784D784892F800E0784A32
:1025E0000192784A96F800B02D7807782678039201
:1025F000CFE5DFF8F081654E08AF0025E9B27248FB
:1026000009F056FA58F8043BC3F5967300FB03F043
:1026100086FB00230135C017C0EB63100C2D47F873
:10262000040BEBD15B4B0C9D1F885F4B02935F4B00
:1026300000930B9B0A98099ADFF8A0C1089EDFF867
:10264000A0910F99BB429E46ACBF4FF0000E4FF0D9
:10265000010EAF42D4BF002501258742109B8CF8A4
:102660000050D4BF00200120504D89F8000097424F
:10267000D4BF00220122B742D4BF4FF000084FF070
:1026800001082A709F42474A4448474E80F800801C
:10269000D4BF002301231370129A414886F800E04A
:1026A0008F42D4BF00210121974201701ADC002221
:1026B0004648DFF824A102708BE7039C46B12678D8
:1026C000002E40F06081441EABE50C3C012285E504
:1026D00094F800E00138CEEB0004BEF1000F7FF467
:1026E000A0AD9DE5119A9742D4BF00220122DFE7F9
:1026F0000C9A374B9142CCBF012200221A7040F352
:10270000458105258AF80050234B52E7002E3FF4FF
:1027100087AD012685E51C78009B029893F8008020
:10272000019B9CF800601B7890F800C099F800703D
:102730000398A4EB4604E71B90F800E0C3EB837416
:10274000A8EB88003844C3EB8403034403EB4C0339
:1027500003EB8103BEF1000F40F0488101269AF897
:102760000010074833440C2414FB0131016088E554
:102770007E9FFF1F269DFF1F1A8AFF1F979FFF1F27
:10278000389FFF1F789DFF1FD4A0FF1FB5814E1BF0
:10279000409DFF1FAC9FFF1FFA9EFF1F309FFF1F32
:1027A000329FFF1F319FFF1FC09DFF1F829FFF1F92
:1027B000EC9FFF1F919DFF1F379FFF1F909DFF1FE5
:1027C000959FFF1F969FFF1F749DFF1F5A9DFF1F20
:1027D000B19FFF1F4C8AFF1FED9EFF1FE59FFF1F4C
:1027E000AA9FFF1F1C8AFF1FA34CDFF89CE22078E2
:1027F00005909EF8004001980494059C0078019093
:102800000134A4EB40040498002840F0AF80039802
:1028100090F800E00498261ACEEB06000390BEF173
:10282000000F40F09E8074460298944E007802900B
:10283000039836780496041BA4EB460402983C44A3
:10284000CBEB0404002800F08780B7FA87F040093A
:102850009CF800602044871B1EB10498061C18BF1A
:102860000126009C99F800002478BE1B301AA0EBCA
:10287000440080440198C3EB0803A3EB4103002804
:1028800067D1BEF1000F40F0BB807344002C5ED1D5
:1028900000290CBF00206FF009009AF80010784C56
:1028A00003440C2010FB01312160EAE4039E019CEB
:1028B00036780396009E2478019434786F4E7148E0
:1028C00099F800E0009496F800906F4C9DF80C6029
:1028D00086709DF80460067080F806E09DF8006040
:1028E00080F803909CF800C02478DFF8B491DDF8FC
:1028F00004E080F80880077180F805C0C671417255
:1029000044704FF000080120009500215D4C0D46F9
:102910005FFA88FC4F46764607E0022809D00A296C
:102920000BD014F8016F17F8010F864201F1010175
:10293000F3D101350A29EDB2F3D1092D72D808F18E
:102940000108B8F1100F36D019F80A0FDDE70020A2
:10295000A3E74FF0000E98E7029879E7CEEB04006A
:1029600003900198041C18BF01245DE7019800281A
:102970004ED0039890F800E0BEF1000FEED1601E3B
:102980000390744650E7841B01264AE40B9A3F4BA0
:102990009142CCBF012200221A703EDC0A9A3C4BC5
:1029A0009142CCBF012200221A7052DD03258AF821
:1029B0000050384BFDE5304837490478C86B029920
:1029C000009D097801342044CBEB0000084400212D
:1029D0009AF800402A4B401A0C2111FB040119609F
:1029E0004FE41BF1000618BF01269BE52349097837
:1029F00000293FF4B3AE1BF1000618BF0126AEE676
:102A0000049800280CBF4FF0000E4FF0090E3CE771
:102A1000039890F800E03046FDE604258AF800505F
:102A20001C4BC6E514481C49047851F8280002994B
:102A3000009D097801342044CBEB00006646084431
:102A4000002BC4D0002EC2D1BBF1000FBFD001219A
:102A5000BEE7099A114B9142CCBF012200221A70A5
:102A600004DD02258AF800500A4BA2E5089B994232
:102A700018DD01259AE500BF1A8AFF1F979FFF1FE7
:102A8000389FFF1FB49DFF1FD09FFF1FB09FFF1FE8
:102A9000AF9FFF1FFA9EFF1FC889FF1FAE9FFF1F3A
:102AA000882F0100154B1D78012D25D9144A8AF86D
:102AB00000501288D2B1134A1288013A92B2062A03
:102AC00014D8114A12788AB1104A1268012A7FF488
:102AD00070AD0F4A0F4E10680C2290FBF2F102FB12
:102AE000110232800C4A0321117062E5074A126814
:102AF000012A7FF45EADF5E735465AE5FA9EFF1FE1
:102B0000609FFF1F029FFF1FEA9DFF1F789FFF1F0F
:102B1000D49FFF1F3C9FFF1FBC89FF1F2DE9F04F73
:102B20003A4B1B788BB0002B6BD10E200AF082FF42
:102B30000EF0C0FB01463648364E374DFDF7FAFC25
:102B40003348FDF7CDFC0EF0CFFD80F30C00306074
:102B5000FFF7F2FA2C68012C7AD0022C00F0BF8229
:102B6000032C00F0D3832D4E2D4C33682D4A2E4E6E
:102B70000993099B316812882360591A013A9142DE
:102B8000274F00F2A782294E32689A1A0D2A00F2C6
:102B90009082274E32689A1A132A00F28582254EB7
:102BA00032689A1A252A1AD9234B1B88002B40F029
:102BB0005B81224B1B78002B40F05681FEF764FBB3
:102BC0001F4B1B881B3B9BB2022B04D81D4B1B7851
:102BD000002B40F04C8104F087F8236833601A4DD5
:102BE0002A689B1A502B00F20D82184B1B88012B70
:102BF00000F0258206F030FF06F014FE0BB0BDE8B1
:102C0000F08F08F07FF90BB0BDE8F08F449DFF1FF7
:102C1000109FFF1F4C9FFF1F789FFF1FD4A0FF1F17
:102C20000C9FFF1FC489FF1FE49DFF1FCC9DFF1F4A
:102C3000A09DFF1FA49DFF1FF69EFF1F3C9DFF1F31
:102C40007E9FFF1F269DFF1FF09EFF1F509FFF1FAF
:102C5000DFF820939F4AB9F800001378834204D02C
:102C6000C3B21846137006F0E9FEDFF804839A4AEF
:102C7000B8F800301178994204D0984F397800297B
:102C800040F03287964A33681288964E9A42C0F2D4
:102C9000F880954A1278002A40F0F380DFF8D8A235
:102CA000BAF8003023B9914B1B88002B00F04F85F8
:102CB0008F4A904B11881B888F4A0B4412685B1017
:102CC00093428E4A126880F2F18400219342B4BF8D
:102CD00001230B4604910093ACBF4FF0010B8B46D0
:102CE00005910E200AF0A6FE854B864A1B681768E0
:102CF00003930133A7F25232002B8446029240F331
:102D00000487802BA8BF80237F4A804912780191D5
:102D1000002A00F0C0800978914200F0BC80B8F829
:102D20000010DFF84CE2994201F0EC806B49AEF8FC
:102D30000030774B4FF0010E81F800E01978DFF892
:102D40003CE2019B8EF800101A70009B002B00F0F3
:102D50001781BAF80030002B00F012816D4B1B6810
:102D60005A1C002A40F3DC86802A00F3D8866A4C7D
:102D70006A496B482488098800682144B0EB610FD8
:102D8000C1F25183A3F148020F2A02D8473BA9F8A8
:102D900000300E200AF04EFE6FF454731F44874239
:102DA00002DC604B00221A705F4B1B88002B00F086
:102DB00074845E4B5E4A1B781178994243D0002B95
:102DC00041D05C490C78002C00F097875A4991F863
:102DD00000C0BCF1000F40F08E87584F0097584F4D
:102DE00058480297554F007887F800C0544F4FF06D
:102DF000010E87F800C081F800E0002841F0F28061
:102E000051490978002901F02680504903910C4668
:102E10000978002941F01C804D48494F00783970ED
:102E200001210297217070B14448434900904948FC
:102E300003270770002008700099029F087003990B
:102E400001243C7008701370434B1B88A3F11B02D4
:102E5000012A40F237861D2B7FF486AE3C4A3F4B59
:102E600012781A703E4C80E6FEF7B0F9A6E63D4BAC
:102E70001B78002B3FF4AFAE2B68012B7FF4ABAE79
:102E8000ABE63168384A069106983849106002224C
:102E90000B602A6002E71E49DFF8E0E009780029AC
:102EA0003FF44FAF9EF8000081423FF44AAF0398D1
:102EB0004B2840F3EE871833802BB8F80000A8BFEA
:102EC000802398423FF43DAF294803800348012303
:102ED000037036E7E39EFF1FA89DFF1F2C9DFF1F79
:102EE000E89DFF1FD4A0FF1F3C9DFF1FD29DFF1F29
:102EF000549DFF1F489FFF1F709DFF1F349DFF1FA4
:102F0000C89FFF1F149DFF1FBE9FFF1F849DFF1FB3
:102F1000BF9FFF1F389FFF1FFC9EFF1FF89EFF1FD4
:102F2000649DFF1F4C9DFF1F029FFF1F5A9DFF1FA7
:102F3000049DFF1FE99FFF1F409FFF1F949FFF1FDE
:102F4000EA9DFF1FEA9FFF1FE69FFF1F059DFF1FD2
:102F5000269DFF1FBC89FF1F7E9FFF1F229DFF1F15
:102F60000C9FFF1F839FFF1F989DFF1F089FFF1F40
:102F7000809FFF1F009FFF1F8C9DFF1F859DFF1FD0
:102F8000029B9C45BFF605AF924B1B88002B3FF47C
:102F900000AFBBF1000F7FF4E1AE8F4B1B881BB17C
:102FA000059B002B7FF4DAAE049B002B3FF4F1AEBF
:102FB0008A4B1A78002A7FF4ECAEDFF8A09299F8D9
:102FC000004001221A70002C40F08E83844B1B7845
:102FD000002B02F0B880834B1B78002B02F0878314
:102FE000814B1B78002B7FF4D4AE804B1B78002BD9
:102FF0003FF4CFAEB8F800307D490A3BA8F8003066
:103000000A70C6E605F0CEFA7A4B1B7873B97A4B94
:103010001B785BB9794B1B7843B9794B1B782BB97B
:10302000784B1B7813B903F035FE01E003F03EFE48
:1030300023682B60744B1B88012B7FF4DBAD734B33
:1030400073491A680868734DA92303FB02F3002B28
:10305000B8BF03F57F53704AB8BF3F339B13117855
:10306000543BA0F118022A2000FB023028600029FE
:1030700000F0C08269490A68904200F3738310DA55
:10308000674D2B78002B40F04385664B1B68D3F1CE
:103090007F0348BF03339B100133D21A904242F39F
:1030A000B08608600246A8E2FEF7E4FB23683360BE
:1030B00075E5FDF77BFCFEF713F95B4B1B88032BD3
:1030C00000F04E85594B1B88032B00F04585236883
:1030D00033605EE5FDF7B6FB3B68336053E5544A69
:1030E00034681288A24204DB464B1B78002B00F0A8
:1030F0007283504E504833680793504B07990068CD
:103100001B88091A994200F2AF80002B00F0AC80B6
:103110004B4B198800293FF427AD4A4B4A481B689E
:103120000088A342B8BF23469A4241F36A81474BC5
:103130001A60DFF82C8188F80010354FFDF782FB0C
:1031400038687F2840F3D385414B7F3883FB0032BA
:10315000C317C3EB620303EB4303A0EB830073309D
:103160003C4B01931B883860002B40F0BD86234BFD
:1031700000931B78002B00F02684374C2378002B1B
:1031800000F02184DFF8DC90DFF8C4A04FF0000BE2
:103190000CE003F17300C0B298F8001006F008FDCF
:1031A00023780BF1010B5B4540F30D843B6859F824
:1031B000040F1844A0F17F038AFB0321DA17C2EB46
:1031C000610202EB42027F28A3EB8203E1DCFDF700
:1031D00059FAE0E7D29DFF1F069FFF1F4C9DFF1F7E
:1031E000E69FFF1FE79FFF1FE89FFF1FE99FFF1F4D
:1031F0002C9DFF1FEA9DFF1F409FFF1F949FFF1FF5
:10320000059DFF1F3C9DFF1F509FFF1FC089FF1F93
:10321000D49FFF1FC49DFF1F929DFF1FD49DFF1FC2
:103220009C9FFF1F989FFF1F529FFF1FE49EFF1F41
:10323000E89DFF1FD4A0FF1F989DFF1FD09DFF1F7B
:10324000249DFF1F089FFF1FB29FFF1F089DFF1FA8
:10325000ABAAAA2A6A9DFF1F8489FF1FED9EFF1F4C
:10326000C19DFF1F5C89FF1FBD4BBE491B680888BD
:10327000BD49A342B8BF23469A4200F38982BB4CA2
:1032800009888342A8BF0346236000297FF451AF19
:103290009A42C8BF0B4640F38282801AB0F5804F35
:1032A000AABF9B03C3EB8333013093FBF0F0FDF720
:1032B000AFFAC0F3C6100DF0FDFFAD4B0446188801
:1032C0000DF0F8FFAB49074620460EF047F80146DF
:1032D00038460EF043F821460DF038FF4FF07E518E
:1032E00004460EF0D9F9002841F07080A24920462A
:1032F0000EF0F0F9002840F06F8620460EF01AFA22
:10330000C0B2DFF8A48288F8000016E79B4BD6F81D
:1033100000801988414553DD994B1B78002B4FD114
:10332000DFF8889299F800007F2840F34E86A3F1D9
:1033300055337F3803F1004383FB0032C317C3EBDF
:10334000620303EB4303A0EB830073308D4B0193C7
:103350001B88C0B289F80000002B41F033808A4BF3
:1033600000931B78002B00F0F584884C2378002B09
:1033700000F0F084864FDFF820824FF0000A0AE068
:1033800003F17300C0B206F037FC23780AF1010A9A
:10339000534540F3DF8457F8043F99F80000184480
:1033A000A0F17F0388FB0321DA17C2EB610202EB75
:1033B00042027F28A3EB8203E2DCFDF763F9E1E739
:1033C000744F38687F2800F3F181FDF75BF9DFF86F
:1033D000DC9199F80040844200F04F82624B1B88D8
:1033E000002B43D1614A5F4812680088914205DC96
:1033F0008242D4BFC1EB0203C1EB0003411AB1F515
:10340000804FA6BF9B030131C3EB833393FBF1F0E5
:10341000FDF7FEF9C0F3C6100DF04CFF544B80468B
:1034200018880DF047FF5349824640460DF096FF3D
:10343000014650460DF092FF41460DF087FE4FF0D9
:103440007E5180460EF028F9002840F0AE874A49A8
:1034500040460EF03FF9002840F0BB8540460EF094
:1034600069F9C0B2DFF8408188F800007F2C40F392
:103470002F8449487F3C80FB0430E317C3EB600096
:1034800000EB4000A4EB800073303F4B00931B78AF
:10349000C0B289F80000002B40F069833F4B0393D2
:1034A0001B78002B40F074853D4B02931B78002B5A
:1034B00040F0A087334B0193029B1B78FBB1394B43
:1034C0001B88012B00F0C785022B00F0DF87032B40
:1034D00001F08681042B01F08783052B01F09B848A
:1034E000062B01F00486072B01F0AF87082B02F0B2
:1034F0006680092B02F08C810A2B02F07483009BFA
:103500001B78002B00F0B784019B1E4C1988002902
:1035100000F0378538687F2840F326831E4B7F38BC
:1035200083FB0032C317C3EB620303EB4303A0EB3F
:10353000830073303860002940F0BC84009B1B7806
:10354000002B00F0EF81114C2378002B00F0EA8172
:10355000DFF83CA0DFF850804FF0000B35E000BFF3
:10356000089FFF1FB29FFF1F249DFF1F089DFF1F85
:10357000C09FFF1FCDCCCC3D0000FE42E89DFF1F49
:103580003C9DFF1F6A9DFF1F949FFF1F8489FF1FA3
:103590005C89FF1FD49FFF1FABAAAA2A059DFF1FAE
:1035A000EA9DFF1F029FFF1FC19DFF1F369FFF1F48
:1035B00003F17300C0B298F8001006F0F9FA23780E
:1035C0000BF1010B5B4540F3AD813B685AF8040FEA
:1035D000B04A1844A0F17F0382FB0321DA17C2EB43
:1035E000610202EB42027F28A3EB8203E0DCFDF7DD
:1035F00049F8DFE7A84902460860A84B188858B385
:10360000A74B256853F82040B5FBF4F3772C04FB57
:10361000135300F3A080C3EBC30303EB031393FB2B
:10362000F4F3A048A04C50F8230024689F4BA0F26C
:10363000FF7004FB00F000F57D3000F5607000EBDA
:103640004004C0EBC40083FB00430344C017C0EB3D
:10365000A3400B3802440A609549964B08881988A4
:1036600000F27C704300B3F57C6FA1F164014FEA76
:103670004100B5BF9049914903FB02225A4381FBA7
:1036800002311144D317C3EBE123C11881F30C01BC
:1036900028200AF055FDFFF7ADBA894C89488A49C0
:1036A0008A4A237003700B70FFF7CDBB93424FF033
:1036B000000B80F288800123CDF800B0CDF814B063
:1036C0000493FFF70EBB824B1B78002B7FF461AB9A
:1036D000039B804A243B83F34703D9B25B201360EA
:1036E00006F036FA99F80040032C30D1DFF830822A
:1036F00098F80030002B42F0F281774F3B78002B96
:1037000042F0E081724C2378002B42F0CE81734B63
:103710001B78002B42F0BC81714A1380714B1B78DF
:10372000002B42F0E881704B7F221A8098F800301D
:103730006BB93B785BB923784BB96C4A7F21072082
:10374000138006F005FA7F210B2006F001FA684B82
:103750001F68FFF71EBBC3EB0313D800631C90FB6D
:10376000F3F35EE7634D2B78002B40F0D181624B81
:103770001B68D3F17F0348BF033302EBA30201327E
:1037800090420A60444BBFF638AF1860024634E7F7
:103790005A4B09881A6000297FF4CBAC1346984233
:1037A000D4BFC2EB0003C2EB030376E5394B7F388D
:1037B00083FB0032C317C3EB620303EB4303A0EBAD
:1037C0008300733003E60123CDF810B0CDF800B0CC
:1037D0000593FFF786BA01232B60FFF7C4B9029B5C
:1037E0001B78FBB1464B1B88012B00F0B684022BE3
:1037F00000F0E686032B01F07580042B01F019829E
:10380000052B01F0A382062B01F06984072B01F040
:103810007785082B01F01A87092B02F01A800A2BF2
:1038200002F07681019B1B88002B00F04C83009BEB
:103830001B783BB9039B1B7823B9029B1B78002B99
:1038400000F0C4871F4B1B78002B00F04B812D49E3
:103850000B78082B00F246812B483A6800682B4C05
:103860000133DBB25F1E101A44F827000B70284B9F
:10387000D6F80080198889F800208845254E7FF702
:1038800073A93268244B0892089A244C1A60FFF7F7
:103890006CB900BFABAAAA2AD49DFF1F209DFF1FB1
:1038A000642F01003C280100649FFF1F4D261281F8
:1038B000D89FFF1FA89FFF1F81DFFF818320088201
:1038C000EA9DFF1F409FFF1F949FFF1F059DFF1F45
:1038D000E99FFF1F509DFF1FE89FFF1FE79FFF1FEE
:1038E000DA9DFF1FEA9FFF1F249DFF1F349FFF1FCC
:1038F000149DFF1F9C9FFF1F989FFF1F089DFF1F88
:10390000029FFF1F8489FF1F309DFF1F6089FF1FDB
:10391000E89DFF1FD4A0FF1F80A0FF1F0C9FFF1F6B
:10392000E69FFF1F039B1B78002B3FF458AF3B68BB
:10393000A3F10C007F2840F34283A6488B3B80FB19
:103940000320DA17C2EB600000EB4000A3EB80031A
:1039500003F17300DFF8C082C0B298F8001006F0DF
:1039600027F9009B1B78002B3FF439AF9A4C237842
:10397000002B3FF434AFDFF8A4A24FF0000B0CE0B3
:1039800003F17300C0B298F8001006F011F9237823
:103990000BF1010B5B457FF722AF3B685AF8040F30
:1039A0008C4A1844A0F18B0382FB0321DA17C2EB87
:1039B00061020C3802EB42027F28A3EB8203DFDCBA
:1039C000FCF760FEDEE7854B1B78002B40F0818220
:1039D0003B68834A1278002A45D0A3F10C007F2867
:1039E00040F3F0827B4A8B3B82FB0321DA17C2EB68
:1039F000610202EB4202A3EB820303F17300C0B247
:103A000098F8001006F0D4F8009B1B7853B3724C62
:103A100023783BB3DFF80492DFF8B8A14FF0000B36
:103A20000BE003F17300C0B298F8001006F0C0F884
:103A300023780BF1010B5B4514DD3B6859F8040F4B
:103A40001844A0F18B038AFB0321DA17C2EB610251
:103A50000C3802EB42027F28A3EB8203E1DCFCF787
:103A600011FEE0E73B685F4A1278FAB15E4A1288BD
:103A7000012A00F01784022A00F02386032A00F0AE
:103A8000AE87042A01F00A81052A01F02A82062A5B
:103A900001F04B83072A01F07183082A01F03A866E
:103AA000092A01F00D870A2A02F06980019A12881A
:103AB000002A00F020824D4A4D4C137003232B60E6
:103AC000FFF753B8DFF8408198F80030002B40F042
:103AD0000481484F3B78002B40F09A84444C3B7063
:103AE000FFF743B83A68C2E6DBB21846137006F037
:103AF000EDF8414B39491A46394B184600230B70F3
:103B00003B7013700370FFF7BDB80123FFF7FCB8DB
:103B10000133DBB2022B88BF00232B706DE58024BC
:103B20003649374B374A09881B8812680B44B2EB79
:103B3000630FBFF62EA9344B1B78002B40F0128286
:103B4000B8F80030314AA3423FF423A9304B148027
:103B500001221A70FFF71DB9FCF7FCFDFFF7B7BA99
:103B6000FCF7A2FDFFF7AEBAFCF78CFDE2E4294BAF
:103B700001931B88002B53D1194B0393194B0293CC
:103B8000154C2378002B55D0DFF89080DFF844A047
:103B90004FF0000B09E003F17300C0B206F02CF8FF
:103BA00023780BF1010B5B4544DD58F8043F99F88D
:103BB00000001844A0F17F038AFB0321DA17C2EB4F
:103BC000610202EB42027F28A3EB8203E3DCFCF7F5
:103BD00059FDE2E7ABAAAA2A8489FF1F409FFF1F75
:103BE000059DFF1FEA9DFF1F029FFF1F369FFF1FBE
:103BF0000C9FFF1F229DFF1F949FFF1FF89EFF1F1A
:103C0000FC9EFF1F649DFF1F269DFF1F809FFF1FBF
:103C10002C9DFF1F6A9DFF1FC19DFF1F5C89FF1F19
:103C2000BB4B0393BB4B029305F0E6FF009B1B7855
:103C3000002BA5D1039B1B78002B3FF43DAC99F8DA
:103C40000030A3F10C007F2840F3B681B2488B3BD3
:103C500080FB0320DA17C2EB600000EB4000A3EB0F
:103C6000800303F17300C0B205F0C6FF009B1B7810
:103C7000002B00F09681A94C2378002B01F05C8288
:103C8000DFF8BC82DFF890A24FF0000B0AE003F1EE
:103C90007300C0B205F0B0FF23780BF1010B5B4558
:103CA0007FF70AAC58F8043F99F800001844A0F1D7
:103CB0008B038AFB0321DA17C2EB61020C3802EB9B
:103CC00042027F28A3EB8203E1DCFCF7DBFCE0E7A8
:103CD0002046FCF7D7FCFFF7D8BB914A1278002AA0
:103CE00040F08D818F4F904C3B70FEF73EBFFCF74C
:103CF000C9FCFFF735BA002008708C49087840B13C
:103D00008B4900910978002900F06981009F00210A
:103D100039708849097800297FF477A8002C40F091
:103D20009A80002840F09780834C814F94F800E0FF
:103D3000774C0394774C0294754C80492070754CF5
:103D40000097087038702070BEF1000F7FF46FA8E4
:103D5000FFF779B86E4B1B78002B42D099F80030F2
:103D6000A3F10C007F2840F367836B4A8B3B82FBF7
:103D70000321DA17C2EB610202EB4202A3EB8203DA
:103D800003F17300C0B205F037FF009B1B7843B30B
:103D9000624C23782BB36A4FDFF87C814FF0000A26
:103DA00009E003F17300C0B205F026FF23780AF1A1
:103DB000010A534515DD57F8043F99F800001844EF
:103DC000A0F18B0388FB0321DA17C2EB61020C38E8
:103DD00002EB42027F28A3EB8203E2DCFCF752FCF9
:103DE000E1E74C4B1B78FBB1564B1B88012B00F0D5
:103DF0007486022B00F07D87032B01F0F780042BE3
:103E000001F08281052B01F0BF83062B01F0DC84D9
:103E1000072B01F0A385082B01F01187092B01F076
:103E2000A9870A2B01F08787019B1B88002B00F0D4
:103E3000C482424B1B78002B40F0BA82424B434A6B
:103E40001988D6F800800020012310602B6014E54B
:103E50000398002101703849097800293EF4F3AF36
:103E60002C4902910978002900F069870298002105
:103E70000170FEF7E8BF039B1B78002B7FF444AB77
:103E8000029B1B78002B7FF43FAB019B1988FFF747
:103E900041BB243B002BB8F8000040F391849842CA
:103EA0003EF44FAF9BB22A48A8F8003001230370BC
:103EB000FEF747BFDFF89C80C0B298F8001005F00D
:103EC00077FEFFF73BBB234B3878197805F070FE7F
:103ED000ADE47F21402005F03BFE1F490F4A3B68BF
:103EE0000B600021117074E5C0B298F8001005F065
:103EF0005FFEFFF73CB9D8B298F8001005F058FE05
:103F00003B68D8E5154BDFF858E01978FEF719BF84
:103F1000059DFF1FEA9DFF1FABAAAA2A8489FF1FE8
:103F2000839FFF1F229DFF1F0C9FFF1FEA9FFF1F04
:103F3000949FFF1FE69FFF1F269DFF1F409FFF1FAF
:103F40005C89FF1F029FFF1FE89DFF1F089DFF1F49
:103F50002C9DFF1FC19DFF1F309DFF1FBF9FFF1F97
:103F6000859DFF1F4B2C40F334821834802CB8F809
:103F70000030BD4AA8BF8024A3427FF4E7ADFEF71E
:103F800008BF99F8000005F037FE2188FFF7C2BA94
:103F9000B64B01931B88002B41F02F87B44B029343
:103FA0004DE6029B1B78002B7FF489AA039B1B78AC
:103FB000002B7FF4A9AA68E7FCF764FB53E6FCF743
:103FC00061FBC7E4FCF75EFB19E5FCF75BFBFFF761
:103FD000BDB97F20FFF746BA7F20FFF792B9A44F03
:103FE000A44902974FF0000C81F800C0009F02998D
:103FF0004FF0010E87F800E081F800C089E69E4F7F
:10400000387802F0DBFE9D4B1B78002B00F02182FC
:104010003B887E2B00F21D82994CDFF87892226853
:10402000D9F80010521A0F2A40F20A82954A013339
:10403000108899B23980002800F02482C9B2C0B239
:1040400005F086FD904F226898F80030C9F80020EE
:104050003B70FEF78ABDDFF840A299F80000BAF87D
:1040600000308A4A8A4CC31A82FB031ED917C1EB5F
:104070006E0101EB4101A3EB810303EB430354F811
:10408000233018447F2840F321857F3882FB00329B
:10409000C317C3EB620303EB4303A0EB830073304E
:1040A000DFF8F8B1C0B205F0A7FDBBF80030022B75
:1040B0007FF625AA99F80010BAF80030734ACB1A97
:1040C00082FB030ED817C0EB6E0000EB4000A3EBA1
:1040D000800303EB430304EB8303586808447F2801
:1040E00040F362877F3882FB0032C317C3EB620262
:1040F00002EB4202A0EB82007330C0B205F07CFDFF
:10410000BBF80030032B7FF6FAA999F80010BAF833
:1041100000305E4ACB1A82FB030ED817C0EB6E004C
:1041200000EB4000A3EB800303EB430304EB8304A9
:10413000A06808447F2840F379817F3882FB0032F1
:10414000C317C3EB620202EB4202A0EB82007330A2
:10415000C0B205F051FDFFF7D2B9DFF83CA13868D5
:10416000BAF80030494A4A4CC31A82FB031ED917D9
:10417000C1EB6E0101EB4101A3EB810303EB4303B0
:1041800054F8233018447F2840F325847F3882FB7D
:104190000032C317C3EB620303EB4303A0EB8300BE
:1041A0007330DFF8FC80DFF8F4B098F80010C0B28C
:1041B00005F0FEFCBBF80030022B7FF633AB39680C
:1041C000BAF80030314ACB1A82FB030ED817C0EB85
:1041D0006E0000EB4000A3EB800303EB430304EB12
:1041E0008303586808447F2840F377867F3882FB32
:1041F0000032C317C3EB620202EB4202A0EB820063
:104200007330C0B298F8001005F0D2FCBBF8003053
:10421000032B7FF607AB3968BAF800301B4ACB1A7C
:1042200082FB030ED817C0EB6E0000EB4000A3EB3F
:10423000800303EB430304EB8304A06808447F2856
:1042400040F304817F3882FB0032C317C3EB620264
:1042500002EB4202A0EB8200733098F80010C0B26B
:1042600005F0A6FCFFF7DEBA809FFF1F6A9DFF1FC7
:10427000EA9DFF1F409FFF1F609DFF1FEB9FFF1FD9
:104280000C9FFF1FB09DFF1F229DFF1FABAAAA2AF4
:10429000682E0100CC9FFF1F3C9FFF1F429DFF1F08
:1042A000C19DFF1FDFF80CA3B749BAF80020B74C37
:1042B0009A1A81FB020ED017C0EB6E0000EB400093
:1042C000A2EB800202EB420254F8220018447F283D
:1042D00040F30084A0F17F0381FB0321DA17C2EBD6
:1042E000610000EB4000A3EB80007330DFF8C8B240
:1042F00098F80010C0B205F05BFCBBF80030022B50
:1043000050D93968BAF800309F4ACB1A82FB030EA5
:10431000D817C0EB6E0000EB4000A3EB800303EB6B
:10432000430304EB8303586808447F2840F3468620
:104330007F3882FB0032C317C3EB620202EB4202FA
:10434000A0EB82007330C0B298F8001005F030FC8A
:10435000BBF80030032B25D93868BAF800308A4AF8
:10436000C31A82FB031ED917C1EB6E0101EB410199
:10437000A3EB810303EB430304EB8304A36818441A
:104380007F2856DD7F3882FB0032C317C3EB620201
:1043900002EB4202A0EB82007330C0B298F800102A
:1043A00005F006FC3B68FFF781BB0120FFF75AB818
:1043B0000021402005F0CCFB40E599F8000005F015
:1043C0001BFC36E505F018FCFEF7C9BF0120FEF71F
:1043D00098BF243C002CB8F8003040F3E985A34294
:1043E0003EF4D7ACA4B26A4BA8F8004001221A7080
:1043F000FEF7CFBC674B01931B88002B3FF45CA8F2
:1044000012E4654A8342A8BF03461360FEF791BEDB
:10441000624B634C19886A2005F0F4FC98F8003070
:104420003B70FEF7A2BB1446FFF785BBFCF72AF9E9
:104430008EE6FCF727F9B0E7FCF724F9A2E4584C24
:10444000584F98F800303B70FEF78FBBFCF71AF915
:1044500003E7554B1B78002BF1D03B884F4F002BC7
:10446000EDD04F4CDFF854912268D9F80010521A61
:104470000F2AE5D94D4A013B108899B239800028AE
:104480007FF4DCADC8B205F003FCDBE5DFF824A166
:1044900099F80000BAF800303B4A454CC31A82FB39
:1044A000031ED917C1EB6E0101EB4101A3EB8103A0
:1044B00003EB430354F8233018447F2840F312845D
:1044C0007F3882FB0032C317C3EB620303EB430365
:1044D000A0EB83007330DFF8E0B0C0B205F08CFBD6
:1044E000BBF80030022B7FF60AA899F80010BAF842
:1044F0000030254ACB1A82FB030ED817C0EB6E00A2
:1045000000EB4000A3EB800303EB430304EB8303C6
:10451000586808447F2840F3F3857F3882FB0032D7
:10452000C317C3EB620303EB4303A0EB83007330B9
:10453000C0B205F061FBBBF80030032B7EF6DFAFA5
:1045400099F80010BAF800300F4ACB1A82FB030E1C
:10455000D817C0EB6E0000EB4000A3EB800303EB29
:10456000430304EB8304A06808447F287FF75EAF11
:104570007F3882FB0032C317C3EB620303EB4303B4
:10458000A0EB83007330E3E5ABAAAA2A682E0100F2
:104590002C9DFF1F6A9DFF1F089DFF1F609DFF1F31
:1045A0000C9FFF1F229DFF1FEA9FFF1FB09DFF1F53
:1045B000603101003C9FFF1F429DFF1FCC9FFF1FEA
:1045C000DFF814A33868BAF80030C04AC04CC31AE8
:1045D00082FB031ED917C1EB6E0101EB4101A3EB76
:1045E000810303EB430354F8233018447F2840F33E
:1045F00044837F3882FB0032C317C3EB620303EBB3
:104600004303A0EB83007330DFF8D082DFF8D0B231
:1046100098F80010C0B205F0CBFABBF80030022BBE
:104620007FF600A93968BAF80030A84ACB1A82FB95
:10463000030ED817C0EB6E0000EB4000A3EB800325
:1046400003EB430304EB8303586808447F2840F3DB
:1046500068857F3882FB0032C317C3EB620303EB2C
:104660004303A0EB83007330C0B298F8001005F04C
:104670009FFABBF80030032B7FF6D4A83868BAF84D
:104680000030924AC31A82FB031ED917C1EB6E0198
:1046900001EB4101A3EB810303EB430304EB830430
:1046A000A36818447F287FF7D1AE7F3882FB0032A1
:1046B000C317C3EB620303EB4303A0EB8300733028
:1046C000CBE5DFF814A28149BAF80020804C9A1A91
:1046D00081FB020ED017C0EB6E0000EB4000A2EB96
:1046E000800202EB420254F8220018447F2840F373
:1046F000FD82A0F17F0381FB0321DA17C2EB610089
:1047000000EB4000A3EB80007330DFF8D4B198F8E1
:104710000010C0B205F04CFABBF80030022B7FF657
:1047200041AE3968BAF80030684ACB1A82FB030EF2
:10473000D817C0EB6E0000EB4000A3EB800303EB47
:10474000430304EB8303586808447F2840F3E5845F
:104750007F3882FB0032C317C3EB620303EB4303D2
:10476000A0EB83007330C0B298F8001005F020FA77
:10477000BBF80030032B7FF615AE3868BAF800306E
:10478000524AC31A82FB031ED917C1EB6E0101EB1B
:104790004101A3EB810303EB430304EB8304A36810
:1047A00018447F287FF745AE7F3882FB0032C3175D
:1047B000C3EB620303EB4303A0EB83007330ECE530
:1047C00001283EF4BEAA0123FFF76DBB4FF47A43E4
:1047D000013BFDD199F8000005F00EFAFFF732B861
:1047E000DFF8F4A099F80000BAF80030374A394CE5
:1047F000C31A82FB031ED917C1EB6E0101EB410105
:10480000A3EB810303EB430354F8233018447F28C0
:1048100040F3DB817F3882FB0032C317C3EB6202B7
:1048200002EB4202A0EB82007330DFF8B4B0C0B2FA
:1048300005F0E2F9BBF80030022B7EF660AE99F885
:104840000000BAF80030214AC31A82FB0321DA17AC
:10485000C2EB610202EB4202A3EB820303EB4303D0
:1048600004EB83035B6818447F2840F328847F3877
:104870000C2290FBF2F302FB13007330C0B205F080
:10488000BBF9BBF80030032B7EF639AE99F8000077
:10489000BAF800300D4AC31A82FB0321DA17C2EBC3
:1048A000610202EB4202A3EB820303EB430304EB3E
:1048B0008304A36818447F287FF7B8AD7F380C22A3
:1048C00090FBF2F302FB1300733041E4ABAAAA2A77
:1048D00060310100F03101003C9FFF1FC19DFF1FAF
:1048E000429DFF1FDFF8A8A33868BAF80030E44AF9
:1048F000E44CC31A82FB031ED917C1EB6E0101EB16
:104900004101A3EB810303EB430354F82330184424
:104910007F2840F35D817F3882FB0032C317C3EBF1
:10492000620202EB4202A0EB82007330DFF8648384
:10493000DFF864B398F80010C0B205F039F9BBF89D
:104940000030022B7EF66EAF3868BAF80030CC4AE1
:10495000C31A82FB0321DA17C2EB610202EB4202A7
:10496000A3EB820303EB430304EB83035B6818446C
:104970007F2840F3A1837F380C2290FBF2F302FBE7
:1049800013007330C0B298F8001005F011F9BBF8AD
:104990000030032B7EF646AF3868BAF80030B84ACC
:1049A000C31A82FB0321DA17C2EB610202EB420257
:1049B000A3EB820303EB430304EB8304A3681844D3
:1049C0007F287FF743AD7F380C2290FBF2F302FB88
:1049D0001300733041E4FBF755FEFFF7E2BBDFF84D
:1049E000B0A2A749BAF80020A64C9A1A81FB020E81
:1049F000D017C0EB6E0000EB4000A2EB800202EB90
:104A0000420254F8220018447F2840F3E480A0F1C9
:104A10007F0381FB0321DA17C2EB610101EB410146
:104A2000A3EB81007330DFF870B298F80010C0B2C9
:104A300005F0BEF8BBF80030022B7FF6B3AC386847
:104A4000BAF800308E4AC31A82FB0321DA17C2EB90
:104A5000610202EB4202A3EB820303EB430304EB8C
:104A600083035B6818447F2840F336837F380C2229
:104A700090FBF2F302FB13007330C0B298F8001001
:104A800005F096F8BBF80030032B7FF68BAC386846
:104A9000BAF800307A4AC31A82FB0321DA17C2EB54
:104AA000610202EB4202A3EB820303EB430304EB3C
:104AB0008304A36818447F287FF7BBAC7F380C229F
:104AC00090FBF2F302FB1300733066E4FBF7DAFDB0
:104AD000FFF7E6BAFBF7D6FD08E4DFF8B4A199F8D2
:104AE0000000BAF80030664A674CC31A82FB03170D
:104AF000D917C1EB670101EB4101A3EB810303EB84
:104B0000430354F8233018447F286ADD7F3882FB42
:104B10000032C317C3EB620202EB4202A0EB820039
:104B20007330DFF874B1C0B205F066F8BBF800303E
:104B3000022B7FF679A999F80000BAF80030504AA4
:104B4000C31A82FB0321DA17C2EB610202EB4202B5
:104B5000A3EB820303EB430304EB83035B6818447A
:104B60007F2840F3B6827F380C2290FBF2F302FBE1
:104B700013007330C0B205F03FF8BBF80030032BD0
:104B80007FF652A999F80000BAF800303C4AC31ADF
:104B900082FB0321DA17C2EB610202EB4202A3EBB4
:104BA000820303EB430304EB8304A36818447F28C8
:104BB00014DD7F380C2290FBF2F302FB13007330FC
:104BC000C0B205F019F8FFF72FB9FBF75BFD2CE633
:104BD000FBF758FDAAE6FBF755FD24E7FBF752FD6E
:104BE000EEE7FBF74FFD9CE7DFF8A4A099F8000083
:104BF000BAF80030224A254CC31A82FB031ED9178B
:104C0000C1EB6E0101EB4101A3EB810303EB430315
:104C100054F8233018447F28D7DD7F3882FB0032D8
:104C2000C317C3EB620303EB4303A0EB83007330B2
:104C3000FBE5DFF85CA03868BAF80030104A134C86
:104C4000C31A82FB031ED917C1EB6E0101EB4101B0
:104C5000A3EB810303EB430354F8233018447F286C
:104C6000B6DD7F3882FB0032C317C3EB620303EB70
:104C70004303A0EB8300733058E6FBF703FDC3E466
:104C8000ABAAAA2AF0310100682E0100D42A010043
:104C90003C9FFF1FC19DFF1F429DFF1FDFF840A3E8
:104CA000C849BAF80020C84C9A1A81FB020ED017E6
:104CB000C0EB6E0000EB4000A2EB800202EB420270
:104CC00054F8220018447F2885DDA0F17F0381FB82
:104CD0000321DA17C2EB610000EB4000A3EB800078
:104CE0007330A0E6FBF7CEFCFFF7F5BBFBF7CAFC81
:104CF0000BE5DFF8ECA299F80000BAF80030B14AF1
:104D0000B24CC31A82FB0317D917C1EB670101EB41
:104D10004101A3EB810303EB430354F82330184410
:104D20007F287FF75EAF7F3882FB0032C317C3EB6B
:104D3000620303EB4303A0EB83007330F1E6A44866
:104D40000090A448A4490390FEF771B8DFF890A240
:104D50003868BAF800309B4AA04CC31A82FB032182
:104D6000DA17C2EB610202EB4202A3EB820303EB10
:104D7000430354F8233018447F2840F3A7817F3839
:104D80000C2290FBF2F302FB13007330DFF8548225
:104D9000DFF854B298F80010C0B204F009FFBBF875
:104DA0000030022B1AD93868BAF800300C22C11A28
:104DB00091FBF2F302FB131302FB03435B681844FD
:104DC0007F2840F390847F3890FBF2F302FB1300BE
:104DD0007330C0B298F8001004F0EAFEBBF800305F
:104DE000032B7EF61FADBAF8003038680C22C11ACA
:104DF00091FBF2F302FB131302FB0344A368184474
:104E00007F287FF723AB7F3890FBF2F302FB130080
:104E10007330FFF722BADFF8C8A199F80000BAF89A
:104E20000030684A6D4CC31A82FB0321DA17C2EBCB
:104E3000610202EB4202A3EB820303EB430354F84B
:104E4000233018447F2840F33E817F380C2290FBAA
:104E5000F2F302FB13007330DFF88CB1C0B204F040
:104E6000CBFEBBF80030022B19D999F80000BAF834
:104E700000300C22C11A91FBF2F302FB131302FB68
:104E800003435B6818447F2840F326847F3890FBF7
:104E9000F2F302FB13007330C0B204F0ADFEBBF8B6
:104EA0000030032B7EF62BABBAF8003099F80000E7
:104EB0000C22C11A91FBF2F302FB131302FB034411
:104EC000A36818447F287FF7B1AA7F3890FBF2F3DC
:104ED00002FB13007330FFF73BB9FBF7D3FBFFF77F
:104EE00090B9DFF8FCA03749BAF800203B4C9A1A79
:104EF00081FB0210D117C1EB600101EB4101A2EB74
:104F0000810202EB420254F8220018447F2840F349
:104F1000D080A0F17F030C2093FBF0F200FB123055
:104F20007330DFF8C4B098F80010C0B204F040FE4F
:104F3000BBF80030022B1AD93868BAF800300C22BE
:104F4000C11A91FBF2F302FB131302FB03435B68EC
:104F500018447F2840F3C4837F3890FBF2F302FBB0
:104F600013007330C0B298F8001004F021FEBBF8B3
:104F70000030032B7FF616AABAF8003038680C22EE
:104F8000C11A91FBF2F302FB131302FB0344A36863
:104F900018447F287FF74DAA7F3890FBF2F302FB7D
:104FA00013007330FFF7F9B9FBF76CFBFFF7A5B8F7
:104FB000012B3DF4EEAE0124FFF715BAFBF762FBBF
:104FC000FFF7C1B9ABAAAA2AD42A010060310100B7
:104FD000949FFF1F059DFF1F409FFF1F283001006A
:104FE0003C9FFF1FC19DFF1F429DFF1FDFF800A3D5
:104FF00099F80000BAF80030B34AB44CC31A82FBE7
:105000000321DA17C2EB610202EB4202A3EB820337
:1050100003EB430354F8233018447F2846DD7F38E0
:105020000C2290FBF2F302FB13007330DFF8CCB2DA
:10503000C0B204F0E1FDBBF80030022B19D999F899
:105040000000BAF800300C22C11A91FBF2F302FB07
:10505000131302FB03435B6818447F2840F38B80E3
:105060007F3890FBF2F302FB13007330C0B204F000
:10507000C3FDBBF80030032B7EF6D6AEBAF8003085
:1050800099F800000C22C11A91FBF2F302FB1313F2
:1050900002FB0344A36818447F287FF79FAD7F3845
:1050A00090FBF2F302FB1300733089E5FBF7EAFA99
:1050B000BCE7FBF7E7FA34E7FBF7E4FA62E4FBF757
:1050C000E1FAFFF7DBBBFBF7DDFAC5E6FBF7DAFA3F
:1050D0005CE6FBF7D7FA4DE5FBF7D4FACDE4DFF851
:1050E00010A23868BAF80030774A794C35E6DFF814
:1050F00000A299F80000BAF80030734A744C92E6A6
:10510000FBF7C0FAFFF714BADFF8E4A199F8000042
:10511000BAF800306C4A6F4C70E7FBF7B3FAFFF750
:1051200022BBFBF7AFFAFFF79FBADFF8C4A16649CD
:10513000BAF80020664CDAE6029B1B78002B7EF45E
:10514000BEA9FEF7E1B9644B1B78002B00F0298360
:10515000624B1B78002B7DF41CAE614B1B78002B3F
:105160003DF417AEB8F800305E490A33A8F80030B5
:105170000A70FDF70EBEFBF785FA77E75A4C2288D6
:10518000002A00F02C835949DFF870B10988BBF878
:1051900000000331884227DD554856490088B1F8A0
:1051A00000E0DFF854C1181A0C2190FBF1F901FB63
:1051B00019004FF0900909FB0EFE01FB00E06FF0B3
:1051C0000B0E5CF8000003440EFB02307F2840F316
:1051D00032857F3890FBF1F301FB13007330C0B2CE
:1051E00098F8001004F0E4FCBBF800202388134476
:1051F000022B23DD3E4B3F4A38681B88B2F800C0C3
:10520000DFF8F4E0C31A0C2193FBF1F201FB123238
:10521000902303FB0CF301FB023373445B681844D7
:105220007F2840F362857F3890FBF1F301FB130088
:105230007330C0B298F8001004F0BAFCBBF800203C
:1052400023881344032B23DD294B2A4A38681B8803
:10525000B2F800C0DFF8A0E0C31A0C2193FBF1F212
:1052600001FB1232902303FB0CF301FB0233734466
:105270009B6818447F2840F353857F3890FBF1F3F7
:1052800001FB13007330C0B298F8001004F090FCDA
:10529000BBF8002023881344042B7FF783A8134B0B
:1052A0001B88012B7FF47EA83A68A2F10C007F28AE
:1052B0007FF7BFA88B3A0C2092FBF0F300FB132082
:1052C0007330FFF76AB800BFABAAAA2AF031010019
:1052D000E4320100D42A0100E79FFF1FE89FFF1F6F
:1052E000E99FFF1F2C9DFF1FC89DFF1F5E9DFF1F95
:1052F0003C9FFF1FEE9EFF1F642B0100429DFF1F7E
:10530000C74C2388002B40F06D82DFF83CB3C549C1
:10531000C54A0988D7F80080B2F800E0C348C1EB5D
:10532000080C0C229CFBF2F102FB11C14FF0900C17
:105330000CFB0EFE02FB01E16FF00B0E40588044A7
:105340000EFB03807F2840F37284A0F17F0393FB60
:10535000F2F002FB10307330B54BC0B2197804F094
:1053600027FCBBF8002023881344022B23DDAD4A21
:10537000AD4B11883868B3F800C0DFF8B0E2411ACD
:105380000C2291FBF2F302FB1311902303FB0CF3AD
:1053900002FB013373445B6818447F2840F30D859A
:1053A0007F3890FBF2F302FB13007330A04BC0B2C6
:1053B000197804F0FDFBBBF8002023881344032B6D
:1053C00023DD984A984B11883868B3F800C0DFF89D
:1053D0005CE2411A0C2291FBF2F302FB13119023C1
:1053E00003FB0CF302FB013373449B6818447F28D2
:1053F00040F39D847F3890FBF2F302FB130073307F
:105400008B4BC0B2197804F0D3FBBBF80020238883
:105410001344042B7EF706AA864B1B88012B7EF4CF
:1054200001AA3A68A2F10C007F2840F3D5818B3A9B
:105430000C2092FBF0F300FB132073307C4BC0B2C6
:10544000197804F0B5FBFEF7EDB9754C2388002BF5
:1054500040F0D381DFF8F0B17249734A098899F8B6
:105460000000B2F800E0DFF8C481C1EB000C0C22B0
:105470009CFBF2F102FB11C14FF0900C0CFB0EFEF5
:1054800002FB01E16FF00B0E58F8011008440EFB0F
:1054900003007F2840F3C883A0F17F0393FBF2F061
:1054A00002FB10307330C0B204F0A6FBBBF8002042
:1054B00023881344022B22DD5A4A5B4B118899F84A
:1054C0000000B3F800C0DFF864E1411A0C2291FB40
:1054D000F2F302FB1311902303FB0CF302FB0133E5
:1054E00073445B6818447F2840F36B847F3890FBDB
:1054F000F2F302FB13007330C0B204F07DFBBBF883
:10550000002023881344032B22DD464A464B118892
:1055100099F80000B3F800C0DFF810E1411A0C223E
:1055200091FBF2F302FB1311902303FB0CF302FB3C
:10553000013373449B6818447F2840F3F5837F3818
:1055400090FBF2F302FB13007330C0B204F054FB83
:10555000BBF8002023881344042B7DF7D0AF354BD4
:105560001B88012B7DF4CBAF99F80020A2F10C0031
:105570007F287EF75BAF8B3A0C2092FBF0F300FBA9
:1055800013207330FEF7E4BDDFF898A099F800000F
:10559000BAF80030284CC11A0C2291FBF2F302FB3E
:1055A000131302FB03F3E35818447F287FF77EAD03
:1055B0007F3890FBF2F302FB1300733036E51F4B8C
:1055C0001B88182B12D099F800201344A3F118005F
:1055D0007F2840F3A2830C20973B93FBF0F200FB63
:1055E000123303F17300C0B204F006FB144A154BEA
:1055F000127833F81230182B3DF481AF99F800205F
:105600001344A3F118007F287EF710AF0C20973BBE
:1056100093FBF0F200FB123303F17300FEF798BD29
:10562000C89DFF1F3C9FFF1FEE9EFF1F642B0100C4
:10563000C19DFF1F5E9DFF1F28300100929FFF1F2D
:10564000BC89FF1F589FFF1F429DFF1FB64B1A8842
:10565000182A13D03B681344A3F118007F2840F3A5
:105660004B830C20973B93FBF0F200FB123303F1CA
:105670007300AE4BC0B2197804F09AFAAC4BAD4946
:105680001A78022A94BF013200221A701A7831F86F
:105690001200182810D10424022A02F10100C2B21B
:1056A00088BF002231F81200182804D1013CF3D140
:1056B0001A70FEF7B7B81A703B680344A3F11800DC
:1056C0007F2840F389800C20973B93FBF0F200FB8E
:1056D000123303F17300B1E6FAF7D4FFFFF7DCBB36
:1056E000FAF7D0FF3EE4FAF7CDFFFFF772BB924B1B
:1056F0001B78002B7DF44DAB904B1B78002B3DF4B9
:1057000048ABB8F800308E49013BA8F800300A7069
:10571000FDF73FBB844A1288182A12D01344A3F124
:1057200018007F2840F3E5820C20973B93FBF0F2B2
:1057300000FB123303F17300C0B298F8001004F0BC
:1057400037FA7B4B7B491A78022A94BF0132002238
:105750001A701A7831F81200182811D10424022A7C
:1057600002F10100C2B288BF002231F812001828ED
:1057700005D1013CF3D11A703B68FEF797B91A7056
:105780003B680344A3F118007F287EF752AE0C203B
:10579000973B93FBF0F200FB123303F17300FEF72B
:1057A000FCBD654B1B78002B7DF48DAF634B1B78E4
:1057B000002B3DF4EEAAB8F8003061490133A8F897
:1057C00000300A70FDF7E5BADFF888A199F800000B
:1057D000BAF800305B4CDEE6FAF754FF2EE6DFF84D
:1057E00078B1D9E4584ADFF870B11288BBF80010DC
:1057F000033291427FF7B5AD89E5534ADFF858B1DE
:105800001288BBF80010033291427FF74FAE23E6B7
:105810004E4B1B88182B12D099F800201344A3F18B
:1058200018007F2840F3C6820C20973B93FBF0F2D0
:1058300000FB123303F17300C0B204F0DDF93C4AFF
:10584000434B127833F81230182B7FF4D7AEFDF7A4
:1058500056BE3E4B1A88182A13D03B681344A3F156
:1058600018007F2840F33E820C20973B93FBF0F218
:1058700000FB123303F173002C4BC0B2197804F013
:1058800097F92B4B32491A78022A94BF0132002231
:105890001A701A7831F8120018287FF40DAF04241A
:1058A000022A02F1010294BFD2B2002231F81200A2
:1058B00018287FF400AF013CF2D11A70FDF7B2BF97
:1058C000224A1288182A12D01344A3F118007F2804
:1058D00040F3E6810C20973B93FBF0F200FB123380
:1058E00003F17300C0B298F8001004F061F9104B96
:1058F00017491A78022A94BF013200221A701A78C6
:1059000031F8120018287FF43BAF0424022A02F178
:10591000010294BFD2B2002231F8120018287FF49D
:105920002EAF013CF2D126E7929FFF1FC19DFF1FC2
:10593000BC89FF1F589FFF1FE89FFF1FE99FFF1FA4
:105940002C9DFF1FE43201005E9DFF1F569DFF1F2F
:10595000D09EFF1F3C9FFF1F429DFF1FD24C2388FC
:10596000002B40F0CF81DFF878B3D04999F80000E0
:10597000CF4A09881788DFF83CE3411A0C2291FBD3
:10598000F2FC02FB1C114FF0900C0CFB07F702FB22
:1059900001716FF00B075EF80110014407FB031063
:1059A0007F2840F3AC817F3890FBF2F302FB1300B9
:1059B0007330C0B204F020F9BBF8002023881344F0
:1059C000022B21DDB94BBA4A99F800001B88B2F8C6
:1059D00000E0B84FC31A0C2193FBF1F201FB123225
:1059E000902303FB0EF301FB02333B445B68184436
:1059F0007F2840F3F3817F3890FBF1F301FB130024
:105A00007330C0B204F0F8F8BBF8002023881344C8
:105A1000032B21DDA54BA64A99F800001B88B2F89C
:105A200000E0A44FC31A0C2193FBF1F201FB1232E8
:105A3000902303FB0EF301FB02333B449B681844A5
:105A40007F2840F3D7817F3890FBF1F301FB1300EF
:105A50007330C0B204F0D0F8BBF8002023881344A0
:105A6000042B7EF7E1A9944B1B88012B7EF4DCA963
:105A700099F80020A2F10C007F287FF7AFA88B3A9D
:105A80000C2092FBF0F300FB13207330FFF798B863
:105A90008A4B01227F2107201A8004F059F87F21C8
:105AA0000B2004F055F8FDF739BE854B04227F2109
:105AB00007201A8004F04CF800210B2004F048F86D
:105AC000FDF725BE7E4B02227F2107201A8004F0BD
:105AD0003FF87F210B2004F03BF8FDF713BE784B15
:105AE000002107201C8004F033F87F210B2004F0F4
:105AF0002FF8FDF702BE734B00227F2107201A808A
:105B000004F026F87F210B2004F022F8FDF70EBEEA
:105B10006D4B1A88182A13D03B681344A3F1180060
:105B20007F2840F364810C20973B93FBF0F200FB4D
:105B3000123303F17300654BC0B2197804F038F8E2
:105B4000634B64491A78022A94BF013200221A700A
:105B50001A7831F8120018287FF4AEAD0424022A16
:105B600002F1010294BFD2B2002231F812001828CB
:105B70007FF4A1AD013CF2D11A70FDF753BE524A39
:105B80001288182A12D01344A3F118007F2840F37A
:105B900022810C20973B93FBF0F200FB123303F1C0
:105BA0007300C0B298F8001004F002F8484B49495D
:105BB0001A78022A94BF013200221A701A7831F83A
:105BC000120018287FF4DCAD0424022A02F101023D
:105BD00094BFD2B2002231F8120018287FF4CFAD62
:105BE000013CF2D1C7E5384B1B88182B12D099F82D
:105BF00000201344A3F118007F2840F3E9800C2013
:105C0000973B93FBF0F200FB123303F17300C0B239
:105C100003F0F2FF2E4A2F4B127833F81230182B74
:105C20007FF4ECACFDF76BBCFAF72CFD3BE4FAF724
:105C300029FDFFF791BBFAF725FDFFF7D0BA264BF8
:105C40001B88182B12D099F800201344A3F11800D8
:105C50007F2840F3C6800C20973B93FBF0F200FBBB
:105C6000123303F17300C0B203F0C6FF184A1B4B96
:105C7000127833F81230182B3EF4D6A899F8002089
:105C80001344A3F118007F287EF7A8AF0C20973BA0
:105C900093FBF0F200FB123303F17300FEF790BFA9
:105CA000FAF7F0FC1EE600BFC89DFF1F3C9FFF1FD8
:105CB000EE9EFF1F642B01005E9DFF1FDA9DFF1FFC
:105CC000349FFF1F249DFF1F589DFF1FC19DFF1F75
:105CD000BC89FF1FD89EFF1F929FFF1F589FFF1F69
:105CE000429DFF1FFAF7CEFCC6E5FAF7CBFCFFF7A3
:105CF000A0BAFAF7C7FC1FE5FAF7C4FCB9E4FAF753
:105D0000C1FC56E6404ADFF81CB11288BBF800100F
:105D1000033291427FF750AE27E6FAF7B3FC62E414
:105D2000FAF7B0FCFFF7AFBAFAF7ACFC0DE4FAF7FC
:105D3000A9FCFFF765BB354B1B88182B11D099F8D0
:105D400000201344A3F118007F284DDD0C20973B61
:105D500093FBF0F200FB123303F17300C0B203F0C7
:105D60004BFF2B4A2B4B127833F81230182B85D16E
:105D7000FEF75AB8284B1B88182B11D099F8002031
:105D80001344A3F118007F281FDD0C20973B93FBE1
:105D9000F0F200FB123303F17300C0B203F02CFFEA
:105DA0001B4A1E4B127833F81230182B7FF466AF63
:105DB000FEF73AB8FAF766FC3EE5FAF763FCFFF740
:105DC000F5BAFAF75FFCFFF797BBFAF75BFCE4E77D
:105DD000FAF758FC1BE7FAF755FCE2E6FAF752FC33
:105DE0000FE6FAF74FFC3EE7FAF74CFCB6E7FAF796
:105DF00049FCA0E6FAF746FC2BE6094B0293FDF7B7
:105E000013BF0A60FDF7F9BB5E9DFF1F589DFF1F82
:105E1000BC89FF1FD89EFF1F569DFF1FD09EFF1FEE
:105E2000EA9DFF1F429DFF1F38B507F09FFE0E48F9
:105E300005F0D6FD0D4805F0D3FD0D4805F0D0FD69
:105E400000234FF07E5201210A48FAF70FFB0A4B5C
:105E50000A4A0B49802400251C7118461D60BDE8C4
:105E600038400BF087BC00BF409DFF1F749DFF1F93
:105E7000E09DFF1F109FFF1FA09FFF1F1C89FF1F9A
:105E80002906000010B50446A4206368198803F0B1
:105E9000B9FFE368A6201988BDE8104003F0B2BF3F
:105EA00043682A20198803F0ADBF00BF10B504462F
:105EB00022206368198803F0A5FFE368242019886D
:105EC000BDE8104003F09EBF10B504460A20636889
:105ED000198803F097FFE3680C201988BDE810408B
:105EE00003F090BF10B5044606206368198803F0DC
:105EF00089FFE36808201988BDE8104003F082BFDD
:105F000010B5044602206368198803F07BFFE3683C
:105F100004201988BDE8104003F074BF70B50E4C22
:105F200084B01225042201230646039002932046E2
:105F30008DE824001423102106F056FF06220923C1
:105F4000029303960195204600921423102106F037
:105F50004BFF04B070BD00BF1CA0FF1FF8B5B04CD4
:105F6000B4F90030032B00F01281002B6AD0022B11
:105F700000F08A80052B00F0B580012B00F0DD8059
:105F8000042B00D0F8BDA74FA74E00254FF4AF74E7
:105F9000E9B2A64805F08CFD57F8043BC3F59673AB
:105FA00000FB03F086FB0023C017C0EB63108442A4
:105FB00005F10105A8BF0446062DE9D19C4F9A4E74
:105FC0000025E9B29B4805F073FD57F8043BC3F583
:105FD000967300FB03F086FB0023C017C0EB631031
:105FE000844205F10105A8BF04460C2DE9D1924F6A
:105FF0008D4E0025E9B2914805F05AFD57F8043B53
:10600000894AC3F5967300FB03F086FB0013C017A3
:10601000C0EB6310844205F10105A8BF04460C2DB6
:10602000E8D1A4F11401312900F3A38040F26C728D
:1060300032218348834B01801A602A20BDE8F84052
:1060400003F0E0BE0E2007F0F5FC40F6FF71C8300B
:106050008842A8BF084620EAE07000F2DC5283B212
:106060008A42794D794EA8BF0A46022019463380EC
:106070002A8003F0C7FE2988042003F0C3FEB4F988
:106080000030022B7FF476AF012008F0EFFD0546CB
:10609000002008F0EBFDA842B8BF284600F1C80177
:1060A000B1F5FA7FC0F2B480B1F57A6FA8BF4FF4B2
:1060B0007A6101F54873B3F57A6FA8BF4FF47A633C
:1060C0009BB289B2624A634D11800A202B8003F093
:1060D00099FE29880C2003F095FEB4F90030052BB9
:1060E0007FF44BAF0F2008F0C1FDC0F53F630433D0
:1060F000B3F5AF6FC0F28980B3F5FA6FA8BF4FF464
:10610000FA6399B2544BC0F54360B0F5AF6F198094
:1061100061DBB0F5FA6FA8BF4FF4FA6083B24F4D60
:10612000A4202B8003F06EFE2988A62003F06AFECF
:10613000B4F90030012B7FF423AF152007F07AFC6F
:1061400000F59671B1F52F7F4DDB41F25C2399424A
:1061500063DC434A00F5617089B2B0F52F7F11808E
:10616000B8BF4FF42F7344DB8342A8BF03469BB2F2
:106170003FE040F23A73A4F5B97403FB04F482FBE8
:106180000432E417A4EB621289B2323251E71020D4
:1061900008F06CFDC830B0F5FA7F1FDBB0F57A6F00
:1061A0000146A8BF4FF47A6101F51673B3F57A6F13
:1061B000A8BF4FF47A639BB289B22A4A2A4D118054
:1061C00022202B8003F01EFE2988242003F01AFED3
:1061D000B4F90030C9E64FF4AF63A0E740F24C4396
:1061E0004FF4FA71E9E740F214534FF42F711C4A4F
:1061F00011801E4D06202B8003F004FE2988082004
:1062000003F000FEB4F90030BAE64FF4AF6179E76D
:1062100040F214534FF4FA7154E71946E7E700BF10
:10622000F69FFF1F4C8AFF1FB5814E1B409DFF1F2D
:106230001C8AFF1F749DFF1F2C89FF1FE09DFF1FFD
:10624000AC9FFF1F088AFF1FB29FFF1FE89DFF1F23
:10625000489FFF1F549DFF1FEC9DFF1F689FFF1F5E
:106260008E9DFF1FFC9EFF1FF89EFF1F7C9FFF1F40
:106270002DE9F041224D82B0012602B284B2009293
:10628000284601967823192106F0F4FC04F10C024B
:1062900012B28DE844002846A7197823192104F189
:1062A000020806F0E7FC3FB20FFA88F819233A46D5
:1062B000284619460196CDF8008006F0DBFC7823CD
:1062C0003A4628461946CDF80080019604F10A079F
:1062D0000B3406F0CFFC3FB224B278233A4628466E
:1062E00019468DE8500006F0C5FC192300943A4683
:1062F00001962846194606F0BDFC02B0BDE8F081C3
:106300001CA0FF1F30B583B000230C4605B20093DC
:1063100026225B231C210C4806F0FCF929460123A8
:106320002622094805F006FD002C24B205DB214693
:1063300001232622044805F0FDFC044A044B158085
:106340001C8003B030BD00BF1CA0FF1F668AFF1F6A
:10635000688AFF1F2DE9F041BB4C237882B01BB146
:10636000BA4B4FF6FF721A80B94BB3F90030CBB974
:10637000B84AB64B1068B3F9002080F30C005B23D9
:1063800003FB00F000131C3082424BD04FF0FF3172
:10639000FFF7B8FFB04806F021FA0023237002B0DF
:1063A000BDE8F081012B1BD0022B5AD0032B3FD02C
:1063B000042B00F09980052BEFD10F2008F056FC3C
:1063C000C0F53B600830B0F5AF6F48DBB0F5FA6F51
:1063D000A8BF4FF4FA60A0F5AF625B239F4835E099
:1063E0009F4B1B78002B75D0152007F023FB9D4B8E
:1063F0001860B0F52F7F32DB41F25C239842A8BFD2
:106400001846A0F52F735B22974802FB03F380FB2D
:106410000320DB17C3EBA0201C308C4BB3F90030FA
:106420008342B3D1914BB3F900300133AED1B4E71D
:106430008F4B1B68B3F5FA7F11DBB3F57A6FA8BFFA
:106440004FF47A638B48A3F5FA725B2303FB02F3E4
:1064500080FB0320DB17C3EB20201C30DDE71C2072
:10646000DBE7854B1B68B3F5FA7F3BDBB3F57A6F4F
:10647000A8BF4FF47A63A3F5FA727E485B2303FB4F
:1064800002F380FB0320DB17C3EB20201C307B4B87
:106490001B68B3F5FA7F23DBB3F57A6FA8BF4FF41F
:1064A0007A63A3F5FA7273495B2303FB02F381FB62
:1064B0000321DB17C3EB21211C31644BB3F90030FE
:1064C00083427FF465AF694BB3F900308B427FF4B0
:1064D0005FAF62E7112008F0C9FB624B186088E7E4
:1064E0001C21EAE71C20D2E7252200258DE82400A4
:1064F00076231C215848624E624FDFF8A08106F0D7
:10650000B9FB16E0B0F5AF7FA8BF4FF4AF703238DB
:1065100002FB00F088FB0031C017C0EB61111C3199
:1065200009B201231D4425224B4805F003FC0C2D24
:1065300014D0E9B2544805F0BBFA56F8043BC3F551
:10654000967300FB03F087FB0013C017C0EB6310CA
:1065500031284FF05B02D5DC1C21E2E72622002522
:106560008DE8240076231C213B48484E454FDFF838
:106570002C8106F07FFB16E0B0F5AF7FA8BF4FF48B
:10658000AF70323802FB00F088FB0031C017C0EB5F
:1065900061111C3109B201231D4426222E4805F049
:1065A000C9FB0C2D14D0E9B2394805F081FA56F830
:1065B000043BC3F5967300FB03F087FB0013C01781
:1065C000C0EB631031284FF05B02D5DC1C21E2E701
:1065D000272200258DE8240076231C211E482D4EFD
:1065E000284FDFF8B88006F045FB17E0B0F5AF7F25
:1065F000A8BF4FF4AF70323802FB00F088FB0031C7
:10660000C017C0EB61111C3109B201231D442722C0
:10661000114805F08FFB062D3FF4BCAEE9B21E48D1
:1066200005F046FA56F8043BC3F5967300FB03F0F9
:1066300087FB0013C017C0EB631031284FF05B02DB
:10664000D4DC1C21E1E700BFF09FFF1F668AFF1F1B
:10665000F69FFF1F4C9FFF1F1CA0FF1F37800B6D75
:10666000049FFF1F109DFF1FD3058541688AFF1FF0
:10667000649DFF1F011FB812709DFF1F349DFF1FF7
:106680001C8AFF1FB5814E1B749DFF1F2C89FF1FA5
:10669000E09DFF1F4C8AFF1F409DFF1F4B48371B8B
:1066A0002DE9F041044682B071482768E56805F09D
:1066B00089FF1120FFF7DCFD012619234FF0280880
:1066C000194624226A480196CDF8008006F0D2FAD5
:1066D00078231946242266480196CDF8008006F0FA
:1066E000C9FA3146624806F05BFE02221921604871
:1066F00006F052FE38460BF003FE394602465C486F
:1067000006F0E4FF5A4806F0F7FF1422002158482B
:1067100006F042FE03225749554806F0D7FF544879
:1067200006F0EAFF23220021514806F035FE03223D
:1067300051494F4806F0CAFF4D4806F0DDFF7DB1D4
:106740002F20FFF795FD32220021494806F024FE54
:1067500003224A49464806F0B9FF454806F0CCFFF7
:106760000123474A18461370FFF7D8FB2189638934
:1067700062685B1A5C2B128854DD521A02EB4202EB
:10678000C2EB4212013392FBF3F31B333D4A38480C
:10679000138001261A221BB28DE8440019461422E8
:1067A00006F068FA002D4FD0218A638AE2685B1AEE
:1067B0005C2B12883EDC511A5C2202FB01F292FB38
:1067C000F3F31B33304A2A48138001251BB23822C9
:1067D00019468DE82400322206F04CFA40230022AC
:1067E00009218DE806002248194606F011FA2946CB
:1067F0001F4806F0D5FD022244211D4806F0CCFDBD
:1068000063681B48198806F0C7FF2A461F491848C5
:1068100006F05CFFE3681648198802B0BDE8F04155
:1068200006F0BABF511A5C2202FB01F292FBF3F3AD
:106830001B33ABE7521A02EB4202C2EB4212334463
:1068400092FBF3F31B33BDE7402309212A46009155
:1068500007480195194606F0DBF93146044806F071
:106860009FFD02226821024806F096FD6368D2E788
:106870001CA0FF1F4C3401005034010054340100AF
:1068800095A0FF1FF29FFF1FF49FFF1F58340100C8
:106890002DE9F0471F4682B01446002A4ED0052A43
:1068A0000646D0F80C8000F0AB800B9B894A00EBC9
:1068B000C305012CB5F80AE029896868C1EB0E030D
:1068C00082FB03C21A444FEAE373C3EBA2130288AC
:1068D00051D0042C00F08D800022402309218DE846
:1068E00006007D48194606F093F901217A4806F022
:1068F00057FD0222B8F1000F00F0E18044217648F4
:1069000006F04AFD73687448198806F045FF73491C
:106910007148012206F0DAFEF3686F48198806F024
:106920003BFF6F4B022CB3F9001000F0A680082C3F
:1069300000F0C280012002B0BDE8F087694E6A4ACB
:1069400033681268CB1A93420D4655D9674A3B8883
:1069500011786148012918BF012414700A9A06327F
:106960001BB212B28DE814001946BDF9282006F0BA
:1069700081F93560DEE79BB2D31A994203DC9E456C
:106980007146A8BF19460A9A0180B7F90030BDF9CF
:1069900028A0514802F106094FF0000E0FFA89F9BC
:1069A00019465246CDF80090CDF804E006F062F9A1
:1069B00029896A896868521A03885C2AA3EB010353
:1069C00073DD03EB43030132C3EB431393FBF2F399
:1069D00003F11B0213B201203A801946524601907E
:1069E000CDF800903C4806F045F9404B00221A7063
:1069F00072E712FA83F3C0E7204602B0BDE8F087E1
:106A000007254FF000095A2323228DE820021A217E
:106A1000314806F0FDF801212F4806F0C1FC0121A4
:106A20002D4806F0C3FC232235212B4806F0B4FC88
:106A30002A462F49284806F049FE274806F05CFE02
:106A4000254805F0CBFE4FF4FA6007F045FDFFF74F
:106A500085FA5A2323221A218DE820021E4806F0C7
:106A6000D7F81D4805F0BAFE3046FFF719FE214B56
:106A700001221A70FFF76EFC2EE74A1C12B21A8030
:106A800091423FF457AF0A9AB7F9003012480632E4
:106A9000012412B2009219460194BDF9282006F093
:106AA000E9F8204602B0BDE8F0875C2101FB03F362
:106AB00093FBF2F21B328DE700221A80E0E7682197
:106AC000054806F069FC73680348198806F064FEFF
:106AD00027E700BFC94216B21CA0FF1F58340100AF
:106AE000FA9FFF1F80A0FF1F5044010095A0FF1FC9
:106AF0005C340100F09FFF1F2DE9F04F5A4E5B4DB3
:106B0000B6F900704C7855F8277085B081469846E4
:106B100004B10C78DFF874A11AB99AF80030002B90
:106B200039D0534D002338462B808AF80030FFF7C8
:106B3000B7FD504A504BB5F90000012111704FF6D6
:106B4000FF721A8060B301285ED0012032232246F2
:106B5000019000934946494B3846FFF799FE0024BF
:106B60000346B5F90020022A39DD00222A80B6F951
:106B700000203D49002A3BDB052AC4BF00220A80D1
:106B8000B8F1000F39D1002C0CBF18464FF0FF3080
:106B900005B0BDE8F08F364DB5F900000028D2D120
:106BA000DFF8ECB0364ADBF800301268C3EB0903BB
:106BB000934227D9334B1A78012A18BF0120187045
:106BC000FFF7ACF90123CBF80090012C2AD0042C5C
:106BD00035D0022C3AD0082C3ED00024C1E7C6D1D3
:106BE000FA68002AC1D0B6F900201F49002AC3DA8A
:106BF00005220A80B8F1000FC5D00393FFF7AAFB66
:106C0000039BC0E70346E0E74FF0000E1423224643
:106C10008DE8084049461C4B38467446FFF738FE5D
:106C200003469EE732888AF80040013232807A6952
:106C300082B10024384603939047039B91E7328842
:106C40000121013A32808AF80010F0E701222A80FF
:106C500000248CE7144684E77A69002129804FF0EC
:106C6000FF34002AE6D182E7F69FFF1F6C8AFF1FE0
:106C7000FA9FFF1FF09FFF1F668AFF1FF49FFF1FF1
:106C80005044010095A0FF1FF29FFF1FF89FFF1FB8
:106C900080A0FF1F01210D2007F0E2BB00210D2085
:106CA00007F0DEBB01460D2007F0DABB08B50D206A
:106CB00007F0DCFBB0FA80F149090D20BDE808407F
:106CC00007F0CEBB10B5002144080D2007F0C8FB2B
:106CD000204607F001FC0D20012107F0C1FB2046F2
:106CE000BDE8104007F0F8BB2D4A2E4B10881B68FA
:106CF000984210B549DA2C4A1288141A9A42A8BF51
:106D00001A46B4F5157F36DA121A40F2532303FB04
:106D100002F393FBF4F105310A2007F011FA234B3B
:106D20001978C9B3224B23491B6840F2271283F319
:106D3000070302FB03F381FB03211944DB17C3EBB9
:106D4000A1110531092007F0FBF91B4B1968F1B1BE
:106D500081F3070140F22712164802FB01F380FB82
:106D600003211944DB17C3EBA11105311620BDE83F
:106D7000104007F0E5B9131A4FF41572611C02FBBD
:106D800003F393FBF1F10531C6E70021C4E71620B8
:106D9000BDE8104007F0D4B9092007F0D1F9D4E7D5
:106DA000E89DFF1F089DFF1FB29FFF1F929DFF1FC1
:106DB000989FFF1F09040281649FFF1F7F2838B539
:106DC000A8BF7F200F4C4FF4167202FB00F284FB29
:106DD00002311144D2170546C2EBA1110A2007F077
:106DE000AFF97F3D4FF4967303FB05F384FB03215A
:106DF0001944DB17A3EBA1110920BDE8384007F0C7
:106E00009FB900BF09040281C368B3F9003030B5EF
:106E100083EAE374A4EBE374002BA0B218DB012334
:106E200000E0134603EB830252009442F9DA0A4D64
:106E300090FBF3F285FB03E403FB1200DB17303217
:106E4000D3EBA40380B201F8012BF1D10B7030BD5C
:106E50002D230B700131E2E76766666638B5094D90
:106E60008224204602F0E8FF35F8021B00B2884277
:106E7000204601D002F0C6FF0234A4B28A2CF0D121
:106E800038BD00BFD89EFF1F024B8020198802F03A
:106E9000B9BF00BF589DFF1F38B5094D7824204663
:106EA00002F0CAFF35F8021B00B28842204601D02A
:106EB00002F0A8FF0234A4B2802CF0D138BD00BF8C
:106EC000D09EFF1F024B7620198802F09BBF00BFA7
:106ED000569DFF1F38B5094D4624204602F0ACFFF1
:106EE00035F8021B00B28842204601D002F08AFF2A
:106EF0000234A4B24E2CF0D138BD00BF589FFF1F02
:106F0000024B4420198802F07DBF00BF929FFF1FF3
:106F1000024B4E20198802F075BF00BF6A9DFF1F0B
:106F2000024B9A20198802F06DBF00BFC89DFF1F59
:106F3000024B9820198802F065BF00BF5E9DFF1FBD
:106F4000024B8C20198802F05DBF00BFEE9EFF1F30
:106F5000024B9C20198802F055BF00BF429DFF1FC5
:106F6000024BA020198802F04DBF00BF609FFF1F99
:106F7000024B9620198802F045BF00BF3C9FFF1FBF
:106F8000024B8A20198802F03DBF00BF029FFF1FFD
:106F9000024B1020198802F035BF00BF009FFF1F71
:106FA000024B2C20198802F02DBF00BF3E9DFF1F11
:106FB000024B1E20198802F025BF00BF5C9DFF1FF9
:106FC000C3680E20198802F01DBF00BF024B2820A5
:106FD000198802F017BF00BF569FFF1F024B6420A5
:106FE000198802F00FBF00BF509FFF1F024BB42053
:106FF000198802F007BF00BFA89FFF1F024BB620F1
:10700000198802F0FFBE00BFD89FFF1F024B5A2015
:10701000198802F0F7BE00BF189DFF1F024B162013
:10702000198802F0EFBE00BF249DFF1F024B2E20E7
:10703000198802F0E7BE00BFD09DFF1F024B302031
:10704000198802F0DFBE00BFC09FFF1F024B9E20C9
:10705000198802F0D7BE00BFC489FF1F024BAC20C5
:10706000198802F0CFBE00BF529FFF1F024BAE2017
:10707000198802F0C7BE00BF689DFF1F024BB020F9
:10708000198802F0BFBE00BFE49EFF1F024BB22072
:10709000198802F0B7BE00BF869DFF1F024B182063
:1070A000198802F0AFBE00BFEE9DFF1F024BA22069
:1070B000198802F0A7BE00BF869FFF1F024B1A204F
:1070C000198802F09FBE00BF769DFF1F024B1C2057
:1070D000198802F097BE00BF6C9DFF1F024B66200F
:1070E000198802F08FBE00BF909FFF1F024B7220D5
:1070F000198802F087BE00BFBC9FFF1F024B2020F3
:10710000198802F07FBE00BF8E9FFF1F024B322006
:10711000198802F077BE00BF7E9FFF1F024B6820D8
:10712000198802F06FBE00BFB09DFF1F024B6C209C
:10713000198802F067BE00BF0C9DFF1F024B6E2036
:10714000198802F05FBE00BFEE9FFF1F024B522066
:10715000198802F057BE00BF5E89FF1F024B502006
:10716000198802F04FBE00BF2089FF1F024B542038
:10717000198802F047BE00BF188AFF1F024B5C202F
:10718000198802F03FBE00BF648AFF1F024B5E20D9
:10719000198802F037BE00BF5C89FF1F024B5620E2
:1071A000198802F02FBE00BFBE9DFF1F244B1B8815
:1071B0000B2B43D8DFE803F00B10151A1F24292EE0
:1071C00033383D06084604221E490BF057B90846DD
:1071D00004221D490BF052B9084604221B490BF04A
:1071E0004DB9084604221A490BF048B90846042252
:1071F00018490BF043B90846042217490BF03EB971
:107200000846042215490BF039B9084604221449EE
:107210000BF034B90846042212490BF02FB9084686
:10722000042211490BF02AB9084604220F490BF039
:1072300025B9084604220E490BF020B9704700BF5B
:107240003C9FFF1FF0400100443E0100AC3C0100A8
:10725000E03D0100B03C010034420100B43C0100BB
:10726000B83C0100883F0100BC3C0100FC4001002B
:10727000C03C0100064B074A10B41C88064B084668
:10728000002C14BF11461946042210BC0BF0F6B8AE
:107290008C9DFF1FC43C0100C83C0100064B074AFF
:1072A00010B41C88064B0846002C14BF1146194622
:1072B000042210BC0BF0E2B8D29DFF1FC43C0100B9
:1072C000C83C0100064B074A10B41C88064B084610
:1072D000002C14BF11461946042210BC0BF0CEB886
:1072E000F69EFF1FC43C0100C83C0100064B074A44
:1072F00010B41C88064B0846002C14BF11461946D2
:10730000042210BC0BF0BAB83E9FFF1FC43C010022
:10731000C83C0100064B074A10B41C88064B0846BF
:10732000002C14BF11461946042210BC0BF0A6B85D
:10733000DA9DFF1FC43C0100C83C01001B4B1B88A9
:107340000A2B0AD8DFE803F00A0E12161A1E2226AC
:107350002A2E0600164B186808607047154B1868EF
:1073600008607047144B186808607047134B186822
:1073700008607047124B186808607047114B186816
:1073800008607047104B1868086070470F4B18680A
:10739000086070470E4B1868086070470D4B1868FE
:1073A000086070470C4B186808607047029FFF1F09
:1073B000F03C0100C83C0100CC3C0100D03C010085
:1073C000D43C0100D83C0100DC3C0100E03C010061
:1073D000E43C0100E83C0100EC3C0100F0B52B4E20
:1073E0002B4FDFF8C4E005460FCE87B06C460FC4C4
:1073F00096E803003B68274A274F44F8040B40F601
:10740000CC308342C8BF3A46BEF800602180012ECE
:1074100011889278ADF80D108DF80F202AD032D354
:1074200040F6CA02022E18BF00229A4226DAA3F6BC
:1074300098031A491A4AC3EB031381FB0301194449
:10744000DB17C3EB6123243382FB0321DA17C2EB82
:10745000A10202EB8201A3EB4103303330328DF8FD
:1074600013308DF811206946284616220BF006F8D5
:1074700007B0F0BD40F698029A42D8DB094B186875
:10748000CDF81100EFE740F6FC02CEE7043D010025
:10749000449FFF1FF83C0100F43C01003B773B9800
:1074A00067666666FC3C0100E09EFF1FF8B5174C5E
:1074B000174E2278174D33782F888E46003218BF2A
:1074C000012201467046FFF717FB002398423370F4
:1074D000237015DB14BF012000202B889F420ED0A3
:1074E00040F23A72A3F5AF730B490C4C02FB03F365
:1074F00081FB0312DB17A3EB621332332360F8BD69
:107500000749012218460A702270E6E7148BFF1F14
:1075100009A0FF1FAC9FFF1FB5814E1B088AFF1FEC
:1075200094A0FF1F014B187802F004BC7CA0FF1F41
:10753000014B187802F018BCD091FF1F134BB3F920
:10754000003030B583EAE374A4EBE374002BA0B2FF
:1075500018DB012300E0134603EB83025200944240
:10756000F9DA0B4D90FBF3F285FB03E403FB120009
:10757000DB173032D3EBA40380B201F8012BF1D139
:107580000B7030BD2D230B700131E2E7D091FF1F4E
:1075900067666666144BB3F9003070B583EAE3752D
:1075A000A5EBE375002BACB21ADB012300E0034628
:1075B00003EB830040008542F9DA0C4E94FBF3F0B4
:1075C00086FB03E503FB1044DB173030D3EBA50348
:1075D000A4B201F8010BF1D105480B70106070BD29
:1075E0002D230B700131E0E7189DFF1F676666666B
:1075F0001C3D0100134BB3F9003030B583EAE3744E
:10760000A4EBE374002BA0B218DB012300E01346C7
:1076100003EB830252009442F9DA0B4D90FBF3F234
:1076200085FB03E403FB1200DB173032D3EBA4032A
:1076300080B201F8012BF1D10B7030BD2D230B70FE
:107640000131E2E7C489FF1F67666666134BB3F931
:10765000003030B583EAE374A4EBE374002BA0B2EE
:1076600018DB012300E0134603EB8302520094422F
:10767000F9DA0B4D90FBF3F285FB03E403FB1200F8
:10768000DB173032D3EBA40380B201F8012BF1D128
:107690000B7030BD2D230B700131E2E7689DFF1F99
:1076A00067666666134BB3F9003030B583EAE3745E
:1076B000A4EBE374002BA0B218DB012300E0134617
:1076C00003EB830252009442F9DA0B4D90FBF3F284
:1076D00085FB03E403FB1200DB173032D3EBA4037A
:1076E00080B201F8012BF1D10B7030BD2D230B704E
:1076F0000131E2E7869DFF1F67666666134BB3F9AB
:10770000003030B583EAE374A4EBE374002BA0B23D
:1077100018DB012300E0134603EB8302520094427E
:10772000F9DA0B4D90FBF3F285FB03E403FB120047
:10773000DB173032D3EBA40380B201F8012BF1D177
:107740000B7030BD2D230B700131E2E7869FFF1FC8
:1077500067666666134BB3F9003030B583EAE374AD
:10776000A4EBE374002BA0B218DB012300E0134666
:1077700003EB830252009442F9DA0B4D90FBF3F2D3
:1077800085FB03E403FB1200DB173032D3EBA403C9
:1077900080B201F8012BF1D10B7030BD2D230B709D
:1077A0000131E2E75E89FF1F67666666134BB3F936
:1077B000003030B583EAE374A4EBE374002BA0B28D
:1077C00018DB012300E0134603EB830252009442CE
:1077D000F9DA0B4D90FBF3F285FB03E403FB120097
:1077E000DB173032D3EBA40380B201F8012BF1D1C7
:1077F0000B7030BD2D230B700131E2E72089FF1F94
:1078000067666666134BB3F9003030B583EAE374FC
:10781000A4EBE374002BA0B218DB012300E01346B5
:1078200003EB830252009442F9DA0B4D90FBF3F222
:1078300085FB03E403FB1200DB173032D3EBA40318
:1078400080B201F8012BF1D10B7030BD2D230B70EC
:107850000131E2E7188AFF1F67666666134BB3F9CA
:10786000003030B583EAE374A4EBE374002BA0B2DC
:1078700018DB012300E0134603EB8302520094421D
:10788000F9DA0B4D90FBF3F285FB03E403FB1200E6
:10789000DB173032D3EBA40380B201F8012BF1D116
:1078A0000B7030BD2D230B700131E2E7648AFF1F9E
:1078B00067666666134BB3F9003030B583EAE3744C
:1078C000A4EBE374002BA0B218DB012300E0134605
:1078D00003EB830252009442F9DA0B4D90FBF3F272
:1078E00085FB03E403FB1200DB173032D3EBA40368
:1078F00080B201F8012BF1D10B7030BD2D230B703C
:107900000131E2E75C89FF1F6766666608B5B8204B
:1079100002F092FA044B1988884204D0B820BDE8DE
:10792000084002F06FBA08BD209DFF1F08B5702007
:1079300002F082FA044B1988884204D07020BDE816
:10794000084002F05FBA08BDE09EFF1F08B5742032
:1079500002F072FA044B1988884204D07420BDE802
:10796000084002F04FBA08BD749FFF1F054B1B88EB
:107970000846042213B904490AF080BD03490AF0FD
:107980007DBD00BF6A9DFF1F243D0100203D010019
:107990000E4B1B88032B17D8DFE803F0110C0702EE
:1079A000084604220A490AF069BD0846042209492A
:1079B0000AF064BD0846042207490AF05FBD084684
:1079C000042206490AF05ABD704700BFEE9EFF1F11
:1079D000303D0100C83D01002C3D0100283D010063
:1079E00010B40A4B0A4C0A4693E8030083B023887C
:1079F00002AC04E9030004EB8303104653F8081CAF
:107A0000052203B010BC0AF039BD00BFDC34010010
:107A1000509FFF1F30B40A4B0A4D0C4693E80700F5
:107A200084B02B8804AD05E9070005EB83032046ED
:107A300053F80C1C042204B030BC0AF01FBD00BF78
:107A4000E4340100E09EFF1FF0B40C4D0C4F0E46D5
:107A50000FCD8CB001AC0FC40FCD0FC495E807005B
:107A60003B8884E807000CAA02EB8303304653F8F6
:107A70002C1C04220CB0F0BC0AF000BDF034010054
:107A8000349FFF1F30B50A4B0A4D0C460FCB85B013
:107A90000DF1100E0EE90F002B880EEB830320462C
:107AA00053F8101C042205B0BDE830400AF0E6BCD3
:107AB0002C350100529FFF1F30B50A4B0A4D0C4672
:107AC0000FCB85B00DF1100E0EE90F002B880EEBD9
:107AD0008303204653F8101C042205B0BDE8304053
:107AE0000AF0CCBC2C350100E49EFF1FF0B40B4D16
:107AF0000B4F0E460FCD86B06C460FC495E80300C1
:107B00003B8884E8030006AA02EB8303304653F85F
:107B1000181C042206B0F0BC0AF0B0BC3C350100D1
:107B2000EE9DFF1FF0B40A4D0A4F0E460FCD86B0F2
:107B300001AC0FC42A683B88226006AA02EB8303CB
:107B4000304653F8141C0C2206B0F0BC0AF096BC68
:107B5000543501006C9DFF1FF0B40B4D0B4F0E46CA
:107B60000FCD86B06C460FC495E803003B8884E8CF
:107B7000030006AA02EB8303304653F8181C0422C4
:107B800006B0F0BC0AF07ABC68350100749FFF1F94
:107B9000164B1B880BB31BB283EAE370A0EBE370B8
:107BA000002B30B584B21DDB012300E0134603EB4C
:107BB000830252009042F9DA0D4894FBF3F280FB05
:107BC00003E503FB1244DB173032D3EBA503A4B269
:107BD00001F8012BF1D10B7030BD08460422054994
:107BE0000AF04CBC2D230B700131DDE7B09DFF1F67
:107BF00067666666343D0100F0B40A4D0A4F0E46D2
:107C00000FCD86B001AC0FC42A683B88226006AA5B
:107C100002EB8303304653F8141C042206B0F0BC78
:107C20000AF02CBC803501000C9DFF1F054B1B8802
:107C30001BB9054B186808607047084604220349C1
:107C40000AF01CBCC89DFF1FC83C0100C43C0100D9
:107C5000164B1B880BB31BB230B583EAE374A4EB5D
:107C6000E374002BA0B21CDB012300E0134603EBFE
:107C7000830252009442F9DA0D4D90FBF3F285FB3A
:107C800003E403FB1200DB173032D3EBA40380B212
:107C900001F8012BF1D10B7030BD064B186808605C
:107CA00070472D230B700131DEE700BF5C9DFF1F85
:107CB00067666666C83C0100164B1B880BB31BB297
:107CC00030B583EAE374A4EBE374002BA0B21CDBB1
:107CD000012300E0134603EB830252009442F9DAD9
:107CE0000D4D90FBF3F285FB03E403FB1200DB1761
:107CF0003032D3EBA40380B201F8012BF1D10B7029
:107D000030BD064B1868086070472D230B70013199
:107D1000DEE700BF209DFF1F67666666C83C010066
:107D2000164B1B880BB31BB230B583EAE374A4EB8C
:107D3000E374002BA0B21CDB012300E0134603EB2D
:107D4000830252009442F9DA0D4D90FBF3F285FB69
:107D500003E403FB1200DB173032D3EBA40380B241
:107D600001F8012BF1D10B7030BD064B186808608B
:107D700070472D230B700131DEE700BF429FFF1FCC
:107D800067666666C83C0100164B1B880BB31BB2C6
:107D900030B583EAE374A4EBE374002BA0B21CDBE0
:107DA000012300E0134603EB830252009442F9DA08
:107DB0000D4D90FBF3F285FB03E403FB1200DB1790
:107DC0003032D3EBA40380B201F8012BF1D10B7058
:107DD00030BD064B1868086070472D230B700131C9
:107DE000DEE700BF249DFF1F67666666383D010021
:107DF000174B1B881BB31BB270B583EAE375A5EB69
:107E0000E375002BACB21EDB012300E0034603EB5D
:107E1000830040008542F9DA0E4E94FBF3F086FBB6
:107E200003E503FB1044DB173030D3EBA503A4B20A
:107E300001F8010BF1D108480B70106070BD074BC1
:107E40001868086070472D230B700131DCE700BF14
:107E5000D09DFF1F676666663C3D0100C83C01007F
:107E6000164B1B880BB31BB230B583EAE374A4EB4B
:107E7000E374002BA0B21CDB012300E0134603EBEC
:107E8000830252009442F9DA0D4D90FBF3F285FB28
:107E900003E403FB1200DB173032D3EBA40380B200
:107EA00001F8012BF1D10B7030BD064B186808604A
:107EB00070472D230B700131DEE700BFC09FFF1F0D
:107EC00067666666C83C0100164B1B880BB31BB285
:107ED00030B583EAE374A4EBE374002BA0B21CDB9F
:107EE000012300E0134603EB830252009442F9DAC7
:107EF0000D4D90FBF3F285FB03E403FB1200DB174F
:107F00003032D3EBA40380B201F8012BF1D10B7016
:107F100030BD064B1868086070472D230B70013187
:107F2000DEE700BF909FFF1F67666666C83C0100E2
:107F3000164B1B880BB31BB230B583EAE374A4EB7A
:107F4000E374002BA0B21CDB012300E0134603EB1B
:107F5000830252009442F9DA0D4D90FBF3F285FB57
:107F600003E403FB1200DB173032D3EBA40380B22F
:107F700001F8012BF1D10B7030BD064B1868086079
:107F800070472D230B700131DEE700BFBC9FFF1F40
:107F900067666666C83C0100174B1B881BB31BB2A3
:107FA00070B583EAE375A5EBE375002BACB21EDB7D
:107FB000012300E0034603EB830040008542F9DA29
:107FC0000E4E94FBF3F086FB03E503FB1044DB1736
:107FD0003030D3EBA503A4B201F8010BF1D108486E
:107FE0000B70106070BD074B1868086070472D2338
:107FF0000B700131DCE700BF8E9FFF1F676666666E
:108000003C3D0100C83C0100054B1B881BB1054BE2
:10801000186808607047044B18680860704700BF14
:10802000BE9DFF1F503D01004C3D010070B5FAF7A9
:1080300083F8164B1B7813B1154C237833B9154BC5
:108040001020198801F0DEFE012070BD124D134E84
:108050002B783288B3FA83F382F008025B09114669
:1080600042202B70328001F0CDFE23780BB12B78AB
:108070002BB90021212006F0F3F9002070BD012169
:10808000212006F0EDF9002070BD00BF269DFF1FE6
:10809000E69EFF1F009FFF1FFE9EFF1FB49FFF1F56
:1080A000184B1A8852B3184A128830B50A80B3F9AF
:1080B0000030002B83EAE374A4EBE374BCBF2D23F0
:1080C0008B70A0B2ACBF02310331012300E0134634
:1080D00003EB830252009442F9DA0C4D90FBF3F269
:1080E00085FB03E403FB1200DB173032D3EBA40360
:1080F00080B201F8012BF1D10B7030BD044B186830
:1081000008607047769DFF1F543D010067666666F4
:10811000C83C010070B53C4D2B780646002B35D18C
:108120001C4673780BB9204670BDFAF705F8374A3C
:10813000374B3848127831781B78007802EB4303CC
:108140004A1E03EB80030E2AEDD801A050F822F05E
:10815000B9810000DB81000027810000B9810000A7
:10816000278100002781000027810000A7810000EF
:10817000278100002781000027810000278100005F
:108180002781000027810000A3810000AE21224842
:1081900003F0C8FF204804F015FA00232B700124D7
:1081A000BFE706F083FEAF211B4803F0BBFF1B4A6D
:1081B000012313702B70B6E783B91948038804298B
:1081C0004FF6FF7103F1FF320CBF01230B4613443E
:1081D00003F07F03013303800FE073B1013B114AC9
:1081E00032F813304BB10E4E0F481049104A33800D
:1081F0000123002606700B701370084A0221012328
:1082000011702B70204670BD148BFF1F959FFF1FB0
:10821000969FFF1F979FFF1F1CA0FF1F94A0FF1F8B
:10822000809FFF1FC09EFF1FA89DFF1F2C9DFF1F4B
:1082300097A0FF1F10B5064B064C1A882046012157
:1082400001F0CEFD21884220BDE8104001F0DABDEA
:108250008C9DFF1FB49FFF1F10B5064B064C1A885C
:108260002046022101F0BCFD21884220BDE81040DB
:1082700001F0C8BDD29DFF1FB49FFF1F10B5064B74
:10828000064C1A882046042101F0AAFD21884220CC
:10829000BDE8104001F0B6BDF69EFF1FB49FFF1F62
:1082A00010B5064B064C1A882046002101F098FDB7
:1082B00021884220BDE8104001F0A4BD3E9FFF1F71
:1082C000B49FFF1F08B5122001F0B6FD054B1988B9
:1082D000884206D0122001F095FDBDE8084001F06B
:1082E0005BBC08BD349FFF1F08B5582001F0A4FDFA
:1082F000054B1988884206D0582001F083FDBDE85F
:10830000084001F049BC08BD429FFF1F08B514207A
:1083100001F092FD054B1988884206D0142001F027
:1083200071FDBDE8084001F037BC08BDDA9DFF1FB4
:10833000F0B480EAE075A5EBE0750028ACB21FDB75
:108340001DBF2B230B704E1C0E46012300E013466D
:1083500003EB830252009542F9DA0B4F94FBF3F2E0
:1083600087FB030503FB1244DB173032D3EBA50375
:10837000A4B206F8012BF1D133700846F0BC704767
:108380002D230B704E1CE0E767666666084B188865
:1083900028B10D2807D00D3800B2FFF7C9BF054A34
:1083A000106808607047044A10680860704700BF92
:1083B000EE9FFF1FC83C0100583D0100174B188875
:1083C0000C2813D0192815D01A2817D01B2819D01B
:1083D0001C281BD01D281DD01E2803D00C3800B22D
:1083E000FFF7A6BF0E4A1068086070470D4A106874
:1083F000086070470C4A1068086070470B4A1068A4
:10840000086070470A4A106808607047094A106897
:1084100008607047084A1068086070477E9FFF1F19
:10842000743D01005C3D0100603D0100643D0100C0
:10843000683D01006C3D0100703D0100034B188850
:10844000A0EB8000400000B2FFF772BF7CA0FF1FCE
:10845000024B1888643800B2FFF76ABFD89FFF1F2D
:10846000024B1888643800B2FFF762BFA89FFF1F55
:10847000024B1888033800B2FFF75ABF569FFF1F00
:10848000024B18880C3800B2FFF752BF1E9DFF1F29
:10849000024B1888183800B2FFF74ABF589DFF1FDB
:1084A000024B1888183800B2FFF742BF569DFF1FD5
:1084B000024B1888183800B2FFF73ABF929FFF1F8F
:1084C000C3681888183800B2FFF732BF054B1B8805
:1084D0001BB9054B18680860704708460422034919
:1084E00009F0CCBF609FFF1FC83C0100C43C0100E5
:1084F000054B1B881BB9054B186808607047084678
:108500000422034909F0BABF5E9DFF1FC83C010069
:10851000C43C010030B5134C85B001252B463C22EC
:1085200002212046009503F073FE204604F04AF82D
:1085300000224021802320460191009311460A4BDE
:10854000029504F0EDFC204604F048F9074808497C
:10855000084A0023036083800B608B801360938044
:1085600005B030BD1CA0FF1F30380100FC9FFF1F6D
:1085700014A0FF1F84A0FF1F10B500EBC00000F186
:108580000F02D2B293B284B09C1E981C3D2303917B
:108590008DE819003921024804F026FC04B010BD12
:1085A0001CA0FF1F014B01221A70704709A0FF1F7A
:1085B000F0B5784B784C794F794E7A4D85B00422DE
:1085C0008DE80C0002932046774B4022802103F077
:1085D00027FC2046754A7649764C09F0CBF8764B55
:1085E00076489F61764FDF61764FB761764FF761CE
:1085F000764FAF61764FEF61764FA761764FE761B7
:10860000764F87617649774FC761774F8F61774A99
:10861000774FCF61774F9761774B784FD761784F1E
:108620009F61784E784FDF61784FB761784D794F11
:10863000F761794F794CAF61794FEF61794F7A48A3
:10864000A7617A4FE7617A4F7A4987617A4FC761AC
:108650007A4F7B4A8F617B4FCF617B4F7B4B97611A
:108660007B4FD7617B4F7C4E9F617C4FDF617C4F9E
:108670007C4DB7617C4FF7617C4FAF617C4C7D4F87
:10868000EF617D4FA7617D487D4FE7617D4F876139
:108690007D497E4FC7617E4F8F617E4A7E4FCF619D
:1086A0007E4F97617E4B7F4FD7617F4F9F617F4E9B
:1086B0007F4FDF617F4FB7617F4D804FF761804F04
:1086C000AF61804C804FEF61804FA7618048814F40
:1086D000E761814F87618149814FC761814F824A3C
:1086E0008F61824FCF61824F824B9761824FD761FA
:1086F000824F834E9F61834FDF61834F834DB7610C
:10870000834FF761834F844CAF61844FEF61844F97
:108710008448A761844FE761844F85498761854F0D
:10872000C761854F8F61854A854FCF61854F9761BE
:10873000854B864FD761864F9F61864E864FDF619E
:10874000864F874DB761874FF761874F874CAF6181
:10875000874F88488849EF61884F894DA761E56157
:10876000884F894D894CDFF848E2894A894B8761F7
:10877000C5618C61884E894F894D8A4CC1F81CE0D7
:1087800089488A499761D5619C61D861B16005B01B
:10879000F0BD00BF40420F001CA0FF1F81840000FD
:1087A000D08FFF1F1C8FFF1FEC91FF1F1C89FF1F25
:1087B00079BE00009C8CFF1F048EFF1FF48FFF1FEB
:1087C000C16F000071840000CD6F00007572000061
:1087D000358200009D72000059820000C5720000C1
:1087E000BC8DFF1F7D820000E1790000088DFF1F16
:1087F000DD6F0000ED720000E08DFF1FA182000020
:10880000618400007C91FF1FED6F00005184000027
:108810005891FF1FFD6F0000B97C0000988DFF1F6D
:108820000D7900003D840000748DFF1F2575000048
:108830003D750000AC8FFF1F31750000157A0000F8
:10884000308CFF1F2D790000497A00006090FF1FD7
:10885000C5820000217D0000E48CFF1FE98200003A
:1088600095750000F08BFF1F0D7000001573000060
:10887000F090FF1F0D830000897D0000C08CFF1F5A
:108880001D700000F17D00004C8EFF1F2D70000058
:10889000617E0000788CFF1F3D700000F5750000C0
:1088A000A88BFF1F4D700000857A0000A890FF1F65
:1088B0005D7000004D760000648FFF1F6D7000003A
:1088C000B97A0000848BFF1F7D700000A576000040
:1088D000288EFF1F8D700000ED7A0000CC8AFF1FEC
:1088E0009D700000FD7600002C8DFF1FAD70000014
:1088F000A1800000888FFF1FBD700000257B000055
:10890000AC91FF1FCD700000C97E0000F88EFF1FE4
:10891000DD700000317F0000608BFF1FED700000F4
:10892000597B00008490FF1F4D790000997F000063
:10893000408FFF1FFD700000BD8300003C8BFF1FB8
:108940000D710000917B0000188BFF1F1D7100004E
:10895000F97B0000848AFF1F2D7100008D830000C9
:10896000508DFF1F3D71000055770000548CFF1F94
:108970004D710000F08AFF1FCC8BFF1FAD77000008
:108980005D710000057800006D7100005D780000E9
:108990001890FF1FA88AFF1FA091FF1FB578000045
:1089A0008D710000098000009D710000758F00002E
:1089B0007D710000F0B5461C83B00D4601270323EE
:1089C00036B22AB2044631468DE888002348ADB25B
:1089D00004F0A0F90C23AA1C12B2009301970523FE
:1089E00021B21E4804F096F91D4A1E4B12881B68DE
:1089F000BA422AD023D3022A10D11B4CA3F6CA03B1
:108A000084FB03241C44DB17C3EB24140A2CA8BFEB
:108A10000A2424EAE474A2B223B202E000231A4634
:108A20001C460D35AA1A01200093019012B231465E
:108A300003230A4804F0ECF8204603B0F0BD0B4CC9
:108A4000A3F6FC0384FB0324DDE7094CA3F698039B
:108A500084FB0324DB17C3EBA404D7E71CA0FF1F90
:108A6000E09EFF1F449FFF1F09CB3D8D1F85EB51EB
:108A7000398EE3382DE9F0438FB283B0DFF84C80B4
:108A8000BD1D461D2DB204B236B24FF001090AB227
:108A90002346314640460095CDF8049004F0EAF8AC
:108AA0002A463346214640468DE8200204F0E2F88B
:108AB00007F10C020095334612B22146CDF804901E
:108AC000404604F0D7F803B0BDE8F0831CA0FF1FB8
:108AD0002DE9F043804685B0002956D10121304868
:108AE00004F05EFC2F4998F8062098F8083011F839
:108AF0000290994522DA4FEA89064D460C24D8F8AF
:108B00000C3027489B595F6822B2002104F044FCD6
:108B1000384609F0F5FB39460246214804F0D6FDF7
:108B20001F4804F0E9FD98F8083001350934AB42DC
:108B3000A4B206F1040601DD422CE0D1B9F1000F28
:108B400013D109F1060999450CDA3C2301213B2296
:108B5000039102930093019239233F223A21104856
:108B600004F042F905B0BDE8F0830F2301213B2258
:108B7000039102930093019239230C223A21084871
:108B800004F032F998F80830DBE700213423009331
:108B900001913F230C22024804F03AF89EE700BFFF
:108BA0001CA0FF1F14A0FF1F10B5104C0121204670
:108BB00004F0FCFB2046012104F0F2FB20463422A5
:108BC000552104F0E9FB20460222094904F07EFD0C
:108BD00020460522074904F079FD204604F08CFD6B
:108BE0002046BDE8104003F0F9BD00BF1CA0FF1FE8
:108BF000C03D0100C43D010070B50D46064609F0B8
:108C00007FFB00EB40008400002D36D0284609F0A1
:108C100077FB00EB4000400023185B1003F160017C
:108C2000091A282209B21748C3F1600404F0B4FB02
:108C30000121144804F0B4FB284609F061FB2946E1
:108C40000246104804F042FD0E4804F055FD022192
:108C50000C4804F0A5FB21B221220A4804F09CFB39
:108C6000304609F04DFB31460246064804F02EFD21
:108C70000448BDE8704004F03FBD6410C4F16004D6
:108C8000E5E700BF1CA0FF1F10B50D4B1B5C51F8A2
:108C90002340237884B013B1012004B010BD04AA8E
:108CA00001A942F8103D2046A3699847A38A9B0773
:108CB000F2D401A80099FFF79FFF012004B010BD76
:108CC000FC9FFF1F2DE9F04F2F4DDFF8CCB0DFF8F0
:108CD000C4A0DFF8C8900FCD91B003AC0FC40FCD86
:108CE0000FC40FCD0FC42B6823600025A8462F4664
:108CF0002E4600E09846BAF8003024495BF823205D
:108D000028461123F7F76EFD00EBC00400EB84004A
:108D100089FB00340444C017C0EB6434C4F13C0048
:108D2000C6F13C0207F14101012600B208F14103FE
:108D300000901BB2019612B209B2154803F09AFFD7
:108D400008EB060305F211153C2B2646ADB247464B
:108D5000D0D134226B210E4804F01EFB00210C48B8
:108D600004F01EFB0B4B1B8810AA02EB830353F885
:108D7000344C204609F0C4FA02460548214611B099
:108D8000BDE8F04F04F0A2BC94350100402F010073
:108D90001CA0FF1F3E9DFF1FA42D010009000280A3
:108DA000234B70B5B3F9003083EAE374A4EBE374AA
:108DB000002B82B0A1B234DB68466D46012300E08F
:108DC000134603EB830252009442F9DA194E91FBE9
:108DD000F3F286FB03E403FB1211DB173032D3EB13
:108DE000A40389B205F8012BF1D119462B70FFF7C6
:108DF00003FF114B1B7813B1104B1B780BB902B05A
:108E000070BD01210E4804F0CBFA332264210C48D6
:108E100004F0C2FA04220B49094804F057FC02B0DE
:108E200070BD2D238DF800300DF101056846C5E7B2
:108E3000009FFF1F67666666E69EFF1FFE9EFF1F80
:108E40001CA0FF1FCC3D010010B5424C424882B02F
:108E500003F0B8FB2378C3B906213F4804F0A0FA19
:108E60002378012B37D90A22022B11463A486BD0BE
:108E700004F092FA39490322374804F027FC3648B7
:108E800002B0BDE8104004F037BC354B1A78012120
:108E90000523002A35D10191009311462E4803F095
:108EA00039FF304B1A78002A36D00523012201926F
:108EB000009300220A21284803F0AAFE2A4B1A78C0
:108EC000002A35D101210523019100931421224864
:108ED00003F020FFC0E7254C2388092B32D9632BF0
:108EE0008CBF0A211F210A221B4804F055FA218851
:108EF000194804F051FC184802B0BDE8104004F0D5
:108F0000FBBB0022019100931146134803F080FE41
:108F1000144B1A78002AC8D105230121019100932E
:108F20000A210D4803F0F6FE0F4B1A78002AC9D02B
:108F3000012205230192009300221421064803F028
:108F400067FE89E73021CEE704F026FA03220849BC
:108F500092E700BF97A0FF1F1CA0FF1FD83D010094
:108F6000959FFF1F969FFF1F979FFF1F809FFF1FCB
:108F7000D43D0100F8B56D4D287840B96C4B1B68A5
:108F800099425CD36B4A012313702B70F8BD0C46D9
:108F900000266948664F03F015FB04F6AC533246D1
:108FA00065483B6031212E7004F0F6F901216248DA
:108FB000624D04F0FBF931465F4804F0F1F90522F7
:108FC0005F495D4804F082FB5B4804F095FB0C228E
:108FD0001021594804F0E0F90B225A49564804F090
:108FE00075FB05225849544804F070FB524804F0C0
:108FF00083FB564B50481C68A4F69803C3EB03133D
:1090000085FB03251D441021DB172022C3EB6525BA
:1090100004F0C2F940F6CC339C4205F124054FF030
:1090200022014FF004000BDCFFF7C4FC484B1C8806
:10903000064674B3012C46D0022C41D00120F8BD65
:10904000FFF718FD092243493B4804F03FFB2A2261
:109050001021394804F0A0F93F4C374884FB05340F
:10906000EB17C3EBA404214604F096FB01223B4915
:10907000314804F02BFB04EB8401A5EB41012E48A1
:1090800004F08AFB012236492B4804F01FFB012023
:10909000F8BD34491022284804F018FB264804F093
:1090A0002BFB2A221021244804F076F9314622486D
:1090B00004F072FB07222C491F4804F007FBCBE7A2
:1090C0000C222A49E7E70C2229491B4804F0FEFA42
:1090D000194804F011FB2A221021174804F05CF90A
:1090E000314615481C4E04F057FB07221E49124812
:1090F00004F0ECFA86FB0536EB17C3EBA606314607
:109100000D4804F049FB224614490B4804F0DEFAEE
:1091100006EB8601A5EB4101074804F03DFB224622
:109120000F49054804F0D2FA2046F8BD148BFF1F02
:1091300010A0FF1F94A0FF1F1CA0FF1F3B773B98B0
:10914000DC3D0100E43D0100C43D0100449FFF1FE0
:10915000E09EFF1FF03D010067666666DC4501008A
:109160004C450100FC3D0100103E0100283E01007D
:10917000183E01002DE9F041754C2278002A054681
:109180000F4614BF4FF001084FF000084ED1714E4A
:109190003368CB1AB3F5FA6F04D86B78A3B940469D
:1091A000BDE8F0816C4B6D486D49DFF8D0E11A7075
:1091B000012303700988237026208EF8002000F018
:1091C00021FE6B78002BEAD03760F8F7B5FF654ACF
:1091D000654B6649127828781B78097802EB4303BF
:1091E000421E03EB81030E2AD9D801A151F822F0C7
:1091F000E1920000AD9200009F910000E19200001A
:109200009F9100009F9100009F91000095920000A7
:109210009F910000479200009F9100009F910000E5
:109220009F9100009F91000043920000AF215048A1
:10923000484E02F077FFFFF707FE002337602370E8
:10924000ABE705F033FE4A4803F0BCF90221484879
:1092500004F0A6F80F222321454804F09DF80522CA
:109260004449434804F032FA414804F045FA1E22CA
:1092700023213F4804F090F805223F493C4804F080
:1092800025FA3B4804F038FA394803F0A7FA00F011
:10929000D3FC84E7394D2B78012B50D9304B262055
:1092A000198800F0AFFD00232B7078E7002B3FF406
:1092B00076AF013B324A32F81330002B3FF46FAFE8
:1092C000274C304825492D4A23804FF001080023C0
:1092D000037081F8008082F80080FFF7B5FD5EE73B
:1092E00093B1013B264A32F8131019B31C4B254D9C
:1092F0001A4C224A19800026012326202E70237042
:10930000137000F07FFD15E0154C1E4922880B708C
:1093100004284FF6FF7002F1FF310CBF0122024614
:109320000A440E4E154D02F07F02013201212280C7
:1093300031702B70FFF788FD4FF001082FE70649C9
:10934000064A01230020087013702370A6E700BFAF
:10935000148BFF1F90A0FF1F94A0FF1F2C9DFF1FC9
:10936000809FFF1F959FFF1F969FFF1F979FFF1FC7
:109370001CA0FF1F383E0100403E010097A0FF1FC8
:10938000C09EFF1FA89DFF1F2DE9F04F05468BB023
:109390000F46AD480121164604F008F8AA8812F0DD
:1093A000010440F0B080DFF8CC8298F80030002B48
:1093B0007DD1AB79A54AD15CA1B9DFF8BCA279789F
:1093C0001AF8039041B339780139072900F2B780C0
:1093D000DFE811F0F1005401B5006C01B500B500F3
:1093E000B500E9007C78002C00F0CA800139EC68F7
:1093F000387854F82170FC68411EB4F800800729C1
:1094000000F2A780DFE811F074015901A5006C019A
:10941000A500A500A5009F00DFF854A2DAF80020FF
:10942000B21AB2F5967F75D9894A107801281ABF09
:10943000012010701170874A18BF0146D05CC0EB44
:109440000900C0B2FFF798F80124CAF80060AB88A1
:109450009B0770D57B78002B6DD0F8F76DFE7E4BA7
:109460007E4A7F481B78127839780078022515FBF0
:1094700002330A2903EB800300F04E810C295AD1F4
:10948000002B58D003F11900764E774A013B00219A
:10949000400080B226F813100123157088F80030C0
:1094A00000F0B0FC714B032220461A702FE0664892
:1094B00003F088F80121644803F072FF62482246F5
:1094C000214603F069FFAB88580725D42C68204655
:1094D00008F016FF214602465B4804F0F7F85A48A8
:1094E00004F00AF9092201238DE80C0000217F23F2
:1094F000554803F0BFFB00212846FFF7E9FA002397
:1095000088F8003055E7AB683146384698470BB0CD
:10951000BDE8F08F0846FAE72B6804A8984704A82E
:1095200008F0EEFE04A90246474804F0CFF846488A
:1095300004F0E2F8D6E720460BB0BDE8F08F002437
:109540000AF8039083E70021D1543846FB69984715
:10955000FC68A4F80080002725223C238DE88400C5
:1095600041211822384803F053FBE968A879FFF736
:109570008BFB374A3E4B17701E600BB0BDE8F08F77
:109580003B490A68B21AB2F5967FD4D9304F0E60C3
:109590003E78012E00F0B480E968184601233B7044
:1095A000FFF772FBB3E7304AE9791170012288F8BE
:1095B00000200024C4E72A7A013A4A45BFDD09F1B8
:1095C0000104E4B2A145BAD0224E16F803B0CBEBA9
:1095D0000900C0B20021FEF7CFFF2B7A052BD94638
:1095E0001BD9CBEB0402042A40F3AE80A4F1040B98
:1095F000BBF1000FC0F2B080063B5B45A8BF5B46E5
:109600005FFA83F9AA791348B15C994205D000F852
:10961000029001212846FFF75BFAC9EB0400C0B2B3
:1096200001210B4EFEF7A8FF002134230191009386
:109630000548317040230B223F21A14603F0E8FA90
:109640000124AB797CE700BF1CA0FF1F84A0FF1F93
:1096500095A0FF1F14A0FF1F959FFF1F969FFF1F40
:10966000979FFF1FC09EFF1F94A0FF1F97A0FF1F83
:1096700080A0FF1F148BFF1FFC9FFF1F0FFA89F1B3
:10968000E868604C50F821602168049134785E49A4
:1096900004980860002C71D0012C7FF450AF5B4A15
:1096A000317A88F800401170002449E7B9F1000FC1
:1096B00050D009F1FF34E4B284E7B98A01F0040123
:1096C00089B200293FF440AF3B6A03929847039A5E
:1096D00000283FF43DAFAB79FC680021D15438E756
:1096E0007B8A43453CD908F101081FFA88F830E726
:1096F0003B8A43453BD208F1FF381FFA88F828E738
:1097000025238DE8180042483C703C231822412153
:1097100003F07EFA3046FAE6002B3FF40CAF3D4AE8
:109720003D4E1188394A03F11900013B400080B2D7
:1097300026F81310012388F80030157000F062FB42
:10974000364B20461D70E2E6002A3FF755AF04F184
:10975000FF3B4DE74C46F3E64FF000094B4651E71F
:10976000BB8ADA077FF5F5AEB7F81080F1E6BB8A61
:10977000D9077FF5EEAEB7F81280EAE62849C85C53
:10978000C0EB090009F1010EC0B201214FF0340B0A
:1097900002F803E0FEF7F0FEB6681D48019440238E
:1097A0000B223F210124CDF800B003F031FA402311
:1097B0000B223F211648CDF800B0019403F0AAFA1D
:1097C0002146134803F0ECFD304608F099FDA0EB6C
:1097D000800000F15F0109B20F220D4803F0DCFDAB
:1097E000304608F08DFD31460246094803F06EFF11
:1097F000074803F081FFE968A879FFF745FAAB79DC
:109800009EE600BFD4A0FF1F80A0FF1F94A0FF1FF3
:109810001CA0FF1F809FFF1FC09EFF1F97A0FF1F60
:1098200014A0FF1F2DE9F047DFF808926D4B99F85F
:1098300000601B68DFF800A282B0003601934FF091
:10984000030018BF0126019F9AF8008004F00EFE65
:109850000546042004F00AFE0446052004F006FE36
:10986000800040EA4404062004F000FE2C4364B269
:109870005D4944EAC0000A7880F00F03DBB29A42E7
:109880005A4A3CD01760002259480B7003788DF873
:1098900000808DF8012053B3564A12684EF66021BD
:1098A000BA1A8A4219D8022B59D0012B5FD0062B45
:1098B00048D0032B63D0042B69D0052B77D0072B1E
:1098C0007DD0082B00F08380092B68D016B14A4860
:1098D00002F084FF02B0BDE8F087484A484C0023FC
:1098E0000121237003701360938089F800103A46B9
:1098F00069464448FFF748FD3043C6B2E6E71268C0
:10990000BA1A1E2A6BD99AF80020934222D0394CF9
:109910003D488AF80030012B276082EA0302076085
:109920009846B1D0042BAFD137480068381AB0F54B
:10993000C87FA9D9354C2068381A3228A4D92760A5
:109940001A46A1E73A4669463148FFF71DFD304304
:10995000C6B2BBE7012B4FF00002E3D1E4E73A4681
:1099600069462C48FFF710FD3043C6B2AEE73A46D1
:1099700069462948FFF708FD3043C6B2A6E73A46D4
:1099800069462648FFF700FD3043C6B29EE73A46D7
:1099900069462348FFF7F8FC3043C6B296E73A46DB
:1099A00069462048FFF7F0FC3043C6B28EE73A46DE
:1099B00069461D48FFF7E8FC3043C6B286E73A46E1
:1099C00069461A48FFF7E0FC3043C6B27EE73A46E4
:1099D00069461748FFF7D8FC3043C6B276E7002245
:1099E00052E700BFD4A0FF1F98A0FF1F04A0FF1FD5
:1099F00094A0FF1F8CA0FF1F1CA0FF1F84A0FF1FAF
:109A000096A0FF1F003801009CA0FF1F0CA0FF1FA5
:109A1000303C0100583701005C360100F835010088
:109A20009C4401004C360100B43601003C37010073
:109A3000A091FF1F148BFF1F08A0FF1F28B1102843
:109A4000044BA8BF102018607047024B012018601B
:109A5000704700BFA0A0FF1F08B5002006F010F956
:109A60000028FAD108BD00BF10B504464FF440608D
:109A700005F01AF805F072F80A4B1B7833B96CB18F
:109A8000102C094BA8BF10241C6010BD4FF4C0500F
:109A900004F0E0FD04F014FF002CF1D1024B01248E
:109AA0001C6010BDE69EFF1FA0A0FF1F70B50D46F5
:109AB0001446064605F048F8284605F045F82046C5
:109AC00005F042F8084B1B7813B1084B1B7803B91B
:109AD00070BD304604F09CFE284604F099FE2046F6
:109AE000BDE8704004F094BEE69EFF1FFE9EFF1F7F
:109AF00038B5164D2B78044641F6FF72A0F500509C
:109B0000824203F1FF33A8BF02461B0202F5005256
:109B100003F47063100443F4604343F00E0300F455
:109B2000FE005204184302F0FE42104305F0DEFF2F
:109B30002868013860F01F00C4F3C61204F07F01EA
:109B4000C0B2BDE83840FFF7B1BF00BFA0A0FF1F03
:109B500070B5104E3378013B1B0203F4706304466A
:109B600043F430430806220400F0FE4043F00B03A8
:109B7000034302F4FE0018430D4605F0B7FF3068BA
:109B8000013860F04F002A462146C0B2BDE870405F
:109B9000FFF78CBFA0A0FF1F08B564210720FFF7C7
:109BA000D7FF7F210B20BDE80840FFF7D1BF00BFE2
:109BB00070B5104E3378013B1B0203F4706304460A
:109BC00043F410430806220400F0FE4043F009036A
:109BD000034302F4FE0018430D4605F087FF30688A
:109BE000013860F06F002A462146C0B2BDE87040DF
:109BF000FFF75CBFA0A0FF1F38B50E4D2B78013BCF
:109C00001B0203F47063044643F41043000443F062
:109C1000090300F4FE00184305F068FF28680138C6
:109C200060F06F002146C0B20022BDE83840FFF767
:109C30003DBF00BFA0A0FF1F10B500217B20FFF794
:109C400087FF0024E0B2FFF7D7FF0134022004F0C1
:109C500043FC802CF6D110BD38B50C46054604F007
:109C600073FF204604F070FF074B1B7813B1074BBE
:109C70001B7803B938BD284604F0CAFD2046BDE86C
:109C8000384004F0C5BD00BFE69EFF1FFE9EFF1FCB
:109C900038B50D4D2B78013B1B0203F4706304466D
:109CA00043F45043000443F00D0300F4FE00184356
:109CB00005F01CFF2868013860F02F002146C0B273
:109CC000BDE83840FFF7C8BFA0A0FF1F38B50E4D54
:109CD0002B78013B01381B02C4B203F470632004EB
:109CE00043F4404343F00C0300F4FE00184305F036
:109CF000FDFE2868013860F03F002146C0B2BDE893
:109D00003840FFF7A9BF00BFA0A0FF1F38B5044629
:109D10000D46F02004F018FF35B1254414F8010B6E
:109D200004F012FFAC42F9D1F720BDE8384004F04E
:109D30000BBF00BF00B50B4B83B002469988186873
:109D40000090032AADF8041002D903B05DF804FBBB
:109D5000684606218DF80520FFF7D8FF03B05DF8AF
:109D600004FB00BF0C45010000B50B4B024683B05D
:109D7000186899880090131F4C2BADF8041002D975
:109D800003B05DF804FB684606218DF80520FFF757
:109D9000BDFF03B05DF804FB14450100030203F4AA
:109DA000FE43C0F3C6101843704700BF03784078E5
:109DB000DB0103F47E5300F07F001843704700BFBF
:109DC00082B002AA114642F8040D002012F8013BAD
:109DD00003F07F03914243EA0020F7D102B07047BD
:109DE000003210B403884FF0010404FA01F418BFE4
:109DF000012202FA01F123EA04020A43028010BCA4
:109E0000704700BF70B5CEB20C46054603F0F6FEB3
:109E1000864203D03146284603F00AFF0135284622
:109E200003F0ECFE240A844205D021462846BDE812
:109E3000704003F0FDBE70BD38B5054603F0DEFE90
:109E40004FF0000460F30704681C03F0D7FE60F3D2
:109E50000F24A0B238BD00BFF8B504460020FFF7BC
:109E6000EBFF002C00F0D1854FF4AF610220FFF72B
:109E7000C9FF4FF47A610420FFF7C4FF4FF49661E5
:109E80000620FFF7BFFF4FF4FA610820FFF7BAFF83
:109E90004FF4FA610A20FFF7B5FF40F6B8310C2005
:109EA000FFF7B0FF4FF42F612220FFF7ABFF40F622
:109EB000AC512420FFF7A6FF7D212A20FFF7A2FF47
:109EC0000C210E20FFF79EFF01211020FFF79AFFC3
:109ED00002211220FFF796FF00211420FFF792FFC6
:109EE00000211620FFF78EFF02211820FFF78AFFBE
:109EF00001211A20FFF786FF01211C20FFF782FFB6
:109F000004211E20FFF77EFF14212020FFF77AFF97
:109F100001212620FFF776FF03212820FFF772FF9B
:109F200004212C20FFF76EFF14212E20FFF76AFF7B
:109F300000213020FFF766FF0C213220FFF762FF7F
:109F400000213420FFF75EFF00213620FFF75AFF83
:109F500000213820FFF756FF00213A20FFF752FF7B
:109F600000213C20FFF74EFF00213E20FFF74AFF73
:109F700000214020FFF746FF00214220FFF742FF6B
:109F80001F214420FFF73EFF13214620FFF73AFF31
:109F90000E214820FFF736FF11214A20FFF732FF3C
:109FA0000A214C20FFF72EFF00214E20FFF72AFF49
:109FB00006215020FFF726FF02215220FFF722FF43
:109FC0000C215420FFF71EFF00215620FFF71AFF37
:109FD00000215820FFF716FF01215A20FFF712FF3A
:109FE00008215C20FFF70EFF0A215E20FFF70AFF21
:109FF00000216020FFF706FF04216220FFF702FF27
:10A0000001216420FFF7FEFE00216620FFF7FAFE23
:10A010000B216820FFF7F6FE7F216A20FFF7F2FE92
:10A0200000216C20FFF7EEFE00216E20FFF7EAFE14
:10A0300000217020FFF7E6FE00217220FFF7E2FE0C
:10A0400000217420FFF7DEFE1F217620FFF7DAFEE5
:10A0500013217820FFF7D6FE0E217A20FFF7D2FEDB
:10A0600011217C20FFF7CEFE0A217E20FFF7CAFED9
:10A070001F218020FFF7C6FE13218220FFF7C2FEBA
:10A080000E218420FFF7BEFE11218620FFF7BAFEC5
:10A090000A218820FFF7B6FE00218A20FFF7B2FED2
:10A0A00000218C20FFF7AEFE00219620FFF7AAFECC
:10A0B00000219820FFF7A6FE00219A20FFF7A2FEBC
:10A0C00005219C20FFF79EFE06219E20FFF79AFEA9
:10A0D0000021A020FFF796FE7F21A220FFF792FE2D
:10A0E00040F2A461A420FFF78DFE4FF4E161A620A9
:10A0F000FFF788FE0021A820FFF784FE0021AA2098
:10A10000FFF780FE0221AC20FFF77CFE0121AE208C
:10A11000FFF778FE0121B020FFF774FE0B21B2207B
:10A12000FFF770FE6421B420FFF76CFE6421B620B7
:10A13000FFF768FE0321B820FFF764FE2C21002002
:10A14000FFF760FE0220FFF777FEB0F5805F034661
:10A1500080F03486D24A04201380FFF76DFEB0F5FC
:10A16000805F034680F02186CE4A06201380FFF7E9
:10A1700063FEA0F52F739BB2B3F57A6F024606D942
:10A1800040F628210620FFF73DFE40F62822C64B68
:10A1900008201A80FFF750FEA0F52F739BB2B3F58D
:10A1A0007A6F024606D940F6E4410820FFF72AFEFE
:10A1B00040F6E442BD4B0A201A80FFF73DFEA0F5B1
:10A1C000FA739BB240F6AC518B42024606D94FF46B
:10A1D000FA610A20FFF716FE4FF4FA62B44B0C2026
:10A1E0001A80FFF729FEA0F5FA739BB240F6AC5136
:10A1F0008B42024606D940F6B8310C20FFF702FE2A
:10A2000040F6B832AB4B0E201A80FFF715FE182827
:10A21000034600F2C385A84A10201380FFF70CFE06
:10A22000431E9BB20F2B024604D901211020FFF7D9
:10A23000E9FD0122A14B12201A80FFF7FDFD0A283B
:10A24000034600F2A4859E4A14201380FFF7F4FD14
:10A250000128034604D900211420FFF7D3FD002371
:10A26000984A16201380FFF7E7FD7F28034600F287
:10A270008785954A18201380FFF7DEFD05280346E1
:10A2800000F27785914A1A201380FFF7D5FD0C283C
:10A29000034600F267858E4A1C201380FFF7CCFD31
:10A2A0000428034600F257858A4A1E201380FFF7D0
:10A2B000C3FD0928034600F24785874A2020138002
:10A2C000FFF7BAFD4628034600F23785834A22206D
:10A2D0001380FFF7B1FDA0F5FA739BB240F6AC51C5
:10A2E0008B42024606D94FF42F612220FFF78AFDE8
:10A2F0004FF42F627A4B24201A80FFF79DFDA0F5C2
:10A30000FA739BB240F6AC54A342024604D92146EC
:10A310002420FFF777FD2246724B26201A80FFF794
:10A320008BFD7F28034600F201856F4A28201380A9
:10A33000FFF782FD0628034600F2F1846B4A2A20CB
:10A340001380FFF779FDA0F132039BB2B3F5967F3E
:10A35000024604D97D212A20FFF754FD7D22644B5B
:10A360002C201A80FFF768FD0C28034600F2D084E9
:10A37000604A2E201380FFF75FFD1E28034600F27F
:10A38000C0845D4A30201380FFF756FD092803463C
:10A3900000F2B084594A32201380FFF74DFD1E2889
:10A3A000034600F2A084564A34201380FFF744FD90
:10A3B0007F28034600F29084524C36202380FFF71A
:10A3C0003BFD7F28034600F2808438206380FFF73E
:10A3D00033FD7F28034600F271843A20A380FFF703
:10A3E0002BFD7F28034600F262843C20E380FFF7C8
:10A3F00023FD7F28034600F253843E202381FFF78C
:10A400001BFD7F28034600F2448440206381FFF750
:10A4100013FD7F28034600F235844220A381FFF715
:10A420000BFD394D28804420FFF706FD30280346F8
:10A4300000F2FD83354A46201380FFF7FDFC3028EB
:10A44000034600F2EE83324C48202380FFF7F4FCF1
:10A450003028034600F2DF834A206380FFF7ECFCDC
:10A460003028034600F2D1834C20A380FFF7E4FCA0
:10A470003028034600F2C3834E20E380FFF7DCFC64
:10A480000128034604D900214E20FFF7BBFC00231E
:10A49000204A50201380FFF7CFFC431E3CE000BF52
:10A4A000E89DFF1FB29FFF1F8E9DFF1F7C9FFF1F18
:10A4B000489FFF1F549DFF1F1E9DFF1F009FFF1FF2
:10A4C000349FFF1FDA9DFF1F249DFF1FEE9DFF1F7E
:10A4D000769DFF1F6C9DFF1F5C9DFF1F8E9FFF1FC2
:10A4E000FC9EFF1FF89EFF1F809FFF1F569FFF1FB0
:10A4F000AC9FFF1F3E9DFF1FD09DFF1FC09FFF1FF2
:10A500007E9FFF1FC09EFF1FB49FFF1F929FFF1FD4
:10A51000589FFF1F6A9DFF1F9BB20B2B024604D959
:10A5200006215020FFF76EFC0622CF4B52201A80E6
:10A53000FFF782FC0428034600F25B83CB4A5420D9
:10A540001380FFF779FC431E9BB21D2B024604D9F2
:10A550000C215420FFF756FC0C22C54B56201A80C4
:10A56000FFF76AFC0128034604D900215620FFF7B3
:10A5700049FC0023BF4A58201380FFF75DFC7F2869
:10A58000034600F23083BC4A5A201380FFF754FC84
:10A59000431E9BB2092B024604D901215A20FFF722
:10A5A00031FC0122B54B5C201A80FFF745FC431EAD
:10A5B0009BB2102B024604D908215C20FFF722FC35
:10A5C0000822AF4B5E201A80FFF736FC431E9BB279
:10A5D0001D2B024604D90A215E20FFF713FC0A2234
:10A5E000A84B60201A80FFF727FC0228034600F2E0
:10A5F000F482A54A64201380FFF71EFC012803465D
:10A6000004D901216420FFF7FDFB01239F4A62204A
:10A610001380FFF711FCC31E9BB2012B024604D925
:10A6200004216220FFF7EEFB0422994B66201A807A
:10A63000FFF702FC7F28034600F2C982954A682092
:10A640001380FFF7F9FB7F28034600F2BA82924A93
:10A650006A201380FFF7F0FB7F28034600F2AB82ED
:10A660008E4A6C201380FFF7E7FB0428034600F2B4
:10A670009C828B4A6E201380FFF7DEFB192803466D
:10A6800000F28D82874A70201380FFF7D5FB0228E5
:10A69000034600F27E82844A72201380FFF7CCFBCF
:10A6A0000628034600F26F82804A74201380FFF769
:10A6B000C3FB0528034600F260827D4A8A2013808E
:10A6C000FFF7BAFB0A28034600F25182794A8C2030
:10A6D0001380FFF7B1FB0428034600F24282764A5A
:10A6E00098201380FFF7A8FB0128034604D9002116
:10A6F0009820FFF787FB0023704A9A201380FFF70A
:10A700009BFB0128034604D900219A20FFF77AFB1E
:10A7100000236B4A96201380FFF78EFB0B2803461D
:10A7200000F21982674A9C201380FFF785FB831E85
:10A730009BB2032B024604D905219C20FFF762FB44
:10A740000522614B76201A80FFF776FB30280346FE
:10A7500000F2FB815D4A78201380FFF76DFB302803
:10A76000034600F2EC815A4C7A202380FFF764FB09
:10A770003028034600F2DD817C206380FFF75CFB1C
:10A780003028034600F2CF817E20A380FFF754FBE0
:10A790003028034600F2C1818020E380FFF74CFBA4
:10A7A0003028034600F2B3814A4A82201380FFF723
:10A7B00043FB3028034600F2A481474C84202380C9
:10A7C000FFF73AFB3028034600F29581862063802C
:10A7D000FFF732FB3028034600F287818820A380F0
:10A7E000FFF72AFB3028034600F27981A020E3809E
:10A7F000FFF722FB0128034604D90021A020FFF720
:10A8000001FB0023354A9E201380FFF715FBC31E72
:10A810009BB20C2B024604D906219E20FFF7F2FAC8
:10A8200006222F4BA2201A80FFF706FB431E9BB285
:10A830007E2B024604D97F21A220FFF7E3FA7F2274
:10A84000284BA4201A80FFF7F7FAA0F5AF639BB25C
:10A85000B3F5167F024647D940F2A461A420FFF762
:10A86000D1FA40F2A4623FE02089FF1F5E89FF1FFA
:10A87000188AFF1FBE9DFF1F429FFF1F189DFF1FCD
:10A88000648AFF1F5C89FF1FF49EFF1F509FFF1FFC
:10A890007C9DFF1F909FFF1FB09DFF1F609DFF1FAE
:10A8A0000C9DFF1FEE9FFF1FE09EFF1FBC9FFF1F21
:10A8B000749FFF1F029FFF1FEE9EFF1F5E9DFF1FE5
:10A8C000C89DFF1F3C9FFF1F429DFF1F569DFF1FFE
:10A8D000D09EFF1F589DFF1FD89EFF1F609FFF1F28
:10A8E000C489FF1F869FFF1FD44BA6201A80FFF745
:10A8F000A3FAA0F5AF639BB2B3F5167F024606D963
:10A900004FF4E161A620FFF77DFA4FF4E162CC4BF2
:10A91000A8201A80FFF790FA0628034600F2D98093
:10A92000C84AAA201380FFF787FA0328034600F2DB
:10A93000CA80C54AAC201380FFF77EFA032803467D
:10A9400000F2BB80C14AB0201380FFF775FA0328DC
:10A95000034600F2AC80BE4AAE201380FFF76CFACB
:10A960007F28034600F29D80BA4AB2201380FFF789
:10A9700063FA7F28034600F28E80B74AB420138022
:10A98000FFF75AFA431E9BB2C62B024604D9642134
:10A99000B420FFF737FA6422B04BB6201A80FFF7D5
:10A9A0004BFA431E9BB2C62B024604D96421B62043
:10A9B000FFF728FA6422AA4BB8201A80FFF73CFA66
:10A9C000082862D82B88DFF8B8E2A64FA64AA74D20
:10A9D000A74EA84CA84903F0010CAEF800C0C3F381
:10A9E000400EA7F800E0C3F380071780C3F3C00749
:10A9F000A24A2F70C3F30017C3F34015C3F38013AB
:10AA0000378025800B801080F8BD4FF6FF73984289
:10AA10003FF42AAA2C283FF495AB17287FF624AAE6
:10AA200019287FF68DAA1B287FF6AAAA1C283FF4B6
:10AA3000BFAA1E287FF6C4AA1F283FF4C9AA20284F
:10AA40003FF4E2AA21283FF4EBAA22283FF4F0AA1F
:10AA500023283FF4F9AA24283FF42AAB25283FF401
:10AA60002FAB26283FF430AB27283FF435AB2828FE
:10AA70003FF440AB29283FF445AB2A283FF452ABC2
:10AA80002B287FF45BABFFF755BBB8200321FFF702
:10AA9000B9F9032096E70B21B220FFF7B3F90B2396
:10AAA0006BE70121AE20FFF7ADF901235CE701213F
:10AAB000B020FFF7A7F901234DE70221AC20FFF7F3
:10AAC000A1F902233EE70021AA20FFF79BF900230A
:10AAD0002FE70021A820FFF795F9002320E70A219E
:10AAE0008820FFF78FF90A2380E611218620FFF7DF
:10AAF00089F9112372E60E218420FFF783F90E23D2
:10AB000064E613218220FFF77DF9132355E61F2108
:10AB10008020FFF777F91F2346E60A217E20FFF702
:10AB200071F90A2338E611217C20FFF76BF9112314
:10AB30002AE60E217A20FFF765F90E231CE6132181
:10AB40007820FFF75FF913230DE61F217620FFF72A
:10AB500059F91F23FEE500219620FFF753F9002342
:10AB6000E0E500218C20FFF74DF90023B7E5002137
:10AB70008A20FFF747F90023A8E500217420FFF79A
:10AB800041F9002399E500217220FFF73BF90023EA
:10AB90008AE500217020FFF735F900237BE50021CD
:10ABA0006E20FFF72FF900236CE500216C20FFF7E2
:10ABB00029F900235DE57F216A20FFF723F97F2330
:10ABC0004EE50B216820FFF71DF90B233FE500211F
:10ABD0006620FFF717F9002330E500216020FFF71A
:10ABE00011F9002305E500215820FFF70BF9002398
:10ABF000C9E402215220FFF705F902239EE40A214D
:10AC00004C20FFF7FFF80A2336E411214A20FFF712
:10AC1000F9F8112328E40E214820FFF7F3F80E235A
:10AC20001AE413214620FFF7EDF813230BE41F214C
:10AC30004420FFF7E7F81F23FFF7FCBBEC9DFF1F45
:10AC4000689FFF1F1A9DFF1F949DFF1F529FFF1FAC
:10AC5000E49EFF1F689DFF1F869DFF1FA89FFF1F8B
:10AC6000D89FFF1F8C9DFF1FD29DFF1FFE9EFF1FC1
:10AC7000F69EFF1F549FFF1F069FFF1F209DFF1F73
:10AC80003E9FFF1F00214020FFF7BCF80023FFF785
:10AC9000C4BB00213E20FFF7B5F80023FFF7B5BB8A
:10ACA00000213C20FFF7AEF80023FFF7A6BB0021F0
:10ACB0003A20FFF7A7F80023FFF797BB00213820C1
:10ACC000FFF7A0F80023FFF788BB00213620FFF72D
:10ACD00099F80023FFF779BB00213420FFF792F8A1
:10ACE0000023FFF769BB0C213220FFF78BF80C2300
:10ACF000FFF759BB00213020FFF784F80023FFF74E
:10AD000049BB14212E20FFF77DF81423FFF739BB30
:10AD100004212C20FFF776F80423FFF729BB032139
:10AD20002820FFF76FF80323FFF708BB0121262037
:10AD3000FFF768F80123FFF7F8BA14212020FFF786
:10AD400061F81423FFF7C2BA04211E20FFF75AF856
:10AD50000423FFF7B2BA01211C20FFF753F80123A7
:10AD6000FFF7A2BA01211A20FFF74CF80123FFF7E1
:10AD700092BA02211820FFF745F80223FFF782BAA2
:10AD800000211620FFF73EF80023FFF772BA0221D8
:10AD90001220FFF737F80223FFF755BA0C210E20D7
:10ADA000FFF730F80C23FFF736BA4FF47A6104202E
:10ADB000FFF728F84FF47A63FFF7D6B94FF4AF6185
:10ADC0000220FFF71FF84FF4AF63FFF7C3B900BFCE
:10ADD000F8B5CB2006F008FD204B214A054603CBF1
:10ADE0001368C5F803001A0CBA20C5F807102B80A9
:10ADF000AA70FEF7D3FF2E46002426F80B0FA0B250
:10AE0000FFF71AF8FEF7CAFF0234BA2C26F8020F31
:10AE1000F5D16C1E05F1C6064FF0FF3014F8013F66
:10AE2000082758400F4B40F300017A1E0B4012F0E8
:10AE3000FF0783EA5000F5D1B442EFD1C043FEF7DB
:10AE4000BFFF3A46C5F8C700CB21284604F09CFE58
:10AE50002846BDE8F84006F0CFBC00BF2045010001
:10AE60001C4501002083B8EDF0B50E4B0E4C054695
:10AE700093E8070085B024682E88AD7801AB83E89D
:10AE80000700270C184600220B21ADF804408DF86E
:10AE90000670ADF80C608DF80E5004F075FE05B02C
:10AEA000F0BD00BF2C4501001C450100F0B5124B60
:10AEB000124D1E68124F0FCD87B06C460FC495E837
:10AEC000030044F8040B38683B79CDF80D00320CD0
:10AED0002C2021808DF802208DF81130ADF8006013
:10AEE000FEF75CFF0022ADF80B001221684604F06B
:10AEF0004BFE07B0F0BD00BF1C4501003845010006
:10AF0000C43D0100002004F0BBBE00BF02F02EBE15
:10AF100070B5124C82B000254023064629462046D3
:10AF2000009301958023202201F072FE2022294601
:10AF3000204602F031FA2046012102F037FA30466D
:10AF400007F0DEF931460246204602F0BFFB2046FC
:10AF500002B0BDE8704001F041BC00BF1CA0FF1F63
:10AF6000F0B5CA2983B075D90546441E00F1C6065E
:10AF70004FF0FF3014F8012F08275040404A40F3AB
:10AF800000017B1E0A4013F0FF0782EA5000F5D152
:10AF9000B442EFD1C043FEF713FF0146D5F8C70016
:10AFA0000190019A914202D0B2F17F2F0BD105F1AD
:10AFB0000B00FEF7FBFEBA280BD03248FFF7A8FFC4
:10AFC000002003B0F0BD3048FFF7A2FF384603B0C1
:10AFD000F0BD05F10D00FEF7E9FE2C2840D100245C
:10AFE00040F6AC5613E004281AD0062821D00828D1
:10AFF0001FD00A2828D00C2822D1A1F5FA7292B2CB
:10B00000B24201D8FEF7FEFE0234BA2C0ED004F193
:10B010000D002844FEF7CAFE022C0146A0B2E2D180
:10B02000B1F5805FEED30234BA2CF0D1012003B029
:10B03000F0BDA1F52F7292B2B2F57A6FE4D8E1E7D4
:10B04000222801D0242811D1A1F5FA7292B2B2427D
:10B05000DAD8D7E70D48FFF75BFF002003B0F0BD5B
:10B060000B48FFF755FF002003B0F0BD2A28C9D1D7
:10B07000A1F1320292B2B2F5967FC5D8C2E700BF05
:10B080002083B8ED7C450100684501005045010072
:10B090009045010003290CD970B5461C82B00546C5
:10B0A0000C46304603222A4907F098F910B102B045
:10B0B00070BD70470B2C05D905222649281D07F0C5
:10B0C0008DF940B12448FFF723FF244802B0BDE8C2
:10B0D0007040FFF7C9BE05F10901032201A807F07E
:10B0E000CDF901A803221E4907F078F9D8B103224F
:10B0F0001C4901A807F072F908B301A803221A49F4
:10B1000007F06CF9B0B91948FFF702FFA11E89B228
:10B110003046FFF725FF0028C9D0154802B0BDE82A
:10B120007040FFF7F5BE1348FFF7F2FEFFF750FE41
:10B130001148F3E71148FFF7EBFE1148C6E7114845
:10B14000FFF7E6FE02B0BDE87040FFF7AFBE00BFFC
:10B150001C450100A8450100B0450100C44501009F
:10B16000C8450100F0450100084601000C460100F9
:10B1700020460100CC450100E045010034460100B5
:10B1800048460100F44501002DE9F043174D2B68B6
:10B1900083B081460F469046F3B1154E34880A19A4
:10B1A00092B218461146328006F09CFE28603A465C
:10B1B0004946204402F06CFDB8F1000F09D03188F7
:10B1C0002868FFF767FF286806F016FB00232B604E
:10B1D000338003B0BDE8F083054E0193084631800B
:10B1E00006F002FB019B28601C46E0E7A8A0FF1FB9
:10B1F000A4A0FF1F10B51F4C4FF4FA70FBF762FDBF
:10B20000204601F0DFF900221146204602F0C4F882
:10B210002046012102F0CAF82046002102F0C0F8C1
:10B220000B221549204602F051FA204602F064FA3A
:10B230000F221249204602F049FA204602F05CFA39
:10B240000F490722204602F041FA204602F054FA44
:10B25000204601F0C3FA0B4B0B4A1A604FF4FA7008
:10B26000FBF730FDFFF722FE0848BDE81040FFF76E
:10B270004FBE00BF1CA0FF1F4C46010058460100F6
:10B2800068460100DCA2FF1F89B100007046010082
:10B290000020704790F8392090F83800101A704755
:10B2A00090F8383090F839209A4205D95A1C034456
:10B2B00080F83820187E70474FF0FF30704700BF8D
:10B2C00090F8383090F839209A4286BF1B18187EC3
:10B2D0004FF0FF30704700BF704700BF38B50546DC
:10B2E000B0F85E0090B195F85D301446C3F12102CC
:10B2F00094420CD805F13B001844224602F0C8FCE9
:10B3000095F85D30234485F85D30204638BD012036
:10B3100014462871EEE700BFB0F85E306BB190F8CC
:10B320005D30202B07D8C218013380F85D30012032
:10B3300082F83B107047012303710020704700BF63
:10B340000023426980F8383080F8393080F85C306A
:10B3500080F85D3080F85E3080F85F3006CA30B427
:10B360000D68046943662A4383660A60A3704269D4
:10B3700090F861301649146813441D7A5B7B01EB29
:10B38000C5051B026D6803F4E06343F064032B60A2
:10B3900090F8623013449D7CDB7D01EBC5011B02FC
:10B3A000496803F4E06343F064030B602168536869
:10B3B000194205D0036927225A70036904229A7141
:10B3C000036920225A71036980229A7030BC704749
:10B3D000A451010043690CCB12681A420CD0094BEE
:10B3E00099420AD9084B9942036994BF1A220D2247
:10B3F0005A70036904229A717047036927225A70B0
:10B40000F7E700BF7F1A06003F420F0010B5026940
:10B41000D378DBB2D90604463DD510215806D17049
:10B4200038D503F0040303F0FF02002B51D03D494F
:10B43000626E00230B7084F85D30002A5BD0904769
:10B4400094F85D30002B56D02369D0229A7023697E
:10B4500094F83B201A712369012284F85C200222AF
:10B46000DA7010BD304B84F860009C424AD02F4BFC
:10B470009C4252D094F8391013791F29DBB207D8B7
:10B480002848007820B16018013184F8391003761B
:10B490000223D37010BD5906C3D4917801F0100176
:10B4A00001F0FF000029DDD013F001031ED194F854
:10B4B0005C1094F85D00884281BF4B1C091984F828
:10B4C0005C3091F83B3013712369D0229A70226965
:10B4D000DEE7236984F83920C0229A702369114A73
:10B4E0001979012111700222DA7010BDC023937006
:10B4F00022691379CCE70122002384F85D2084F8C7
:10B500003B30A1E7626994F8613009491344032292
:10B51000187A02F043FD2269ACE7626994F8613061
:10B520000449F3E7ACA0FF1FEC91FF1F5892FF1FE7
:10B5300095B50000A1B500000369DB7803F0200396
:10B5400073B190F860300133DBB2012B80F86030CA
:10B550001AD9426990F861301344187A02F09ABD02
:10B5600070B5426903F0FF0590F86130134404465A
:10B57000187A02F08FFDA36E5BB184F8385094F80E
:10B580003900BDE87040184790F85F30002BE0D0DC
:10B59000704770BD0148FFF7CFBF00BFEC91FF1FA0
:10B5A0000148FFF7C9BF00BF5892FF1F2DE9F047C0
:10B5B000374FDFF8E0903B68026982B0064600939F
:10B5C000DDF800800021A025D3789B065BD53B6881
:10B5D0000193019BC8EB03030F2BF5D949B1102B45
:10B5E000F2D000209070336980229A7002B0BDE8DA
:10B5F000F087726996F8613013440521187A02F0D9
:10B6000043FF726996F861301344012193F812A048
:10B61000504602F039FF09240021504602F020FF75
:10B620002B46013BFDD10121504602F019FF2B466C
:10B63000013BFDD1013CEFD1706996F861100144E6
:10B640004FF4A0720C7A4B7B09EBC4011B024968D2
:10B6500003F4E06343F064030B6096F86230034444
:10B66000997CDB7D09EBC1011B02496803F4E063AF
:10B6700043F064030B60013AFDD13269D3789B0635
:10B680004FF00101A3D4012002B0BDE8F08700BF54
:10B69000D4A0FF1FA4510100F0B503691222DA7093
:10B6A0000269937803F0200385B004460D46002B11
:10B6B0005ED0B42393703C4922690B680093009ECE
:10B6C00005E00B680193019B9B1B042B42D8D378A8
:10B6D00003F0200303F0FF00002BF2D094F85D305C
:10B6E000002B31D04FF0000E4FF0020C04EB0E0394
:10B6F00093F83B3013710B680393039F206907E0B5
:10B700009B060DD50B680293029BDB1B052B28D8EB
:10B71000C378DBB203F0020202F0FF06002AEFD08A
:10B7200080F803C02669F378DBB2DF0632462DD4F9
:10B730009F062BD5DB0731D40EF1010E94F85D3056
:10B740005FFA8EFE7345D1D800201DBB002384F81C
:10B750005E3004E09070236980229A70042005B066
:10B76000F0BD86702369802204209A7005B0F0BD78
:10B7700003F0FF06FFF71AFF10B9042005B0F0BD73
:10B78000236984F85F60B0229A7094E78023B370D5
:10B790000420DAE726698023B370D7E7BEF1000FF3
:10B7A0000CBF02200320F6E7D4A0FF1F2DE9F041D3
:10B7B00006690025122780F8385080F83950F77054
:10B7C000D0F810C09CF802E00EF0200E88B00446BD
:10B7D000884615461E46BEF1000F49D0B4238CF8AA
:10B7E0000230784B21691A680092DDF800E006E02B
:10B7F0001A6801920198CEEB0000042830D8C8786E
:10B8000000F0200000F0FF070028F1D04FEA4802C6
:10B8100042F00102D2B20A711A680292DDF808E021
:10B82000206906E01A6803920399CEEB010105290D
:10B830002AD8C17801F0020101F0FF070029F1D0F8
:10B840004FF0020C80F803C02269D17811F0110783
:10B8500022D12DBB002E0CBFA0238023937003E0C8
:10B860008F70236980229A70384608B0BDE8F08155
:10B870000EF0FF07FFF79AFE0028F5D0236984F841
:10B880005F70B0229A70ACE78770236980223846D7
:10B890009A7008B0BDE8F081802393700027E3E739
:10B8A000012D75D0A021917021690A79BE466746A5
:10B8B0004FF0A80C1A680492049805E01A680592E3
:10B8C000059A121A052A4AD8CA7802F0020202F032
:10B8D000FF08002AF2D0CF702169CA78D2B212F0E4
:10B8E000100F08465AD1920658D5013DEDB2012DF0
:10B8F00049D0BEF11F0F3BD90A79012DDAD11A6860
:10B900000692069D05E01A680792079A521B052ABF
:10B9100046D8C27802F0020202F0FF01002AF2D0FB
:10B920000223C3702269D378DBB2D9063AD49B06CE
:10B9300034D5B023BEF11F0F93703FD8226904EBBA
:10B940000E0312791A760EF1010E5FFA8EFE16B111
:10B95000236980229A7084F839E0774684E781F879
:10B960000280236980229A70774684F839E07BE769
:10B9700004EB0E0291F8048082F818800EF1010E9B
:10B980005FFA8EFEB9E781F802C021690846B0E788
:10B99000A82191702069BE460279B0E7774663E737
:10B9A0008170DEE71021A023D170013BFDD1226917
:10B9B000937803F0F7037746937055E723691B7973
:10B9C000C5E700BFD4A0FF1F0148FFF71FBD00BFA0
:10B9D000EC91FF1F0148FFF719BD00BF5892FF1FF0
:10B9E000704700BF38B5144C037801225B00054650
:10B9F000204684F83B3084F85E2084F85D20FFF711
:10BA00008BFC20460021FFF747FE0B4C29780123D1
:10BA100020461A46FFF7CAFE0128F6D194F83830BE
:10BA200094F839209A4205D9E218013384F8383065
:10BA3000107E38BDFF2038BDEC91FF1F38B51B4C80
:10BA4000037801225B000546204684F83B3084F8E9
:10BA50005E2084F85D20FFF75FFC20460021FFF7A1
:10BA60001BFE124C2978204601230222FFF79EFE7E
:10BA70000228F6D194F8382094F839108A420FD26F
:10BA8000531CDBB2A018994284F83830007E0AD9E2
:10BA9000234402321B7E84F8382040EA032038BD5C
:10BAA0004FF6FF7038BD40F47F4038BDEC91FF1F6A
:10BAB0000C2901D9002070470231490001F0FE0134
:10BAC000FFF7BCBF70B50C4C0378164601255B0030
:10BAD000204684F83B3084F85E5084F85D50FFF7D0
:10BAE0001BFC31462046FFF717FC29462046BDE8DF
:10BAF0007040FFF7D1BD00BFEC91FF1FF8B50546C0
:10BB00000F461646412421463A462846FFF7DAFFFB
:10BB1000611C0234C9B232462846E4B2FFF7D2FFB4
:10BB2000592CF0D1F8BD00BF38B504460D46354854
:10BB3000FFF706FC6322802120462570FFF7C2FF35
:10BB4000012002F0C9FC204600225E21FFF7BAFF67
:10BB500020465D21FFF746FF242801D0002038BD94
:10BB6000204606220C21FFF7C9FF204601222B2187
:10BB7000FFF7A8FF204601222C21FFF7A3FF204654
:10BB80000E222D21FFF79EFF204600222E21FFF7D7
:10BB900099FF204601222F21FFF794FF204605221E
:10BBA0003021FFF78FFF204601223121FFF78AFF66
:10BBB000204600223221FFF785FF20460022332154
:10BBC000FFF780FF204600223421FFF77BFF20464D
:10BBD00000223521FFF776FF204600225B21FFF788
:10BBE00071FF204610225C21FFF76CFF20462022C7
:10BBF0005D21FFF767FF20468F225E21FFF762FF7E
:10BC0000012038BDEC91FF1F10B4047F4160022C6D
:10BC1000C26002D010BC01F0D7BB836810BC1847CB
:10BC200090E80C00F0B41C6859682568164F174E50
:10BC300029432160164D17491760D66015611160C0
:10BC4000417A154A5C180A3194F8244053F821507F
:10BC500002EBC40149680D60017A5C1803EB8101B5
:10BC6000247ECD6902EBC40149680D60817A5818C1
:10BC700003EB810390F83000596B02EBC002F0BC7B
:10BC800053681960704700BF01401F000110003861
:10BC90000110007800001F80A4510100704700BF10
:10BCA000F0B50C1EBDF8146034DBB0F9067019193C
:10BCB000B942C4BF3B1B1BB2002BA6461CDD002AA9
:10BCC0001146B8BFD11D02F00705CC10826A0120D1
:10BCD00007FB04E1A840012E0A44C0B21ED00CD3D9
:10BCE000022E09D1013B12FA83F3013A12F8011F27
:10BCF00041409A421170F9D1F0BDC043013B12FAA4
:10BD000083F3C0B2013A12F8011F0140934211704F
:10BD1000F9D1F0BD23441BB20024C6E7013B12FA5F
:10BD200083F3013A12F8011F01439A421170F9D1CD
:10BD3000F0BD00BFF8B50D1E0EDB14461F460646CB
:10BD400001F03AFBA84207DD002C05DB304601F08C
:10BD500037FBA04201DCF8BDF8BD304601F02AFBFC
:10BD6000022853D003284BD0012806D16540F38820
:10BD70006C406540013B5D1B2DB2012F03D02AD3DF
:10BD8000022F14D0F8BD002C2246B6F90630B06A56
:10BD9000B8BFE21D42F3CF0202FB035504F00704D3
:10BDA000435D012101FA04F41C434455F8BD002C05
:10BDB0002246B6F90630B06AB8BFE21D42F3CF02A0
:10BDC00002FB035504F00704435D012101FA04F46A
:10BDD0005C404455F8BD002C2246B6F90630B06AE6
:10BDE000B8BFE21D42F3CF0202FB035504F0070483
:10BDF000435D012101FA04F423EA04044455F8BD2B
:10BE00003389013B591B25460CB2B6E7F1883289CC
:10BE10000139013A4D1B141B2DB224B2ADE700BF0E
:10BE20002DE9F041079E9DF91880089D04461F46A4
:10BE300000F0C0FF0D4B0E480E4984F83380FF22FE
:10BE4000002F08BF1F4684F82F20002384F83020DD
:10BE500084F8312084F832202060A665E5656762A9
:10BE600061652362A3622046BDE8F081EC91FF1F6B
:10BE7000FC4601000110013810B50446806A034BEE
:10BE8000236008B105F0B8FC204610BDFC46010057
:10BE9000F8B5436ADBB190F82C200125AA4083F85D
:10BEA0003B2083F85E5083F85D500446406A036887
:10BEB0000E461B6800219847606A036831461B687C
:10BEC00098472946606ABDE8F840FFF7E5BBC26BBA
:10BED000C56C1368046A23EA050313604CB1226839
:10BEE0004FF00043D3625163D36A002BFCDA936BAB
:10BEF000F8BD836B466B0825802410E03768426CE0
:10BF00003A4332601F68826C3A431A601A68876C41
:10BF1000013D22EA07024FEA54041A6007D0214289
:10BF2000ECD13268476C22EA07023260EAE7F8BDDA
:10BF300070B50446406A0D4600282BD0A16DFFF76E
:10BF400049FA002D20460CBFA621A721FFF7A0FF2C
:10BF5000606A20B1E16DBDE87040FFF73BBA216C2B
:10BF6000226D0868236A02430A6093B1DA7A82B1CB
:10BF7000D00703D5224A99691160DA7A910703D56F
:10BF8000204AD9691160DA7A520702D51E4A1B6A23
:10BF9000136070BD236A002B2BD0D97A626DE1B19A
:10BFA00072B6D97ACE0706D51848D96806683140E6
:10BFB00099610160D97A880706D51548196906681C
:10BFC0003140D9610160D97A4E0705D511485969C8
:10BFD000066831401962016062B61B68D9689142F7
:10BFE00007D00D4818600D49DA6042F080401861B2
:10BFF0001960226C216D136823EA01031360A0E726
:10C0000000E100E004E100E008E100E080E100E0A0
:10C0100084E100E088E100E001403F0000003F8053
:10C02000436A2DE9F04105460E469046002B3ED06E
:10C0300090F82C100124A14083F83B1083F85E4057
:10C0400083F85D40406A036800211B6808F1FF37F0
:10C050009847FFB2B8F1000F23D03744A046013E05
:10C06000686A16F8011F03681B6898470134B742D5
:10C07000E4B216D0202CF3D10121686AFFF70CFB43
:10C0800095F82C206B6A520083F83B2083F85E8081
:10C0900083F85D80686A036800211B689847012463
:10C0A000DEE7686A0121BDE8F041FFF7F5BAC26B2F
:10C0B000C16C136823EA010306EB080413604FF018
:10C0C0000048A6420ED02B6A16F801EB63B11A683D
:10C0D000C2F82C80C2F834E0D36A002BFCDAA64206
:10C0E000936BF0D1BDE8F081AB6BD5F834C008207C
:10C0F0008021DCF800206F6C1EEA010F14BF3A4368
:10C10000BA43CCF800201A68AF6C3A431A601A6838
:10C11000AF6C013822EA07024FEA51011A60E8D1F8
:10C12000CFE700BF70B50446406A0D46002828D00E
:10C13000A16DFFF74FF920462946FFF7A9FE606A77
:10C1400020B1E16DBDE87040FFF744B9216C226D6C
:10C150000868236A02430A6093B1DA7A82B1D00791
:10C1600003D5234A99691160DA7A910703D5214AE8
:10C17000D9691160DA7A520702D51F4A1B6A136027
:10C1800070BD236A002B2BD0D97A626DE1B172B6F3
:10C19000D97ACE0706D51948D96806683140996121
:10C1A0000160D97A880706D51548196906683140B3
:10C1B000D9610160D97A4E0705D5124859690668D8
:10C1C00031401962016062B61B68D968914207D09C
:10C1D0000D4818600D49DA6042F08040186119601E
:10C1E000226C216D136823EA01031360A3E700BFEB
:10C1F00000E100E004E100E008E100E080E100E0AF
:10C2000084E100E088E100E001403F0000003F8061
:10C210002DE9F041044686B0806A9DF830801E46C4
:10C220000F461546B4F90830002800F04281DA1DA7
:10C2300048BF03F10E02B4F90630D21003FB02F23C
:10C24000002105F0FDFDB4F90820202A00F39280BA
:10C25000B4F90610A34B0120203A733902EBD272D5
:10C2600001EBD1714FF0200E029073208DE8014058
:10C2700042F34F0241F34F01204600F051FE606A45
:10C2800084F82D70002800F04D81002D40F08A8048
:10C29000B4F90830202B14BF3D253C2584F82C50E0
:10C2A000B8F1000F40F0858006B394F93300002800
:10C2B00018DBC0B2012102F0E7F8012194F8330045
:10C2C00002F0CEF8012002F007F9002194F83300C3
:10C2D00002F0C6F80A2002F0FFF8012194F83300BA
:10C2E00002F0BEF8606A002800F08280A16DFFF7BE
:10C2F00071F804227C492046FFF792FE217A013929
:10C30000C9B22046FFF7C4FD784904222046FFF752
:10C3100087FE94F92D30012B14BF142110212046E3
:10C32000FFF7B6FD042272492046FFF779FEB4F903
:10C330000630802B00F09280602B00F0A680D9217F
:10C340002046FFF7A5FD94F92D30012B14BFF121F4
:10C3500022212046FFF79CFD204606226549FFF773
:10C360005FFE606A50B3E16DFFF734F8012006B05C
:10C37000BDE8F081B4F906105F4B0120403A523914
:10C380004FF0400E029002EBD272522001EBD171BD
:10C390008DE8014042F34F0241F34F01204600F087
:10C3A000BFFD6CE76DB284F82C50B8F1000F3FF47C
:10C3B0007BAFFEF7C5FF002E94D076E7216C226D8F
:10C3C0000868236A02430A6073B1DA7A62B1D0075F
:10C3D00003D54A4A99691160DA7A91077CD45207E9
:10C3E00002D5474A1B6A1360012006B0BDE8F08100
:10C3F000236A002B2BD0D97A626DE1B172B6D97A5B
:10C40000CF0706D53F48D968056829409961016082
:10C41000D97A8E0706D53C48196905682940D96143
:10C420000160D97A4D0705D5384859690568294012
:10C430001962016062B61B68D968914207D034481E
:10C4400018603449DA6042F0804018611960226C4B
:10C45000216D136823EA010313604AE7B4F9083039
:10C46000202B00F08680402B7FF469AF2A492046BC
:10C470000322FFF7D5FD94F92D30012B14BFCF21F6
:10C480009F212046FFF704FD59E7B4F90830102B2F
:10C490007FF455AF214920460322FFF7C1FD94F9EF
:10C4A0002D30012B14BFAF2110212046FFF7F0FCE7
:10C4B00045E7DA1D48BF03F10E02B4F90630D21089
:10C4C00003FB02F21046059205F08EF9A0620028E7
:10C4D0003FF44DAF059AB3E6114AD9691160DA7A93
:10C4E0007DE700BF5447010034490100384901008D
:10C4F0003C490100404901004849010000E100E0D9
:10C5000008E100E080E100E084E100E088E100E093
:10C5100001403F0000003F8050470100084C0100EF
:10C5200004E100E0012194F83100244F01F0ACFF58
:10C5300094F83200012101F0A7FF94F9312094F919
:10C54000323057F83220E26357F83330206A2364E0
:10C550000125E56425651A682A431A6078B1B8F1A7
:10C56000000F3FF428AFFFF75BFB002E3FF4BAAE9D
:10C570009BE6042212492046FFF752FDDFE62946DA
:10C5800094F82F0001F080FF294694F8300001F064
:10C590007BFF94F92F2094F9303057F832206263F2
:10C5A00057F833306564A5641A68A36322F001026A
:10C5B0001A60002E3FF496AE77E600BFA45101004A
:10C5C0004C470100B0F90820D31D48BF02F10E030B
:10C5D000B0F90620806ADB1002FB03F2002105F0AF
:10C5E0002FBC00BFF0B50029BDF814502EDBB0F908
:10C5F0000660B1422ADA002A59DBB0F90870144605
:10C600001C44BC42C4BFBB1A1BB2002B1EDDD2B2FD
:10C61000D408D0F828E016FB041112F00702DBB2B0
:10C620000EEB010421D0C2F10807FAB2374F934252
:10C63000BF5C0CD2C3EB020CFF2646FA0CF6012DB0
:10C6400007EA06073FD005D3022D36D0F0BD012DF5
:10C6500039D030D21EF8016026EA07070EF80170C3
:10C660009342F3D3B0F906100C449A1AD2B2072AB7
:10C6700010D9022D36D0002D14BFFF2600261346F8
:10C680002670083BB0F90610DBB2072B0C44F7D834
:10C6900002F00702002AD9D01D4B012D9B5C1DD052
:10C6A00017D3022DD2D1227853402370F0BD13440A
:10C6B0001BB20022A1E7022D25D11EF801607740B0
:10C6C0000EF80170CCE71EF8016037430EF80170D8
:10C6D000C6E7227822EA03032370F0BD22781343D1
:10C6E0002370F0BD11462378DB4323700839B0F97D
:10C6F0000630C9B207291C44F5D812F00702A5D0AC
:10C70000034B9B5CCFE73444AFE700BFEC4601002E
:10C71000DC46010070B4C47DBDF80C50022C18D06A
:10C72000032C1FD0012C0BD0002A03DBB0F90840EA
:10C73000944201DC70BC7047039570BCFFF7B0BA3F
:10C74000C4880395013CA41A0A4621B270BCFFF7C5
:10C7500049BF0689C488013E641AB21AE41A12B2AB
:10C7600021B2E1E704890395E41A641A114622B262
:10C7700070BCFFF737BF00BF70B4C57DBDF80C605B
:10C78000022D1AD0032D12D0012D03D0039670BCB8
:10C79000FFF728BFC488E41AA41A0A4621B2002A67
:10C7A00003DBB0F90840944213DC70BC7047048985
:10C7B000013C641A114622B2F1E7C4880589039648
:10C7C000013CAD1AED1A621A11B22AB270BCFFF721
:10C7D00009BF039670BCFFF763BA00BF2DE9F843A9
:10C7E0000446406A002863D0A16DFEF7F3FD0522E0
:10C7F00074492046FFF714FCA1790139C9B22046DB
:10C80000FFF746FBB4F90820E588A66AD31D48BFA8
:10C8100002F10E03DB10626A15FB03F51FFA85F8BF
:10C82000002A7BD094F82C300125AB4082F83B30B5
:10C8300082F85E5082F85D50606A036840211B6890
:10C8400008F1FF379847BFB2B8F1000F23D0374443
:10C85000A846013E606A16F8011F03681B689847E6
:10C860000135B742EDB216D0202DF3D10121606A17
:10C87000FEF712FF94F82C20636A520083F83B20E5
:10C8800083F85E8083F85D80606A036840211B68DE
:10C8900098470125DEE70121606AFEF7FDFE606A28
:10C8A000002800F08D80E16DBDE8F843FEF792BDF1
:10C8B000236A002B2BD0D97A626DE1B172B6D97A96
:10C8C000CE0706D54048D9680568294099610160BE
:10C8D000D97A8D0706D53D48196905682940D9617F
:10C8E0000160D97A480705D5394859690568294052
:10C8F0001962016062B61B68D968914207D0354859
:10C9000018603549DA6042F0804018611960226C85
:10C91000216D136823EA0103136068E7E26BE36C9F
:10C920001168276A0B4306EB080913604FF0004EAD
:10C930004E450DD016F801CB2FB33A68C2F82CE063
:10C94000C2F834C0D36A002BFCDA4E45936BF1D1A8
:10C95000226C236D11680B43136097B1FB7A83B18E
:10C96000D90703D51D4BBA691A60FB7A9A0703D51C
:10C970001B4BFA691A60FB7A5B0702D5194B3A6ABE
:10C980001A60BDE8F883A36BD4F8348008208021B6
:10C99000D8F80020656C1CEA010F14BF2A43AA4393
:10C9A000C8F800201A68A56C2A431A601A68A56C9A
:10C9B000013822EA05024FEA51011A60E8D1B7E7CF
:10C9C000276AC5E7E446010080E100E084E100E079
:10C9D00088E100E001403F0000003F8000E100E00E
:10C9E00004E100E008E100E02DE9F04F85B0994650
:10C9F000BDF93870BDF83CA0BB1AC1EB090B002B88
:10CA0000B8BF5B42BBF1000FB8BFCBF1000B5B4579
:10CA10000D4616460093804648DC4D453A4633465F
:10CA20004CDC194613460A46C5EB09019B1A89B22C
:10CA3000002B0CB2B8BF5B4204EBD474BE42ACBF57
:10CA40004FF0FF3201224D45039102924FEA6404F8
:10CA500029DC9BB201930DE0D8F80070BF69B8479C
:10CA6000019BE41AA3B21CB20135002C2DB211DBDC
:10CA7000A94518DB009B5B452A4653463146404694
:10CA8000EADCD8F8002053469769294632464046EA
:10CA9000B847E5E7029A1644039AA94502EB030456
:10CAA00036B224B2E6DA05B0BDE8F08F4A462B462E
:10CAB000B94635464D4517461E46B2DD3046294635
:10CAC0003E464D4607468946AEE700BF10B40468AF
:10CAD0002469A44610BC604730B40468BDF808500F
:10CAE0000295A46BA44630BC604700BF30B4046814
:10CAF000BDF808500295E46BA44630BC604700BF07
:10CB000070B40468BDF90C60BDF81050039604952C
:10CB1000246CA44670BC6047704700BF10B582B05B
:10CB2000B0F90C2001910168009200220C6CB0F960
:10CB30000A301146A04702B010BD00BF704700BFC9
:10CB400001F003010129C17506D0032904D0C28870
:10CB500003894281838170470289C388428183812E
:10CB6000704700BF2DE9F0410568134E6F6986B02C
:10CB7000B7420446BDF8308010D1013B13441BB2CC
:10CB80000093CDF804800B46AD6A2046A847236881
:10CB9000DB6AB3420AD106B0BDE8F0810593049286
:10CBA0000391B84703A925680EC9E6E7204606B0F9
:10CBB000BDE8F041184700BF19CB00002DE9F04156
:10CBC0000568124E6F6986B0B7420446BDF83080E2
:10CBD0000FD1013BCDF804800B4400921BB2AD6A2B
:10CBE0002046A8472368DB6AB3420AD106B0BDE8F5
:10CBF000F081059304920391B84703A925680EC9F3
:10CC0000E7E7204606B0BDE8F041184719CB000021
:10CC10002DE9F04F0568DFF858B06F6985B05F45C2
:10CC20000646BDF93890BDF83CA00C46904615D19B
:10CC30001F19BC420CDACDF800A0214601342D6A40
:10CC40004B464246304624B2A847BC423568F2DB28
:10CC5000EB6A5B4507D105B0BDE8F08F0393B84799
:10CC60003568039BE4E7304605B0BDE8F04F184750
:10CC700019CB00002DE9F04387B099420546BDF974
:10CC80003840BDF83C6025D0A24212D00768DFF8DA
:10CC90008080D7F81490C14532D18DE850002846E5
:10CCA000BC6AA0472B68DB6A434524D107B0BDE8C6
:10CCB000F083994202DD08461946034628680E961D
:10CCC000C46B01335B1A1BB22846A44607B0BDE80B
:10CCD000F0436047A24202DD134622461C46286804
:10CCE0000E96631C846B9B1A1BB22846A44607B0A1
:10CCF000BDE8F0436047284607B0BDE8F043184759
:10CD0000059304920391C84703A92F680EC9C4E78D
:10CD100019CB00002DE9F04FD0F800E0DFF890903B
:10CD2000DEF814B083B0CB450446BDF93080BDF8C1
:10CD300034A00D4617461E4631D1CDF800A0DEF8CE
:10CD400024B0294633463A462046D8472368CDF8D2
:10CD500000A008F1FF323A44D3F824B0294612B2B9
:10CD600033462046D8472368CDF800A02946D3F89B
:10CD700020B03A4643462046D8472068CDF800A068
:10CD8000711E29444346056A09B23A462046A8471F
:10CD90002368DB6A4B4506D103B0BDE8F08FD84766
:10CDA000D4F800E0C9E7204603B0BDE8F04F1847CB
:10CDB00019CB0000F0B4002401264FF6FF75094F8F
:10CDC00007600471C475C48104824476C4618675A9
:10CDD000067685824582C180028141818281F0BCD4
:10CDE000704700BF144C01002DE9F04F85B0066874
:10CDF000BDF84450BDF93880CDF800800446019557
:10CE0000D6F848B00392BDF93C60BDF94070894640
:10CE10009A46D84723680195009742465146D3F871
:10CE2000488020463346C0472068039B0E930F95E9
:10CE3000856C4B463A4631462046AC4605B0BDE8C7
:10CE4000F04F60472DE9F04F87B01746BDF94040DD
:10CE500000912546E91D059344BF2B4603F10E01C1
:10CE60000268BDF8486053690294C91003912B49C8
:10CE7000BDF9444001968B42824645D1002C3CDDF1
:10CE8000029B3C445E1EB6B24FF0000923B20493ED
:10CE900001364D46029B002B28DD059B002403EB49
:10CEA000090806E0EDB22B0604F1010411D4A642F4
:10CEB0001CD0A1B211F0070F23B24FEA4505F1D102
:10CEC000002BB8BF0733DB10013418F803502B06D2
:10CED000EDD5009BD2F818B019443A4609B2019B2F
:10CEE0005046D847A642DAF80020E2D1039B01372A
:10CEF0009944049B3FB2BB42CCD1D36A074A9342C8
:10CF000006D107B0BDE8F08F9847DAF80020B5E702
:10CF1000504607B0BDE8F04F184700BF19CB0000DE
:10CF200070B4BDF90C60BDF91050BDF81440039603
:10CF30000495059470BCFFF785BF00BF2DE9F04F45
:10CF400093B090460591C1691090BDF870000790AC
:10CF5000BDF874909DF878A00493002900F0CD806E
:10CF60000A7A0AC9894604998A1AD2B203EBC20323
:10CF7000BAF1010FDA780B9293F905201E8893F825
:10CF800002B00F9293F9064079D913B2099323B2F4
:10CF90000C93109B1A68A94B1193194653698B4245
:10CFA00040F0A6800B9B002B55D01FFA88F3002180
:10CFB0000D93C8462344DDF8409006910E930F462A
:10CFC0000C46BBF1000F3FD0BDF818100C9B039727
:10CFD0001FFA8AF0CB1813FB00F304900E9801445B
:10CFE0000D98034409B21BB20A910893002505E08D
:10CFF0000135EBB264009B45E4B222D9039B2B447C
:10D00000590703D1731C18F806409EB22306EFD5CA
:10D01000099BBDF81000E91811FB00F10598BAF161
:10D02000010F0FFA8AF301441CD007980190009376
:10D03000D26909B217464846089AB847D9F800207D
:10D04000D6E7039F5F44FFB2069B0B99013306931B
:10D05000DBB29942B5D8D36A119A934243D113B047
:10D06000BDE8F08F0F9B191893690A9A29441F464F
:10D0700009B2079B4846B847D9F80020B8E7002313
:10D080000C93099385E70A9A0D9B0132013B52B23A
:10D0900013F0FF030A920D936FD1DDF81890079BF0
:10D0A000DDF83C80DDF820A04B4517D0BAF1010F28
:10D0B00000F0C8800B9A109DCDF804900BEB8B010B
:10D0C0004FEACB030A4400931146DEF81C40534656
:10D0D000424609B22846A047D5F800E0DEF82C30D9
:10D0E000119A9342BBD0109813B0BDE8F04F184787
:10D0F000109D284698472A6854E7109A0598B2F977
:10D100000A308342ABDDB2F90C304345A7DD06237C
:10D1100013FB0A03002BA2DD08EBCA03002B9EDDE4
:10D12000537E2BB9049BAF2B02D90133DBB204939E
:10D13000109BD3F800E0414B11931A46DEF81430EF
:10D14000934240F08E801FFA88F30E9308339BB20F
:10D15000BDF81420059305230D9300230A93CDF801
:10D160003C800FFA8AF3DDF84080CDF818900B92DE
:10D170001FFA8AFBCDF820A099460A9ABDF8100044
:10D180000B9C0E9D0523194611FB00232C481146CC
:10D19000C75C039702FB0B4214FA81F312B21BB275
:10D1A00009920C932C462E461CE0089B0999012BF2
:10D1B0002AB24B4640462DD0079F0197CDF80090EC
:10D1C000DEF81CA0D047D8F800E0039B5B080134D0
:10D1D0000393059BA4B25D445E44A342ADB2B6B2D4
:10D1E0003FF451AF039BD807DFD4079B069A9342C5
:10D1F000EBD0089B012B16D0069B0193CDF8009035
:10D20000DEF81CA009994B4632B24046D047D8F808
:10D2100000E0DAE7DEF818A0079B0C9922B2D047AD
:10D22000D8F800E0D1E7DEF818A00C991346404684
:10D2300022B2D047D8F800E0C7E700BF19CB000002
:10D24000644C01000B99109DCDF800900531DEF87B
:10D25000204009B2424608232846A047D5F800E0FE
:10D260003CE7109C20469847D4F800E06BE700BFED
:10D27000F0B5C36985B004462BB30A2968D00D29DF
:10D280004AD01A7A914247D3587A884244D35D688B
:10D290008A1A05EBC205AA78002A50D0E87800283F
:10D2A0004DD0207E00283AD095F905E0B4F90E0063
:10D2B000A67DB4F90A70724406FB0202BA4262DC2F
:10D2C000B4F9102030E00A2956D00D2924D0027E6E
:10D2D000002A4BD0B0F90E00A57DB4F90A600622F1
:10D2E00012FB0502B2423EDD228AE38102EBC50257
:10D2F00012B218462282A78A668A02950B468DE8EA
:10D30000C00001462046FFF719FEA37DE28903EB2A
:10D31000430302EB4303E381012005B0F0BDA67D8A
:10D32000B4F90E00B4F91020B4F814E0678A02963C
:10D330000B468DE8804001462046FFF7FFFD297926
:10D34000E389A27D012001FB0233E38105B0F0BD3A
:10D350000022C2819A7A817D038A01FB0233038213
:10D36000012005B0F0BDB4F91020C4E7857DB4F903
:10D370001020B0F90E00BEE7028A817DC38102EB66
:10D38000C1030382C8E70020E0819B7A228A03FB65
:10D39000062212B22282C7E7C1810282704700BF13
:10D3A000002908BF01218175704700BF8182418239
:10D3B000704700BFC07D7047B0F90A00704700BFDA
:10D3C000B0F90C00704700BF10B4EFF3108272B6D2
:10D3D000437F33B9017F012907D003290FD00123EF
:10D3E000437702B962B610BC7047124C2168A1B1F4
:10D3F000114943610B68836108605861EFE70F4C86
:10D40000216881B10E4943610B68836108605861EE
:10D410000C4B4FF080511960E1E7074B416181618E
:10D4200020601860DBE7064B416181612060186075
:10D43000EEE700BFC0A0FF1FBCA0FF1FB0A0FF1FF2
:10D44000B4A0FF1F04ED00E070B5EFF3108272B6D8
:10D450000C4C206880B10C4E00254369236073B1E9
:10D460009D6102B962B6457783689847EFF31082F1
:10D4700072B620680028F0D102B962B670BD336080
:10D48000EFE700BFB0A0FF1FB4A0FF1FFFF7DCBF96
:10D49000184A30B41468002C27D0036821688B42E6
:10D4A0000ED2CB1A00218460C1602360E06010605E
:10D4B0000223037530BC704711688B42144608D3B1
:10D4C000A2685B1A0360002AF6D18260C460A06083
:10D4D000EEE7D268C2608460E060C568CB1A0222C1
:10D4E000A8602360027530BC70478460C46010601F
:10D4F000DEE700BFB8A0FF1FF8B5224E34682CB39A
:10D500002368002B3AD1204F1D4604E03468ECB16B
:10D510002368002B32D1A36803B1DD60206933603A
:10D52000036825751B68BB4221D1037F4560022B30
:10D53000C46020D0FFF748FF6368002BE6D023606B
:10D540002046FFF7A5FF3468002CE1D1EFF31083EC
:10D5500072B60E4A00211068116003B962B628B194
:10D560008468FFF795FF20460028F9D1F8BD2246D0
:10D5700000219847E0E783689847DDE7013B236097
:10D58000E4E700BFB8A0FF1F09BC0000C8A0FF1F50
:10D59000024A136801331360FFF7AEBFD4A0FF1F28
:10D5A000704700BF0368F0B4FBB1002501249D6003
:10D5B000DC601B4C1A601C44241104F144056A1100
:10D5C000032692009E60174F0679174B47F82410E8
:10D5D00002F1604202F5614205F01F05012000FAE8
:10D5E00005F5E6541560F0BC7047104C236843F411
:10D5F0000003236000BF0E4B0E4DA4F58734A4F545
:10D600009E7401261E60234604609C68002CD0D0C6
:10D610001033AB420360F8D1002303601846E2E701
:10D62000008FFCBFC492FF1F44E400E03C80044034
:10D6300000700340407103400168A9B10B4BF0B486
:10D640000B441B110A4E0B4F0B4D46F8237003F190
:10D65000440202F01F0401235211A340002445F8A4
:10D6600022308C600460F0BC704700BF008FFCBFAC
:10D67000C492FF1FA1D5000080E100E0024A034BE5
:10D68000012111601B6818470C710340C492FF1FF1
:10D69000024A034B012111605B6818471C7103406B
:10D6A000C492FF1F024A034B012111609B68184777
:10D6B0002C710340C492FF1F024A034B01211160E9
:10D6C000DB6818473C710340C492FF1FF8B50E4653
:10D6D00071B17AB10746144600253B6816F8011B64
:10D6E0001B6838469847013C0544F6D12846F8BDEA
:10D6F0000846F8BD1046F8BD00B5064A0368128812
:10D700005B6883B001A9ADF804200222984703B0FA
:10D710005DF804FB64510100F0B507468BB0002AA8
:10D7200033D0012A08BF0A2251B3212400E0F4B209
:10D73000B1FBF2F502FB1511C8B2092900F1300165
:10D7400098BFC8B20AA988BF3730214488BFC0B289
:10D7500001F8240C661E2946002DE8D133B1013CA6
:10D76000E4B20AAB23442D2203F8242C3B6801AA1F
:10D7700011195B683846C4F1220298470BB0F0BD1E
:10D7800030228DF825202124E8E70368C9B21B6800
:10D7900098470BB0F0BD00BF0029BABF49422D2306
:10D7A00000230A22FFF7B8BF374A384913681B061F
:10D7B000FCD40B6813F08003F8D172B634490A78B0
:10D7C000002A5FD0334A3448F0B4344C17680668F6
:10D7D0002568D4680C303E44143200681268304F1B
:10D7E00035442C4420440244C2F34E022D4E2E48B0
:10D7F0002E4D2F4C42F400423A60376806682D687F
:10D800002C4A24680C303E44006812682A4F354484
:10D810002C4420440244C2F34E02284E2848294D8D
:10D82000294C42F400423A60376806682D68274A5E
:10D8300024680C303E4400681268254F35442C445F
:10D8400020440244C2F34E02224E2348234D244C6E
:10D8500042F400423A60376806682D68214A24681D
:10D860000C303E440068126835442C442044024485
:10D87000C2F34E021C4842F4004202600B7062B6D2
:10D88000F0BC704762B6704724B0034024B00B4030
:10D89000CDA0FF1F38B003403CB0034040B0034070
:10D8A0002CB0034058B003405CB0034060B003406C
:10D8B00064B003406CB0034030B0034038B00B405C
:10D8C0003CB00B4040B00B4044B00B404CB00B4060
:10D8D0002CB00B4058B00B405CB00B4060B00B401C
:10D8E00064B00B406CB00B4030B00B4030B42948F2
:10D8F000294A2A4B2A4D6024E121047011701B78BB
:10D90000284C082B30D00A2B2748284937D00C2B1D
:10D910000CBF35223D2212232A60236002600B6077
:10D92000234B24491B78244ABBB101230B601360AD
:10D93000224B23491B78234A012B26D9042B0FD9CC
:10D94000082B1ED9102B94BF862387230B601360EE
:10D950001D4B01221A7030BC70470B601360E7E763
:10D9600084230B601360F3E700F58E200F49083025
:10D97000012213232A60236002600B60D0E7392262
:10D98000F7E785230B601360E2E780230B601360E9
:10D99000DEE700BF0040074001400740D492FF1F70
:10D9A00008B003400CB0034008B00B400CB00B4073
:10D9B000D0A0FF1F20B0034020B00B40D592FF1F26
:10D9C00024B0034024B00B40CDA0FF1F0C2830B47E
:10D9D00017D91023984228BF18461C46104A114DEB
:10D9E0001178181A8C42287018D00F4913700B78D0
:10D9F00023B10E490E4A00230B60136030BCFFF7C1
:10DA000075BF0A2802D90C231C46E7E7082802D96B
:10DA10000A231C46E2E708231C46DFE730BC7047B8
:10DA2000D492FF1FCCA0FF1FCDA0FF1F24B0034046
:10DA300024B00B4028282FD8334B2DE9F0411E5C31
:10DA4000FF2E2BD0314B1B78002B2AD132062CD441
:10DA500072B62F4D2F4C2F46012326602B7062B6D5
:10DA600072B623681B060CD43B781BB9F4E72B78FD
:10DA7000002BF1D062B602F073FB72B62368180671
:10DA8000F5D5254B1B6800222A7062B6234A107810
:10DA900043FA00F0BDE8F081002070470020BDE8A7
:10DAA000F081FFF781FE3206D2D572B61C4DDFF849
:10DAB0007C801C4C06F04007FFB206F03F06D8F809
:10DAC0000030DFB123F01003C8F8003001232660D6
:10DAD000134A2B7062B672B6236819060CD41378F9
:10DAE0001BB9ECE72B78002BE9D062B602F038FBCB
:10DAF00072B623681B06F5D50B4BC3E743F0100342
:10DB0000C8F80030E2E700BF68510100CDA0FF1F58
:10DB1000CFA0FF1F00B0034010B00340CCA0FF1FF8
:10DB2000CEA0FF1F00B00B4010B00B400CB00B405C
:10DB30000A4A0B49136843F4805313600B7843B9C6
:10DB4000084BC0221A70084B80F30C0000B21880FA
:10DB50007047044B80221A70F5E700BF2C80044008
:10DB6000D0A0FF1F21C00C4000C00C40F0B51B4BE3
:10DB70001B4E596818689A68DB6885B06C460FC4FC
:10DB8000337899071DD5174A174C1378174913F0A6
:10DB9000700318BF1370164A164B802717700026A3
:10DBA0003320032226706D4608701A7072B6043C4A
:10DBB00045F001052046A84762B6237813F07003AC
:10DBC00009D10D4B064901E0013B02D00A78D2078A
:10DBD000FAD505B0F0BD237005B0F0BD9451010039
:10DBE0000100024000000240040002400B0002401D
:10DBF000070002400A000240410D0300B0F5006F2B
:10DC00000AD210B5094B1B78DB07044606D504F190
:10DC1000A0500078C0B210BD00207047FFF7A6FFEB
:10DC200004F1A0500078C0B210BD00BF0100024056
:10DC3000B0F5006F17D238B50F4B1B78DA070D46D9
:10DC4000044611D504F1A0500378AB420AD00B4A28
:10DC5000137813F0700318BF1370074A0570137818
:10DC6000DB07FCD538BD7047FFF780FF04F1A050FB
:10DC70000378AB42EBD1F5E701000240000002401F
:10DC800008B5F4F703F8F4F749FF02F069FAFAE788
:10DC9000844641EA000313F003036DD1403A41D3B7
:10DCA00051F8043B40F8043B51F8043B40F8043B76
:10DCB00051F8043B40F8043B51F8043B40F8043B66
:10DCC00051F8043B40F8043B51F8043B40F8043B56
:10DCD00051F8043B40F8043B51F8043B40F8043B46
:10DCE00051F8043B40F8043B51F8043B40F8043B36
:10DCF00051F8043B40F8043B51F8043B40F8043B26
:10DD000051F8043B40F8043B51F8043B40F8043B15
:10DD100051F8043B40F8043B51F8043B40F8043B05
:10DD2000403ABDD2303211D351F8043B40F8043BA5
:10DD300051F8043B40F8043B51F8043B40F8043BE5
:10DD400051F8043B40F8043B103AEDD20C3205D3B5
:10DD500051F8043B40F8043B043AF9D2043208D0AD
:10DD6000D2071CBF11F8013B00F8013B01D30B881F
:10DD700003806046704700BF082A13D38B078DD0FD
:10DD800010F003038AD0C3F10403D21ADB071CBFCF
:10DD900011F8013B00F8013B80D331F8023B20F839
:10DDA000023B7BE7043AD9D3013A11F8013B00F872
:10DDB000013BF9D20B7803704B7843708B788370FA
:10DDC0006046704708B5104C08E0236859050DD42B
:10DDD00023681A050FD42368DB0411D42368580381
:10DDE000F3D501F065F823685905F1D502F01CFA66
:10DDF00023681A05EFD500F07FFD2368DB04EDD51D
:10DE000000F0C8FEEAE700BF3480044008B5FFF721
:10DE1000D9FF00BF014B10221A8070470020054037
:10DE2000704700BF094908B50B6830B16A4618440D
:10DE3000A2F58052904202D20860184608BD03F055
:10DE4000A5FC0C2303604FF0FF3008BDD892FF1FE4
:10DE5000FEE700BFEFF3138070B9EFF310836BB9E7
:10DE6000EFF305825AB94FF48070EFF311832BB1B1
:10DE7000984228BF184670474FF0FF3070470F2A6E
:10DE800001D81846F1E7014BD05CEEE7F0E300E083
:10DE9000F0B44D1E2E46002400E00134B0FBF2F336
:10DEA00002FB1300092800F130078ABF3730F8B2AF
:10DEB000C0B206F8010F1846002BEED10A195370B4
:10DEC0004CB1107815F8016F28700133E01A8342C5
:10DED00002F80169F5DB0846F0BC7047704700BFE7
:10DEE00010B40F4B53F8302092F880422CB101232C
:10DEF00069B182F8803010BC704703EBC0035B68E7
:10DF00001A6841B922F002021A6010BC704782F808
:10DF1000003110BC704742F003021A6010BC704719
:10DF2000A45101001C4A02EBC00301295B6811D017
:10DF300004291BD052F83000002280F8802229B139
:10DF4000022920D0032922D01A6070474FF4807232
:10DF50001A60704752F830004FF4A27280F88012B5
:10DF60001A601A6822F020021A60704752F83010C6
:10DF70004FF4A272012081F880021A601A6842F000
:10DF800020021A60704740F203121A6070474FF483
:10DF900081721A60704700BFA4510100212848D83F
:10DFA000F8B5042A44D8DFE802F0484B4E03450098
:10DFB0004FF410262B4B03EBC0030D465C68216821
:10DFC00011F4E06148D0284B284A2949C3F89C2124
:10DFD00004F140422748C3F8A411A2F59221264F2C
:10DFE000C3F8A0017C292548C3F8A871C3F8AC0187
:10DFF0002CD9A2F594237C2B2AD9A2F596237C2B2D
:10E0000028D9A2F598237C2B29D9A2F59A227C2A1B
:10E0100027D81B4872B6236823F4702343F080721C
:10E02000C4F384011643236040F82150266062B691
:10E03000F8BD70474FF43026BCE74FF40026B9E72F
:10E040004FF44026B6E74FF42026B3E70D48E1E74A
:10E050000D48DFE70D48DDE7FFF764FFB3E70C4845
:10E06000D8E7F8BDA45101000082FF1FF188FF1F0F
:10E070009988FF1FC588FF1F6D88FF1F4188FF1FFC
:10E08000B493FF1FDC92FF1F1493FF1F6493FF1FC5
:10E090009493FF1F1A4B03EBC00010B4426802F1C7
:10E0A0004043A3F592217C2923D9A3F594217C290F
:10E0B0000DD9A3F596217C291FD9A3F598217C2998
:10E0C00019D9A3F59A237C2B11D80E4C00E00E4CE5
:10E0D00072B613680D4823F08773C2F3840123F4EA
:10E0E000803343F08073136044F8210062B610BCA3
:10E0F0007047074CECE7074CEAE7074CE8E700BF3E
:10E10000A4510100B493FF1F1493FF1FDDDE000034
:10E11000DC92FF1F9493FF1F6493FF1F30B4054BE5
:10E12000054D064C002210211A602A6020601960FB
:10E1300030BC704714D0034004D0034000D00340EB
:10E14000282838B52ED0002904464FDD5F4B1B78B8
:10E15000012505FA03F28A4202D8212837D938BDB1
:10E160000338C2B2012A3AD9202C4AD0192C48D0FF
:10E17000574A126802FB011222FA03F31D2800F22B
:10E180009B80DFE800F0928B847D9999766F999956
:10E190009999999999999968615A53994C9999992A
:10E1A00099999945494B1B780B2B08D90C2B1CBF0F
:10E1B0000C3B19410846BDE83840FFF7B9BCC3F134
:10E1C0000C0399400846BDE83840FFF7B1BC29462A
:10E1D000FFF786FE2946BDE83840FFF7A3BE3D4A5B
:10E1E000126802FB011222FA03F3C7E72128B6D80E
:10E1F0000021FFF775FE20460121BDE83840FFF7FA
:10E2000091BE354A126802FB011222FA03F3B5E708
:10E210003249334A0B604FF45173136038BD3149B2
:10E22000314A0B604FF45173136038BD2F49304AA7
:10E230000B6040F24443136038BD2E492E4A0B60F8
:10E2400040F24443136038BD2C492D4A0B6040F224
:10E250004443136038BD2B492B4A0B6040F24443C2
:10E26000136038BD29492A4A0B6040F244431360C9
:10E2700038BD2849284A0B6040F24443136038BD3A
:10E280002649274A0B6040F24443136038BD2549B4
:10E29000254A0B6040F24443136038BD2349244AA9
:10E2A0000B604FF45173136038BD2249224A0B6052
:10E2B0004FF45173136038BD212C3FF650AF7F29C6
:10E2C000D4BF00210121204693E700BFBC93FF1F6C
:10E2D000088003400890034008800B4010800B40EA
:10E2E00048A0044018800B404CA004401880034014
:10E2F00008B004401080034004B004404080034054
:10E3000018C004403880034014C0044028800340F3
:10E3100010B00440208003400CB004403080034023
:10E3200010C00440488003401CC0044018900340C3
:10E3300034900440109003403090044038B11028CD
:10E3400028BF1020044AC3B2107813707047024AE5
:10E350000123107813707047BC93FF1F2DE9F84319
:10E360000E4680463249334D304603F095F947F664
:10E37000122300281ABF1D464FF002094FF0010971
:10E38000002425FA04F002F091FF4FF05E51074699
:10E3900002F0E4FF0146304603F092F930B901344F
:10E3A000072CEED1E80902F081FF074631463846D6
:10E3B00003F088F84FF07C5102F0C6FE03F0BAF982
:10E3C0004FF6FF729042A8F1030328BF1046012BBD
:10E3D00029D9B8F1170F17D8174B23FA08F303F010
:10E3E000010383F0010223B9B8F1190F0FD0BDE882
:10E3F000F883124B124D13491A6044EAC9042A608B
:10E4000008601C60BDE8F883B8F1200FECD10E4B1A
:10E410000E4D0F49002244EAC9041A602A600860C0
:10E420001C60BDE8F8830B4B0B4D0C49F2E700BFB5
:10E43000001BB740006CDC026006F0000080034067
:10E44000048003400880034000800B4004800B40A0
:10E4500008800B4000900340049003400890034064
:10E46000212801D8FFF73CBD704700BF212806D8FE
:10E47000044B53F8303093F80002C0B270470020CC
:10E48000704700BFA4510100212801D8FFF74ABD01
:10E49000704700BF72B60C490C4B0D4A1B680868E8
:10E4A000126862B6520102D5322B88BF0130094989
:10E4B000C3F5BB334FF47A72FF33A1FB031302FBA6
:10E4C00000F000EB93107047D4A0FF1F18E000E0AD
:10E4D00004ED00E0ABAAAAAA2DE9F843054672B6FE
:10E4E000204F214B214A1B683C68126862B65201DA
:10E4F00002D5322B88BF013495B3C3F5BB331C4E14
:10E50000DFF86490DFF86480FF334FF47A72A6FB83
:10E51000031302FB04F404EB931472B6D9F8001051
:10E520003A68D8F800E062B6C1F5BB33FF33A6FB0A
:10E5300003031EF0806FC4EB93134FF47A7002D084
:10E54000322988BF013200FB0233B3F57A7F04D34E
:10E55000013D05D004F57A74DFE701F001FEDCE748
:10E56000BDE8F883D4A0FF1F18E000E004ED00E050
:10E57000ABAAAAAAF8B52D4B2D49DFF8D0E0DFF8F9
:10E58000D0C02C4E2C4D2D4C2D4A2E4F4FF4000058
:10E5900018604FF0807018604FF0007018604FF0F6
:10E5A000806018604FF00060186000200860282329
:10E5B0004BF6FF71CCF80010CEF8003033601360DA
:10E5C0002B6023603B60B3629362092245F8242CE0
:10E5D000C4F8D80F05F57F65C7F8D41F07F5FF27E6
:10E5E00007F5FA67C6F8F83F2B6006F5FF26C4F872
:10E5F000D42F05F5FD2504F5FF24386006F2F476E6
:10E600001148316005F5FF6504F5FD642B6023605A
:10E610000260FFF76BF91920FFF75EFF01F08EF93A
:10E6200040F21310BDE8F840FFF756BF08E100E0E4
:10E630000480034014800340248003402C80034066
:10E640001C8003403480034000800B400C8003405A
:10E65000088003402B4A2C491368F0B543F400634B
:10E6600013600A78294F2A4E2A4D2B4C2B49002340
:10E67000092A3B7033702B7023700B703DD01A2A1F
:10E6800021D0274B1B780A2B25D01F2B30D01F28D9
:10E6900027D8002002460125224B234C1A7023491B
:10E6A0005D7004224FF0020E88273C2640259872A8
:10E6B0009A704FF4004083F813E05A751F74DE70AF
:10E6C00025700860F0BD1A4B40F213321A60144BEB
:10E6D0001B780A2BD9D1174B4FF451721F281A609F
:10E6E000D7D9C0F34432C0F3471500F01F00D3E779
:10E6F000114B4FF451721A60C9E7104B40F21332BC
:10E700001A60BEE734800440BD93FF1F48A1FF1F7D
:10E71000DDA0FF1F50A1FF1F49A1FF1FDCA0FF1FAD
:10E72000BE93FF1F00B006402FE400E004E100E0CC
:10E7300004D0044010B0044000D004400CB00440A9
:10E7400009B140F08000174A1378984216D010B4EF
:10E75000154C246824050FD503F07F030A2B1CD029
:10E760001F2B11D0002900F07F0114BF6023442328
:10E770000A290DD01F2902D0107010BC70470B4918
:10E7800043F440730B60F7E7084B00241C60E9E793
:10E79000074943F440730B60EEE7054B00241C600F
:10E7A000E0E700BFBE93FF1F3480044000D0044068
:10E7B00010B00440124B1A7882420CD011490968FB
:10E7C000090507D5092A16D01A2A0AD009280DD01A
:10E7D0001A2801D0187070470B4A40F213311160AB
:10E7E000F8E7094A002109281160F1D1074A40F2EF
:10E7F00013311160EEE7054A00211160E6E700BF22
:10E80000BD93FF1F3480044004D004400CB004408A
:10E810002DE9F84F234B1B681A053BD5224B1B688B
:10E820000BB101221A70DFF89090204D99F800404A
:10E83000DFF888801E4E0134272C8ABF4FF0000A73
:10E840005FFA84FA54460746AB462B789C4216D1B1
:10E85000FFF700FB40281FDC33791B06F5D59BF83A
:10E8600000300133272B86BF00221346DAB218F896
:10E870000330DBB2F3712A702B789C42E8D00D494B
:10E880000B4BFFB20120BC2208F80470087089F815
:10E8900000A0DA70BDE8F88FFF28D6DD01F060FC3B
:10E8A000D3E700BF348004404CA1FF1F49A1FF1FE4
:10E8B00000B00640DCA0FF1F50A1FF1FE0A0FF1F1B
:10E8C00010B5044C237823B101F04AFC2378002BC7
:10E8D000FAD110BDDCA0FF1F054A064B10781B784B
:10E8E000C0B2DBB2984238BF4030C01A704700BF98
:10E8F00048A1FF1FDDA0FF1FF0B4384B1A7912F0BA
:10E90000300F2CD072B6997D01F0FF0200293DD066
:10E9100062B6334F334938780D78334E1C46C0B257
:10E92000EDB2431C402BE17928BF0023AB4202F13A
:10E93000FF32C9B21CBFF154184612F0FF02F0D1E9
:10E940002A4B1B68C2B23A704BB1A84236BFC5F120
:10E950004005401B40192728C4BF01221A701F49D7
:10E96000CA78D2B2150616D452060DD51B4B1B79A8
:10E970005B0609D51E4B1F491B6800220A7003B1B4
:10E980001A70164B3C22DA70F0BC70474022D979DD
:10E990005A7462B6E3E70B791C06E5D5164B174EA1
:10E9A0001C783378E4B2DBB29C420ED0144D01E007
:10E9B000A3420AD00133282B28BF00230879E85C42
:10E9C000C0B2C871087D0728F2D9DBB203493370A1
:10E9D0000B79180644BF7C23CB70C5E700B0064016
:10E9E00048A1FF1FDDA0FF1F08A1FF1FD8A0FF1F28
:10E9F0004CA1FF1FDCA0FF1F50A1FF1F49A1FF1F5B
:10EA0000E0A0FF1F2DE9F84F214B1B6807460BB113
:10EA100001221A70DFF888901E4D99F80040DFF847
:10EA200084801D4E0134272C8ABF4FF0000A5FFA04
:10EA300084FA5446AB462B78A34216D1FFF70AFA64
:10EA400040281FDC33791B06F5D59BF800300133D5
:10EA5000272B86BF00221346DAB218F80330DBB248
:10EA6000F3712A702B78A342E8D00C490A4BFFB20D
:10EA700008F804700120AC22087089F800A0DA7050
:10EA8000BDE8F88FFF28D6DD01F06AFBD3E700BFB1
:10EA9000C8A1FF1FC5A1FF1F00C00640C4A1FF1FE2
:10EAA000CCA1FF1F5CA1FF1F1C4BDFF894C01A68AC
:10EAB0001B49F0B542F480521A4D1A60DFF884E029
:10EAC000194F1A4E1A4C00238CF800304FF4517233
:10EAD0002B701F2840F213358EF800303B703370D6
:10EAE00025600A6012D819460124124A124D11708D
:10EAF0001248547000212C27402693724FF40034A2
:10EB000091701174D7702E700460F0BDC0F3443161
:10EB1000C0F3471400F01F03E7E700BF3480044050
:10EB20000CC0044059A1FF1FC5A1FF1FC4A1FF1FB6
:10EB300008C0044000C0064031E400E004E100E009
:10EB400058A1FF1FCCA1FF1F034B1B68DB0401D59D
:10EB5000FFF758BF704700BF3480044010B5044C25
:10EB6000237823B101F0FCFA2378002BFAD110BDF1
:10EB7000C4A1FF1F054A064B10781B78C0B2DBB258
:10EB8000984238BF4030C01A704700BF58A1FF1FDD
:10EB900059A1FF1F30B42B4B1A7994061FD52A4870
:10EBA000DA790378294901333F2B0978C8BF00235C
:10EBB0008B42D2B203D0264CD9B2E2540170254A1E
:10EBC000116861B1244A1278D2B2934236BFC2F1C1
:10EBD00040029B1A9B18272BC4BF01230B70194AB4
:10EBE000D378DBB2180611D45A060DD5154B1B7914
:10EBF0005B0609D5194B1A491B6800220A7003B13C
:10EC00001A70104B2C22DA7030BC7047117909064B
:10EC1000EAD5144910480C780178C9B28C420DD05D
:10EC20004A1C272A84BF00210A460F4D054C98BF75
:10EC3000D1B2AA5CD2B2E2710170D5E76C21D17079
:10EC4000D2E700BF00C0064058A1FF1F59A1FF1F17
:10EC500084A1FF1F54A1FF1FC5A1FF1FC8A1FF1F53
:10EC6000C4A1FF1FCCA1FF1F5CA1FF1F21282FD82B
:10EC7000184B195CFF292BD0174B184ADFF870C0CE
:10EC800003EBC000F0B54368DFF868E0144F154DA2
:10EC9000154E00241C60DEF80030012043F02003F4
:10ECA0008840CEF8003014604FF4A07338602E60B6
:10ECB000C2F800C0013BFDD113689B05FCD42023A2
:10ECC000013BFDD1094B09B233F8110080B2F0BD10
:10ECD00000207047B4520100A451010000500440CC
:10ECE0000850044004500440000002030051044056
:10ECF00080014A0038800440431E032B14D872B6AA
:10ED00000A4951F8230068B170B4094C058834F8F9
:10ED10001320466841F82360521B24F8132062B682
:10ED200070BC704762B670470020704728A2FF1F72
:10ED3000F0A3FF1F013803280BD872B6074B53F816
:10ED4000203043B100205B680130002BFBD162B65C
:10ED50007047002070471846F9E700BF7CA2FF1FEC
:10ED600030B472B62B4A13781D0706D52A4B196AA0
:10ED7000002936D0996A002941D053781C0706D55E
:10ED8000254B196C00293ED0996C002939D0937815
:10ED9000190705D5204B196E002936D0996E89B117
:10EDA000D3781B0707D51C4BD3F880207AB3D3F850
:10EDB000882011213AB162B6184B00221A7030BC7B
:10EDC00000F04ABE0D21154C154D227843F8315004
:10EDD00003EBC1030830013A5860227062B630BCC0
:10EDE000704704220D4C0F4D217843F8325003EB4D
:10EDF000C20308304A1E5860227062B6EFE7052150
:10EE0000E1E70921DFE70822ECE70C22EAE710221C
:10EE1000E8E700BFD85201000080FF1FA5A2FF1F36
:10EE2000C800400088004000431E032B1DD81B4A29
:10EE3000400140F0100030B4104472B6184CE25C4F
:10EE4000032A1BD8DFE802F00212151703220D88EF
:10EE5000E25410F0080F14BFC823882343EA054387
:10EE600008310360416062B630BC7047083002224E
:10EE7000EDE70522EBE708300422E8E7094A52F8FB
:10EE8000230038B1084A52F82300416042F82310A9
:10EE900062B6E9E742F82310034AF7E70080FF1F54
:10EEA000B4A2FF1F7CA2FF1F8CA2FF1F00BE7047F1
:10EEB0002DE9F04FDFF818B3DFF818A387B044E06E
:10EEC000AD4F4FEA930807EBC809013ED9F804207B
:10EED00003F00803F6B2A2F1080003F0FF04002BD0
:10EEE00040F0018157F838301B0C99B222F8081C09
:10EEF000002B00F0EF80A14B22F8064C42F8044CA6
:10EF000053F82620002A00F0CF819D4D55F8263079
:10EF100058609C4C45F8260034F81630194424F803
:10EF2000161000F079FD002800F0C281964A974B38
:10EF300019F0080F00F1080018BF1346C9F80400C3
:10EF400047F8383008238BF800309BF80040E4B2D3
:10EF500065071CD58E4B1B78B3B18E490A7802F039
:10EF6000FF0322B1013BDBB20B7003B900BE8A493B
:10EF70000A7802F0FF032AB1013BDBB20B70002BD1
:10EF800000F0688100F066FE04238BF8003004F086
:10EF9000080303F0FF02002B00F0C9809AF800304C
:10EFA000DBB21E098CD19A08DFF8CC9159F83210E7
:10EFB00009EBC200C1F38301013940680C2900F25A
:10EFC0008580DFE801F07A7A8383838383834683B5
:10EFD000838307000168714D4068714F714E68600E
:10EFE000296088B240F281610024674B49F83230D1
:10EFF0004FF0010E88423C60C9F81040C9F8184033
:10F0000086F800E05C4A00F2E780B0F5D06F80F04F
:10F010001B82B0F5817F00F0D98100F269818028E0
:10F0200000F02A82822840F0D781A98801F07F0170
:10F03000042900F2D1815C485C4A890008441470BC
:10F04000547001788C0740F1608382F800E002215F
:10F0500073E1534F3A682AB3554B524E55481988BD
:10F060003478057840298E4645F0020828BF4FF0D5
:10F07000400E002C84F001043470CEEB01010CBF73
:10F080008824C82409EBC80689B285F0010544EA42
:10F090000E447260198049F83840724405700029A6
:10F0A00065D03A603D4B1A88B2F5A06F0ED10021B1
:10F0B0009A785970404B1A7008E038493F4C0D68F7
:10F0C000A54200F09880304949F832103C4A0123AB
:10F0D000137037E72C4A2D4B19F0080F18BF134651
:10F0E00047F838302EE700F0B7FC364A364952F878
:10F0F0002630002B00F0E38058688C5D42F8260033
:10F1000003F10802C9F80420032C05D8DFE804F055
:10F110002C02292602228A551A8819F0080F0CBFE2
:10F120008823C82343EA024347F838300AE7E00758
:10F1300000F19380210600F1D180A20706D5234A71
:10F14000234913780220DBB213700870E30602D55E
:10F150001F4B10221A7007B0BDE8F08F04228A55A9
:10F16000DAE705228A55D7E703228A55D4E7BEF1AC
:10F17000400F18BF002294E70080FF1F28A2FF1F46
:10F18000D4A1FF1FF0A3FF1FC8004000880040006B
:10F19000B0A2FF1F39A2FF1F24A3FF1F9CA2FF1FC5
:10F1A000D0A1FF1F38A2FF1FC0200740A8A2FF1F49
:10F1B000E4A1FF1FA4A2FF1F98200740210900031C
:10F1C000942007407CA2FF1FB4A2FF1F88200740A5
:10F1D0008020074090200740B0F5106F00F07C8140
:10F1E00040F2A38040F62112904240F07B82A54A73
:10F1F000012313706AE74C68A3498C427FF463AF24
:10F200000178A9297FF45FAF417845297FF45BAF8E
:10F210008178C2297FF457AFC1786B297FF453AF4F
:10F220009A489B4E0178347881F00105002C41F01A
:10F23000020105700CBF8820C82084F0010449F841
:10F24000310009EBC10193483470002505244D605D
:10F25000047038E700F064FF94E68F4B89488B49CF
:10F260001A614FF0020E80F800E08C4F0A708C4952
:10F27000196099608B4E8C4D8C4C9A610D213970C0
:10F28000FF213170DFF84CE229702270884D894AE5
:10F290008EF800109F27012406F8047C5D6004703E
:10F2A000DA6007B0BDE8F08F43F82600824D30E603
:10F2B000824A47F8380013780133137042E68B5DB9
:10F2C000032B00F2BA8001A252F823F045EF0000B0
:10F2D00045EF000025F300001FF300006F49724B5B
:10F2E00080220D2008701A70A2077FF52FAF26E745
:10F2F00040F20232904240F0ED81AA8802F07F0293
:10F30000042A69D86D88002D66D16449CDF804E0DF
:10F31000920011440A7842F002020A70C1E101230E
:10F320008B550FE600238B550CE6B0F5086F53D1D3
:10F330006349644A097811707146ED888D4280F006
:10F34000E88252480478402DAE4644F0020C28BFB3
:10F350004FF0400E02EB0E0309EBCC0102930123A8
:10F360004A604FEA0E48CEEB050101930025C82202
:10F3700042EA080384F0010249F83C30357002701B
:10F38000DFF814C1424BDFF8048149BBBEF1400FE6
:10F390007FF42DAF42F0020C09EBCC03029ADFF8A8
:10F3A000F8E05A608DBB0D0445F088059DF80430E7
:10F3B0004EF83C500A4433700470134640297FF4E1
:10F3C00016AF0021404A3B60118010E7AA8802F086
:10F3D0007F02042A40F28B81304A0F23137006E724
:10F3E0004029D7D942F002020CEBC200029E4660CF
:10F3F000BDB19DF8045035481D703346403988F83A
:10F40000004040334CF83200DCE79DF804303370A4
:10F410000D04029B047045F0C8050B444EF83C50A7
:10F42000CCE79DF804501D70029B1D4888F80040F1
:10F43000403940334CF83200C4E719F0080F0CBFD4
:10F44000022303238B557DE521494A68002AC3D056
:10F450006C88B5F804E003E00C314A68002ABBD0A0
:10F460000B88A342F8D14B887345F5D1240A032CAD
:10F470000CBF1178098960E7124A02211470547098
:10F480005BE700BF9420074001000400A4A2FF1F17
:10F4900038A2FF1F39A2FF1F0080FF1FC0200740B6
:10F4A00088004000882007408020074098200740BF
:10F4B000E8A1FF1F3CA2FF1FD4A1FF1FA5A2FF1FB1
:10F4C000B0A2FF1FA8A2FF1FE4A1FF1FC8004000B9
:10F4D000DC5201008C200740B248116AAC780470FD
:10F4E0000C0600F19881D9F82820AF49100600F1E8
:10F4F000DB81D9F83020AC49120600F1D081D9F86F
:10F500003820A949130600F1C581D9F84020A64941
:10F51000150600F1BA81D9F84820A349140600F174
:10F52000AF81D9F85020A049100600F1A481D9F884
:10F5300058209D49120600F19981D9F860209A4916
:10F54000130600F18E81D9F868209749150600F15D
:10F550008381D9F870209449140600F17881D9F894
:10F5600078209149100600F16D81D9F880208E49EC
:10F57000120600F16181D9F888208B49130600F149
:10F580005581D9F890208849150600F14981D9F8AC
:10F5900098208549140600F1FF808448844A8549F3
:10F5A00001908548854D864C049700230596029569
:10F5B00080460F4616461D460394306828B14468BD
:10F5C00000F04AFA2046002CF9D100233360029B58
:10F5D00038681A46002342F8253028B1446800F004
:10F5E0003BFA2046002CF9D100223A60019A98F8A3
:10F5F00000301146002241F8042B039A0191023B8E
:10F600004FF0000122F81510032B07D8DFE803F0B4
:10F610005D025D024FF0010388F800300135042DD2
:10F6200006F1040607F1040708F10108C5D1654C8D
:10F63000654D2278654B049F059E002110072970B7
:10F640001A7000F19280624962780A700021C9F84C
:10F650003010C9F838101107DFF84C816ED4A27849
:10F660005C49DFF844810A7000211207C9F8501084
:10F67000C9F858104BD4E27857494B4C0A7013071D
:10F680004FF00001C9F87010C9F8781000F1AE8091
:10F6900033780193002283F00105C9F89020C9F85E
:10F6A00098200021029188468E460A464B480478ED
:10F6B00044F0020C09EBCC030393019B002B039B4A
:10F6C0005A600CBF8822C82252E64FF0000388F827
:10F6D0000030A3E7B0F5A06F7FF47EAE01230025D4
:10F6E0000193DEE740F621229042F7D074E66D8860
:10F6F000002D7FF471AE3A49CDF804E09200114438
:10F700000A7822F002020A70CBE7022115E600F027
:10F7100083F9002800F0EB800830324AC8F8640012
:10F72000C8F8602000F078F9002800F0DA8008308E
:10F730002D4AC9F86C00C9F868209CE700F06CF904
:10F74000002800F0E0800830264AC8F84400C8F8D5
:10F75000402000F061F9002800F0CF800830224AF4
:10F76000C9F84C00C9F8482079E700F055F900289D
:10F7700000F0A58008301B4AC9F82400C9F82020F1
:10F7800000F04AF9002800F094800830164AC9F8C1
:10F790002C00C9F8282056E7D1F89C00083800F062
:10F7A0005BF9FAE6B0A2FF1F0080FF1F8CA2FF1FCB
:10F7B00028A2FF1F7CA2FF1FB4A2FF1FD4A1FF1F1E
:10F7C000F0A3FF1FD8520100A5A2FF1FC4200740CD
:10F7D000C8200740CC200740D0200740A4A2FF1F2C
:10F7E000C020074088004000C800400000F014F925
:10F7F000002870D008304F4AC4F88400C4F8802034
:10F8000000F00AF9002860D008304B4AC9F88C0093
:10F81000C9F888203CE7506A083800F01DF962E614
:10F82000D1F89400083800F017F9B0E6D1F88C0050
:10F83000083800F011F9A4E6D1F88400083800F087
:10F840000BF998E6C86F083800F006F98DE6486FA6
:10F85000083800F001F982E6C86E083800F0FCF8BC
:10F8600077E6486E083800F0F7F86CE6C86D08389F
:10F8700000F0F2F861E6486D083800F0EDF856E661
:10F88000C86C083800F0E8F84BE6486C083800F01F
:10F89000E3F840E6C86B083800F0DEF835E6486B60
:10F8A000083800F0D9F82AE6C86A083800F0D4F819
:10F8B0001FE62A78C9F8280001322A70C3E62A78A0
:10F8C000C9F8200001322A705AE72A78C9F888005E
:10F8D00001322A70DCE62A78C4F8800001322A70EE
:10F8E0008EE72A78C9F8680001322A70C3E62A78C0
:10F8F000C8F8600001322A7014E72A78C9F8480075
:10F9000001322A70ABE62A78C8F8400001322A702A
:10F910001FE740298E4628BF4FF0400E02EB0E0332
:10F9200002930123CEEB01014FEA0E48002501931B
:10F93000BCE600BF88004000C8004000F8B500F0F9
:10F94000F9FC294B29482A4C2A4F2B4DDFF8BCC023
:10F95000DFF8BCE0294E00221A605A609A60DA6033
:10F960001A615A619A61DA611A625A629A62DA62BB
:10F970001A635A639A63DA631A645A649A64DA649B
:10F980001A655A659A65DA651A665A669A66DA667B
:10F990001A675A679A67DA67C3F880200168C3F864
:10F9A000842041F480210160C3F307212170C3F357
:10F9B0000740134938701B0E2B70FF238CF8003062
:10F9C000104D8EF8003010480B700123337084F80E
:10F9D000642070264FF40074102207F82C3C2E701F
:10F9E000046081F8F820F8BD0080FF1F34800440D7
:10F9F0009C200740B0200740B420074094200740D7
:10FA00001020074049E400E008E100E080200740C2
:10FA100088200740704700BF72B60D480268B2FAEE
:10FA200082F30F2B10DC4FF00041D94022EA010293
:10FA3000026062B6074803EBC303DB00C218002173
:10FA4000C15010465160704762B60020704700BF39
:10FA5000C093FF1FBC83FF1F0D4B0E4AC31AA2FBAE
:10FA600003231B090F2B0CD80B4A127852B972B61C
:10FA70000A484FF00041026821FA03F31A4302607A
:10FA800062B67047064A1278002AF0D0FFF768B9CC
:10FA9000BC83FF1F398EE338A5A2FF1FC093FF1F51
:10FAA000B0A2FF1F38B50E4B0E4C1B6821880546CF
:10FAB0008BB1B1F5917F05D20B4A4B1C55549BB2CB
:10FAC000238038BD0022084898470021064A555433
:10FAD0000123238038BDB1F5917FEDD338BD00BF40
:10FAE000DCA2FF1FFAA3FF1F00A4FF1F2DE9F843AC
:10FAF000214E224F3168012380463B70B1B1204D29
:10FB00004B8801EB8302013300240F2BC2F80880DD
:10FB10002C7004D84B8000233B70BDE8F883402351
:10FB20000B800320FFF780F93460F4E7DFF854908E
:10FB300099F80030002BF0D0114D45F6215408E023
:10FB4000013C12D02B7883B900F00AFB99F8003001
:10FB50007BB10320FFF7EEF80528F1D8FFF75CFF33
:10FB6000014630600028EBD0CAE701232B70BDE8C6
:10FB7000F883BDE8F88300BFF8A2FF1FCCA2FF1FE7
:10FB8000FCA2FF1FB0A2FF1F1201F8B5D5B2A1B3AE
:10FB9000012943D04378044600781B0643EA00401D
:10FBA00040F4704045F004068F1E3043FFF79EFF7F
:10FBB000022F04F1020314D9053414F8023C14F89E
:10FBC000032C14F8010C1B0443EA0223334343EAD9
:10FBD0000060033FFFF78AFF022F234604F103046E
:10FBE000EBD8022F23D0012F0DD045F4774040F001
:10FBF0000500BDE8F840FFF779BF14482843BDE889
:10FC0000F840FFF773BF187845F4770545F006050F
:10FC100045EA0020BDE8F840FFF768BF03780C48CC
:10FC200045EA03452843BDE8F840FFF75FBF1A786F
:10FC3000587845F0774545F0070545EA022545EA3D
:10FC40000040BDE8F840FFF751BF00BF06F0F700E5
:10FC500007F000F738B5084B1C7824B9074D296820
:10FC600009B14B8803B938BD9B000B800320FFF717
:10FC7000DBF82C6038BD00BFCCA2FF1FF8A2FF1F2D
:10FC80002DE9F041AD4E33680746002B00F092801D
:10FC90001D885A88910803EB81010432AA428C68BE
:10FCA00042D25A8004F00F064FEA1428A449A6F164
:10FCB000080208F00F00C4F30313062A00F101053F
:10FCC0000B701AD9B31E012B5FFA88F04ED9052E9E
:10FCD00048D0042E00F0A481731F022B7FD90F2E71
:10FCE0000ED1F72842D8F02802D0964B1B883BB1A2
:10FCF000FFF7D8FE0020BDE8F08127B1BD4202D059
:10FD00000020BDE8F081082EC4F3033300F08780A3
:10FD1000092E11D00A2E40F094800A2BF0D18A4B84
:10FD20008A4A1B68A02181E01846FFF795FE04204F
:10FD3000FEF7E2FF3060B5E7092BE1D1270E00F0B6
:10FD40007B81834B814A1B689021C4F30746117065
:10FD5000EDB2FCB2002B00F09D80224631462846D1
:10FD6000984797E0F02843D9F72841D0F1380E287A
:10FD7000C6D801A353F820F02FFF000013FF0000A6
:10FD800001FF000001FD000001FD0000F3FE000086
:10FD900001FD0000D3FF000001FD00009DFF0000F9
:10FDA000B7FF0000DBFE000001FD0000C3FE000005
:10FDB000A7FE0000674B1B78002BA1D00420FEF7A4
:10FDC0009BFF0346306000289AD00588002D7FF401
:10FDD00060AFFFF741FE35602846BDE8F081FFF7D0
:10FDE00061FEC4F30740FFF75DFE072E02D1200E2F
:10FDF000FFF758FE534B584A198858481468584D15
:10FE0000524A017000270E0AF0201F802E701070D9
:10FE10000CB301225348A0470120BDE8F081082B14
:10FE20007FF46EAF504B494A1B688021C4F30746EC
:10FE30001170EDB2240E6BB3284622463146984726
:10FE400028E00B2E11D10B2B7FF45AAF474B3F4AC2
:10FE50001B68B021EAE7464B1B68002B00F0FB80D3
:10FE6000404898470120BDE8F0810C2E40F0008109
:10FE70000C2B7FF445AF3F4B344A1B68C0211170F7
:10FE8000EDB2C4F30746002B00F0C8802846314687
:10FE9000240E98473849314A314B0D7016701C704A
:10FEA0000120BDE8F081354B1B68002B00F0D680A7
:10FEB0009847C4F30746254BEDB2240E83F8008023
:10FEC000E8E72F4B1B68002BF2D12E4B1B68A3B128
:10FED000FE209847C4F30746EDE72B4B1B68002B29
:10FEE000E6D1284B1B6843B1FC209847C4F3074672
:10FEF000E1E7264B1B68002BDAD1C4F30746DAE7AB
:10FF0000234B1B68C4F30746002BD4D030469847D8
:10FF1000D1E7204B1A68002AEFD0260C630C06F0BC
:10FF20007F0003F47E531843F6B29047C3E71A4BA1
:10FF30001B68C4F30746002BE8D1BCE704A3FF1FEE
:10FF4000FEA3FF1FFAA3FF1FE0A2FF1FF8A3FF1FDE
:10FF500014A3FF1FB0A2FF1FDCA2FF1FFCA3FF1F03
:10FF6000FDA3FF1F00A4FF1F0CA3FF1F10A3FF1F73
:10FF7000F4A2FF1FD0A2FF1FFFA3FF1FBCA2FF1F01
:10FF8000C0A2FF1FC4A2FF1F00A3FF1FF0A2FF1FFC
:10FF900008A3FF1FD8A2FF1FECA2FF1F3F4B1B6847
:10FFA000002B85D13E4B1B68002BA6D0FA2098472A
:10FFB000C4F307467FE73B4B1B68002B7FF478AF09
:10FFC000374B1B68002B98D0FB209847C4F307469B
:10FFD00071E7354B1B68002B7FF46AAF304B1B6811
:10FFE000002B8AD0F8209847C4F3074663E70E2B0E
:10FFF0007FF486AE2D4A2E4B1268E0211970002A3C
:020000021000EC
:1000000047D0260C610C06F07F0301F47E511943A2
:10001000EDB2A1F5005128469047F6B2240E39E71B
:10002000FFF740FDC4F30740FFF73CFD200EFFF74C
:1000300039FD0020BDE8F0811E4B1D4A1B68802160
:100040001170EDB2C4F3074683B1314628463A46F3
:1000500098473C461EE70120BDE8F081104B1B6825
:10006000002B3FF44AAFFF20984746E71C4611E7B4
:100070000D2EBCD10D2B7FF443AE0F4B0C4A1B68E9
:10008000D0211170EDB2C4F30746002B7FF4FEAE11
:10009000C4E7C4F30746EDB2240EFBE6E8A2FF1F57
:1000A000C4A2FF1FC8A2FF1FB8A2FF1FD4A2FF1F38
:1000B000F8A3FF1F0CA3FF1FE4A2FF1F38B5164DC6
:1000C0002868E0B101884488A14213DD03191B7A36
:1000D00083B104F10803C2180C1B002302E012F8DC
:1000E000011F21B10133A342F9D1204638BD1C467E
:1000F000204638BDFFF7B0FC0020286038BD074B14
:100100001B780BB9002038BD0220FEF7F5FD2860F2
:100110000028D7D1F6E700BF20A3FF1FB0A2FF1F22
:100120000D4B1B78BBB910B50C4C216803F0FF02D6
:100130004B883F2B07DC07330B4401F1470003F8E2
:10014000012F8342FBD140230B800120FEF76CFE80
:100150000023236010BD704718A3FF1F1CA3FF1FBF
:1001600038B5224C237803B138BD01232370FFF743
:10017000A5FF70BB00F048F840BBFEF7ADFB10BB1D
:10018000FEF7F8FCE0B900232370EFF30583002BA2
:10019000EAD1EFF3108172B6154B1868E0B1154C37
:1001A0002278CAB945691D6001232370C5B1AA61CF
:1001B00001B962B600254577836898472570D3E773
:1001C00000F020F8DFE700F01BF8D9E700F016F8A0
:1001D000D3E7FFF71FFCCDE70029C5D162B638BDD4
:1001E000054B1D600029E5D1E3E700BF25A3FF1FF4
:1001F000C0A0FF1FC4A0FF1FBCA0FF1F704700BF0F
:10020000704700BF704700BF054A064B10781B7847
:10021000C0B2DBB2984238BF4030C01A704700BF4E
:100220002CA3FF1F2DA3FF1FF0B4384B1A7912F037
:10023000300F2CD072B6997D01F0FF0200293DD01D
:1002400062B6334F334938780D78334E1C46C0B20E
:10025000EDB2431C402BE17928BF0023AB4202F1F1
:10026000FF32C9B21CBFF154184612F0FF02F0D1A0
:100270002A4B1B68C2B23A704BB1A84236BFC5F1D7
:100280004005401B40192728C4BF01221A701F498E
:10029000CA78D2B2150616D452060DD51B4B1B795F
:1002A0005B0609D51E4B1F491B6800220A7003B16B
:1002B0001A70164B3C22DA70F0BC70474022D97994
:1002C0005A7462B6E3E70B791C06E5D5164B174E58
:1002D0001C783378E4B2DBB29C420ED0144D01E0BE
:1002E000A3420AD00133402B28BF00230879E85CE1
:1002F000C0B2C871087D0728F2D9DBB20349337058
:100300000B79180644BF7C23CB70C5E700A00640DC
:100310002CA3FF1F2DA3FF1F70A3FF1F28A3FF1FE8
:10032000B4A3FF1FB0A3FF1FB8A3FF1FB1A3FF1FFC
:1003300030A3FF1F70B584B072B6194B194D1A481F
:10034000702241260F2480211A702E701A460470E4
:10035000197013781B06FCD5144B186862B6144B41
:10036000144C984298BF00EB800001A998BF400050
:100370000A22FDF78DFD01A92046002311F8012B6B
:1003800001333AB10A2B20F8022FF7D1162323703C
:1003900004B070BD5B00DBB2237004B070BD00BF61
:1003A0000000024007000240060002400800024030
:1003B0007F9698008C94FF1F2DE9F043DFF8EC80C6
:1003C0008BB006460F4600F073F898F90030013301
:1003D00004460D4637D03046394600F0DFF9002894
:1003E00031D02BA3D3E900233046394600F026FE56
:1003F000814668BB28A3D3E900233046394600F084
:10040000FFFD00B398F90030254ACDF82090042470
:1004100000200021022BCDE90467CDE9026700949A
:100420000192CDE906012CD0684600F0BDF940B339
:10043000089B1BB101F0AAF9089B0360DDE90601E6
:100440000BB0BDE8F083204629460BB0BDE8F08331
:10045000134A98F90030019203210022CDE9046784
:10046000CDE90267009108922BB90E4B4FF0604224
:10047000CDE90623D8E70C490020022BCDE906017F
:10048000D2D101F083F922230360D1E7AFF30080DA
:10049000EF39FAFE422E864051302DD5104987C0E3
:1004A00048530100FFFFEF470000F07FA294FF1FB9
:1004B0002DE9F04FB04F21F00042BA4283B00C4614
:1004C0004FEAD17605460DD9AC4FBA4225D9C1F3D2
:1004D0001303034340F0EF800EB10020014603B048
:1004E000BDE8F08FA64B9A4200F2CC80A54B9A4211
:1004F00000F2DE808AA3D3E9002300F05DF9002238
:10050000A14B00F09BFD002800F005812846214604
:1005100000229D4B00F050F9E1E783A3D3E90023CB
:1005200000F08CFD002840F0CB802846214680A3B7
:10053000D3E9002300F064FD0028CED1934B284678
:1005400003EBC60821467CA3D3E9002300F0E6FABA
:10055000D8E9002300F030F900F07AFD804600F081
:1005600077FA77A3D3E9002306460F4600F0D6FAC0
:1005700002460B462846214600F01CF972A3D3E937
:100580000023CDE900013046394600F0C7FA824623
:100590008B4652465B46DDE9000100F00BF905464B
:1005A0000C462A4623462846214600F0B7FA68A39F
:1005B000D3E9002306460F4600F0B0FA66A3D3E95C
:1005C000002300F0F7F832463B4600F0A7FA64A398
:1005D000D3E9002300F0F0F832463B4600F09EFAE3
:1005E00061A3D3E9002300F0E5F832463B4600F072
:1005F00095FA5FA3D3E9002300F0DEF832463B46CC
:1006000000F08CFA02460B462846214600F0D2F84C
:1006100006460F462846214632463B46B8F1000FB3
:1006200056D000F07BFA324604460D463B46002089
:100630004FF0804100F0BEF802460B4620462946A6
:1006400000F096FB02460B465046594600F0B2F8C1
:10065000DDE9002300F0AEF80B4602464A490020CF
:1006600000F0A8F86FF47F7398454FDA08F57A78B0
:1006700001EB085100224FF0B87300F04FFA03B0BD
:10068000BDE8F08F424B9A423FF658AF414BF40021
:100690002344D3E9002300F08DF83F4BC6F1010855
:1006A0001C44CDE90001D4E900ABC6EB080870E7B3
:1006B0004FF0000875E702460B4600F07DF80EE7A4
:1006C00017A3D3E900231046194600F027FA06E7DE
:1006D00000F024FA0022804689464FF080433046DD
:1006E000394600F067F802460B464046494600F09E
:1006F0003FFB2A46234600F05DF802460B460020E9
:10070000214900F057F803B0BDE8F08F01EB085124
:1007100003B0BDE8F08F804643E700BFAFF3008031
:100720009C7500883CE4377EEF39FAFE422E864005
:1007300051302DD5104987C0FE822B654715F73FF4
:100740000000E0FE422EE63F763C7935EF39EA3D87
:10075000D0A4BE726937663EF16BD2C541BDBB3EC7
:100760002CDE25AF6A56113F93BDBE166CC1663FA5
:100770003E5555555555C53F412E8640FFFFEF7FED
:10078000422ED63FFFFF2F3E0000F03F50530100A6
:10079000B1A2F03F705301006053010041F00041ED
:1007A00001F58010C00F70470020704781F00041B4
:1007B00002E000BF83F0004330B54FEA41044FEA46
:1007C000430594EA050F08BF90EA020F1FBF54EAE1
:1007D000000C55EA020C7FEA645C7FEA655C00F07D
:1007E000E2804FEA5454D4EB5555B8BF6D420CDD4E
:1007F0002C4480EA020281EA030382EA000083EAD1
:10080000010180EA020281EA0303362D88BF30BD70
:1008100011F0004F4FEA01314FF4801C4CEA1131C6
:1008200002D0404261EB410113F0004F4FEA033325
:100830004CEA133302D0524263EB430394EA050FB0
:1008400000F0A780A4F10104D5F1200E0DDB02FA1F
:100850000EFC22FA05F2801841F1000103FA0EF2B3
:10086000801843FA05F359410EE0A5F120050EF179
:10087000200E012A03FA0EFC28BF4CF0020C43FAAA
:1008800005F3C01851EBE37101F0004507D54FF0B7
:10089000000EDCF1000C7EEB00006EEB0101B1F507
:1008A000801F1BD3B1F5001F0CD349085FEA30004D
:1008B0004FEA3C0C04F101044FEA445212F5800F58
:1008C00080F09A80BCF1004F08BF5FEA500C50F1F5
:1008D000000041EB045141EA050130BD5FEA4C0CD8
:1008E000404141EB010111F4801FA4F10104E9D161
:1008F00091F0000F04BF01460020B1FA81F308BF58
:100900002033A3F10B03B3F120020CDA0C3208DD23
:1009100002F1140CC2F10C0201FA0CF021FA02F1FE
:100920000CE002F11402D8BFC2F1200C01FA02F16E
:1009300020FA0CFCDCBF41EA0C019040E41AA2BF93
:1009400001EB0451294330BD6FEA04041F3C1CDA5B
:100950000C340EDC04F11404C4F1200220FA04F07B
:1009600001FA02F340EA030021FA04F345EA030125
:1009700030BDC4F10C04C4F1200220FA02F001FAE7
:1009800004F340EA0300294630BD21FA04F0294669
:1009900030BD94F0000F83F4801306BF81F4801102
:1009A0000134013D4EE77FEA645C18BF7FEA655C75
:1009B00029D094EA050F08BF90EA020F05D054EA47
:1009C000000C04BF1946104630BD91EA030F1EBF4C
:1009D0000021002030BD5FEA545C05D14000494150
:1009E00028BF41F0004130BD14F580043CBF01F543
:1009F000801130BD01F0004545F0FE4141F4700129
:100A00004FF0000030BD7FEA645C1ABF1946104603
:100A10007FEA655C1CBF0B46024650EA013406BF04
:100A200052EA033591EA030F41F4002130BD00BFC3
:100A300090F0000F04BF0021704730B54FF4806480
:100A400004F132044FF000054FF0000150E700BF01
:100A500090F0000F04BF0021704730B54FF4806460
:100A600004F1320410F0004548BF40424FF000014D
:100A70003EE700BF42004FEAE2014FEA31014FEA90
:100A800002701FBF12F07F4393F07F4F81F06051DF
:100A9000704792F0000F14BF93F07F4F704730B54E
:100AA0004FF4607401F0004521F0004120E700BFE1
:100AB00050EA010208BF704730B54FF000050AE068
:100AC00050EA010208BF704730B511F0004502D569
:100AD000404261EB41014FF4806404F132045FEA6B
:100AE000915C3FF4DCAE4FF003025FEADC0C18BF10
:100AF00003325FEADC0C18BF033202EBDC02C2F106
:100B0000200300FA03FC20FA02F001FA03FE40EA97
:100B10000E0021FA02F11444C1E600BF70B54FF097
:100B2000FF0C4CF4E06C1CEA11541DBF1CEA135579
:100B300094EA0C0F95EA0C0F00F0DEF82C4481EAE1
:100B4000030621EA4C5123EA4C5350EA013518BF01
:100B500052EA033541F4801143F4801338D0A0FBEE
:100B600002CE4FF00005E1FB02E506F00042E0FB9B
:100B700003E54FF00006E1FB03569CF0000F18BFA1
:100B80004EF0010EA4F1FF04B6F5007F64F5407449
:100B900004D25FEA4E0E6D4146EB060642EAC621DC
:100BA00041EA55514FEAC52040EA5E504FEACE2E49
:100BB000B4F1FD0C88BFBCF5E06F1ED8BEF1004F4C
:100BC00008BF5FEA500E50F1000041EB045170BDC8
:100BD00006F0004646EA010140EA020081EA03010C
:100BE000B4EB5C04C2BFD4EB0C0541EA045170BD08
:100BF00041F480114FF0000E013C00F3AB8014F182
:100C0000360FDEBF002001F0004170BDC4F10004CA
:100C1000203C35DA0C341BDC04F11404C4F120054B
:100C200000FA05F320FA04F001FA05F240EA0200A6
:100C300001F0004221F0004110EBD37021FA04F6DC
:100C400042EB06015EEA430E08BF20EAD37070BD96
:100C5000C4F10C04C4F1200500FA04F320FA05F0F5
:100C600001FA04F240EA020001F0004110EBD370F7
:100C700041F100015EEA430E08BF20EAD37070BD67
:100C8000C4F1200500FA05F24EEA020E20FA04F340
:100C900001FA05F243EA020321FA04F001F00041EF
:100CA00021FA04F220EA020000EBD3705EEA430E60
:100CB00008BF20EAD37070BD94F0000F0FD101F08F
:100CC0000046400041EB010111F4801F08BF013CC8
:100CD000F7D041EA060195F0000F18BF704703F006
:100CE0000046520043EB030313F4801F08BF013D8D
:100CF000F7D043EA0603704794EA0C0F0CEA135549
:100D000018BF95EA0C0F0CD050EA410618BF52EA02
:100D10004306D1D181EA030101F000414FF0000008
:100D200070BD50EA410606BF1046194652EA430616
:100D300019D094EA0C0F02D150EA013613D195EA8A
:100D40000C0F05D152EA03361CBF104619460AD1D2
:100D500081EA030101F0004141F0FE4141F47001DC
:100D60004FF0000070BD41F0FE4141F4780170BDCC
:100D700070B54FF0FF0C4CF4E06C1CEA11541DBF31
:100D80001CEA135594EA0C0F95EA0C0F00F0A7F833
:100D9000A4EB050481EA030E52EA03354FEA013160
:100DA00000F088804FEA03334FF0805545EA131373
:100DB00043EA12634FEA022245EA111545EA10653B
:100DC0004FEA00260EF000419D4208BF964244F1D2
:100DD000FD0404F5407402D25B084FEA3202B61AF1
:100DE00065EB03055B084FEA32024FF480104FF4C5
:100DF000002CB6EB020E75EB030E22BFB61A754639
:100E000040EA0C005B084FEA3202B6EB020E75EBCB
:100E1000030E22BFB61A754640EA5C005B084FEA33
:100E20003202B6EB020E75EB030E22BFB61A754600
:100E300040EA9C005B084FEA3202B6EB020E75EB0B
:100E4000030E22BFB61A754640EADC0055EA060ECC
:100E500018D04FEA051545EA16754FEA06164FEA0F
:100E6000C30343EA52734FEAC2025FEA1C1CC0D1BB
:100E700011F4801F0BD141EA00014FF000004FF048
:100E8000004CB6E711F4801F04BF01430020B4F109
:100E9000FD0C88BFBCF5E06F3FF6AFAEB5EB030CC1
:100EA00004BFB6EB020C5FEA500C50F1000041EBBE
:100EB000045170BD0EF0004E4EEA113114EB5C048B
:100EC000C2BFD4EB0C0541EA045170BD41F480115E
:100ED0004FF0000E013C90E645EA060E8DE60CEA66
:100EE000135594EA0C0F08BF95EA0C0F3FF43BAF83
:100EF00094EA0C0F0AD150EA01347FF434AF95EA3A
:100F00000C0F7FF425AF104619462CE795EA0C0F1D
:100F100006D152EA03353FF4FDAE1046194622E7EA
:100F200050EA410618BF52EA43067FF4C5AE50EAC4
:100F300041047FF40DAF52EA43057FF4EBAE12E7B4
:100F40004FF0FF3C06E000BF4FF0010C02E000BF95
:100F50004FF0010C4DF804CD4FEA410C7FEA6C5C78
:100F60004FEA430C18BF7FEA6C5C1BD001B050EA1B
:100F7000410C0CBF52EA430C91EA030F02BF90EA06
:100F8000020F0020704710F1000F91EA030F58BFC5
:100F9000994208BF90422CBFD8176FEAE37040F027
:100FA000010070474FEA410C7FEA6C5C02D150EAC5
:100FB000013C07D14FEA430C7FEA6C5CD6D152EA80
:100FC000033CD3D05DF8040B704700BF8446104645
:100FD00062468C461946634600E000BF01B5FFF744
:100FE000B7FF002848BF10F1000F01BD4DF808ED14
:100FF000FFF7F4FF0CBF012000205DF808FB00BFE5
:101000004DF808EDFFF7EAFF34BF012000205DF83E
:1010100008FB00BF4DF808EDFFF7E0FF94BF01208B
:1010200000205DF808FB00BF4DF808EDFFF7CEFF8C
:1010300094BF012000205DF808FB00BF4DF808EDCB
:10104000FFF7C4FF34BF012000205DF808FB00BF9C
:101050004FEA410212F5001215D211D56FF47873E0
:10106000B3EB625212D94FEAC12343F0004343EA83
:10107000505311F0004F23FA02F018BF404270475E
:101080004FF00000704750EA013005D111F00040E8
:1010900008BF6FF0004070474FF00000704700BF7E
:1010A0004FEA4102B2F1E04324BFB3F5001CDCF18A
:1010B000FE5C0DD901F0004C4FEAC0024CEA5070C2
:1010C000B2F1004F40EB830008BF20F001007047F1
:1010D00011F0804F21D113F13872BCBF01F00040F4
:1010E000704741F480114FEA5252C2F11802C2F126
:1010F000200C10FA0CF320FA02F018BF40F00100A7
:101100004FEAC1234FEAD32303FA0CFC40EA0C0058
:1011100023FA02F34FEA4303CCE77FEA625307D195
:1011200050EA01331EBF4FF0FE4040F440007047CC
:1011300001F0004040F0FE4040F40000704700BF66
:1011400080F0004002E000BF81F0004142001FBF7C
:101150005FEA410392EA030F7FEA226C7FEA236C85
:101160006AD04FEA1262D2EB1363C1BFD21841407A
:1011700048404140B8BF5B42192B88BF704710F010
:10118000004F40F4000020F07F4018BF404211F0B3
:10119000004F41F4000121F07F4118BF494292EA1B
:1011A000030F3FD0A2F1010241FA03FC10EB0C0047
:1011B000C3F1200301FA03F100F0004302D54942D4
:1011C00060EB4000B0F5000F13D3B0F1807F06D381
:1011D00040084FEA310102F10102FE2A51D2B1F179
:1011E000004F40EBC25008BF20F0010040EA03006E
:1011F0007047490040EB000010F4000FA2F101021B
:10120000EDD1B0FA80FCACF1080CB2EB0C0200FAA4
:101210000CF0AABF00EBC25052421843BCBFD040F2
:101220001843704792F0000F81F4000106BF80F46C
:1012300000000132013BB5E74FEA41037FEA226C2F
:1012400018BF7FEA236C21D092EA030F04D092F0FA
:10125000000F08BF0846704790EA010F1CBF00202E
:10126000704712F07F4F04D1400028BF40F000408B
:10127000704712F100723CBF00F50000704700F0AB
:10128000004343F0FE4040F4000070477FEA2262D2
:1012900016BF08467FEA23630146420206BF5FEAA3
:1012A000412390EA010F40F4800070474FF00003A3
:1012B00004E000BF10F0004348BF40425FEA000C6A
:1012C00008BF704743F0964301464FF000001CE012
:1012D00050EA010208BF70474FF000030AE000BF68
:1012E00050EA010208BF704711F0004302D54042A6
:1012F00061EB41015FEA010C02BF84460146002018
:1013000043F0B64308BFA3F18053A3F50003BCFA32
:101310008CF2083AA3EBC25310DB01FA02FC6344DF
:1013200000FA02FCC2F12002BCF1004F20FA02F2E6
:1013300043EB020008BF20F00100704702F12002D9
:1013400001FA02FCC2F1200250EA4C0021FA02F23A
:1013500043EB020008BF20EADC7070474FF0FF0C3F
:101360001CEAD0521EBF1CEAD15392EA0C0F93EA3A
:101370000C0F6FD01A4480EA010C400218BF5FEADC
:1013800041211ED04FF0006343EA501043EA51114F
:10139000A0FB01310CF00040B1F5000F3EBF490049
:1013A00041EAD3715B0040EA010062F17F02FD2A4D
:1013B0001DD8B3F1004F40EBC25008BF20F0010030
:1013C000704790F0000F0CF0004C08BF49024CEA47
:1013D000502040EA51207F3AC2BFD2F1FF0340EAD9
:1013E000C250704740F400004FF00003013A5DDC4A
:1013F00012F1190FDCBF00F000407047C2F100028B
:10140000410021FA02F1C2F1200200FA02FC5FEA77
:10141000310040F1000053EA4C0308BF20EADC70C1
:10142000704792F0000F00F0004C02BF400010F433
:10143000000F013AF9D040EA0C0093F0000F01F0E0
:10144000004C02BF490011F4000F013BF9D041EA02
:101450000C018FE70CEAD15392EA0C0F18BF93EA04
:101460000C0F0AD030F0004C18BF31F0004CD8D12E
:1014700080EA010000F00040704790F0000F17BFB5
:1014800090F0004F084691F0000F91F0004F14D0FB
:1014900092EA0C0F01D142020FD193EA0C0F03D153
:1014A0004B0218BF084608D180EA010000F0004056
:1014B00040F0FE4040F40000704740F0FE4040F431
:1014C000400070474FF0FF0C1CEAD0521EBF1CEAD0
:1014D000D15392EA0C0F93EA0C0F69D0A2EB0302EE
:1014E00080EA010C49024FEA402037D04FF0805388
:1014F00043EA111143EA10130CF000408B4238BF4D
:101500005B0042F17D024FF4000C8B4224BF5B1A5A
:1015100040EA0C00B3EB510F24BFA3EB510340EAA8
:101520005C00B3EB910F24BFA3EB910340EA9C0056
:10153000B3EBD10F24BFA3EBD10340EADC001B01C6
:1015400018BF5FEA1C1CE0D1FD2A3FF650AF8B426A
:1015500040EBC25008BF20F0010070470CF0004C77
:101560004CEA50207F32C2BFD2F1FF0340EAC250A2
:10157000704740F400004FF00003013A37E792F063
:10158000000F00F0004C02BF400010F4000F013AC1
:10159000F9D040EA0C0093F0000F01F0004C02BFBC
:1015A000490011F4000F013BF9D041EA0C0195E725
:1015B0000CEAD15392EA0C0F08D142027FF47DAFBE
:1015C00093EA0C0F7FF470AF084676E793EA0C0FAE
:1015D00004D14B023FF44CAF08466EE730F0004CAC
:1015E00018BF31F0004CCAD130F000427FF45CAF3C
:1015F00031F000437FF43CAF5FE700BF4FF0FF3CAA
:1016000006E000BF4FF0010C02E000BF4FF0010CFC
:101610004DF804CD4FEA40024FEA41037FEA226CC5
:1016200018BF7FEA236C11D001B052EA530C18BFE7
:1016300090EA010F58BFB2EB030088BFC81738BF4C
:101640006FEAE17018BF40F0010070477FEA226C3A
:1016500002D15FEA402C05D17FEA236CE4D15FEA36
:10166000412CE1D05DF8040B704700BF844608466A
:101670006146FFE70FB5FFF7C9FF002848BF10F12B
:10168000000F0FBD4DF808EDFFF7F4FF0CBF012070
:1016900000205DF808FB00BF4DF808EDFFF7EAFFFA
:1016A00034BF012000205DF808FB00BF4DF808EDB5
:1016B000FFF7E0FF94BF012000205DF808FB00BFAA
:1016C0004DF808EDFFF7D2FF94BF012000205DF830
:1016D00008FB00BF4DF808EDFFF7C8FF34BF01203D
:1016E00000205DF808FB00BF4FEA4002B2F1FE4F58
:1016F0000FD34FF09E03B3EB12620DD94FEA0023D4
:1017000043F0004310F0004F23FA02F018BF4042AC
:1017100070474FF00000704712F1610F01D1420293
:1017200005D110F0004008BF6FF0004070474FF047
:101730000000704742000ED2B2F1FE4F0BD34FF0C3
:101740009E03B3EB126209D44FEA002343F0004337
:1017500023FA02F070474FF00000704712F1610F5A
:1017600001D1420202D14FF0FF3070474FF000002C
:10177000704700BF0B460146184600F001B800BF95
:1017800013460A460146022000F0ACBE014B186821
:10179000704700BFD098FF1F70B50F4E0F4D761BDE
:1017A000B61018BF002405D0013455F8043B984703
:1017B000A642F9D10A4E0B4D761B03F0E3FDB6109D
:1017C00018BF002406D0013455F8043B9847A642C0
:1017D000F9D170BD70BD00BF90530100905301005E
:1017E000A453010090530100024B0146186800F019
:1017F0000BB800BFD098FF1F024B0146186800F0DD
:1018000035BF00BFD098FF1F2DE9F04F01F10B0548
:10181000162D83B0064640F29F8035F0070500F193
:10182000BF80A94200F2BC8000F058FBB5F5FC7FF8
:10183000C0F09C826B0A00F0BA80042B00F2838116
:10184000A80900F1390E4FEA4E033830C44F07EBB8
:101850008303A3F108015C68A14207D1ACE0002A30
:1018600080F2AC80E468A14200F0A680636823F0B7
:1018700003035A1B0F2AF2DDB9493C6901F1080E36
:10188000744500F0B381636823F003035A1B0F2AE9
:1018900000F39981002AC1F814E0C1F810E080F249
:1018A0009E80B3F5007F80F06781DB0803F1010CB7
:1018B00001229B1002FA03F34A6851F83C80C4F8F5
:1018C000088001EBCC091A43A9F10803E3604A60E0
:1018D00041F83C40C8F80C40831001249C409442DD
:1018E00000F28A80144206D120F003006400144202
:1018F00000F10400FAD007EBC009CC468046DCF8C2
:101900000C108C4507D173E1002A80F28181C968EF
:101910008C4500F06D814B6823F003035A1B0F2A9E
:10192000F2DD0C46D1F80CC054F8088F4B1945F085
:1019300001054D6042F00101C8F80CC03046CCF8FA
:1019400008807B613B61C3F80CE0C3F808E0596094
:101950009A5000F0C5FA1FE0102921D800F0BEFA15
:101960001025062302207E4F07EB8303A3F1080214
:101970005C68944200F045816368E168A56823F0E3
:101980000303234430465A68E96042F001028D6047
:101990005A6000F0A5FA0834204603B0BDE8F08F85
:1019A00000240C232046336003B0BDE8F08F802371
:1019B0004FF0400E3F2049E770465DE72344E16861
:1019C0005A68A56842F00102E96030468D605A60AD
:1019D00000F086FA0834204603B0BDE8F08F2344B7
:1019E00030465A6842F001025A6000F079FA083431
:1019F000204603B0BDE8F08FBC68636823F003089D
:101A0000A84504D3C5EB08030F2B00F38C80554B7E
:101A1000DFF860911A68D9F8003001332A4404EBEA
:101A2000080A00F0608102F580520F3222F47F62D2
:101A300022F00F0211463046019200F04BFCB0F14B
:101A4000FF3F8346019A00F05881824500F2FC80F6
:101A5000454B1968DA451144196000F05381D9F8F3
:101A60000000DFF810E101301BBFCAEB0B0A514444
:101A7000CEF800B019601BF0070100F01781C1F12A
:101A80000800C1F58051834408315A44C2F30B0267
:101A9000C2EB010949463046019300F01BFC431C90
:101AA000019B00F03F81CBEB00024A4442F001026F
:101AB0001968C7F808B04944BC42CBF80420196043
:101AC000DFF8A49016D0B8F10F0F40F2FD806268E5
:101AD000A8F10C0323F00703E01802F001024FF015
:101AE000050E1A430F2B6260C0F804E0C0F808E04E
:101AF00000F21C811D4BBC681A68914288BF1960B6
:101B00001B4B1A689142626888BF196022F0030279
:101B10009542A2EB050301D80F2B04DC304600F000
:101B2000DFF9002438E7621943F0010345F00105AD
:101B300065603046BA60536000F0D2F90834204640
:101B400003B0BDE8F08F142B71D9542B00F2A480A0
:101B5000280B00F16F0E4FEA4E036E3076E600BFA1
:101B6000D498FF1FC4A3FF1FC8A3FF1FC0A3FF1F5C
:101B7000BCA3FF1FE09CFF1F5A0A042A5ED9142A47
:101B800000F2B38002F15C0149005B3207EB810C8B
:101B900057F82110DFF8DC81ACF1080C8C4500F01F
:101BA00088804A6822F00302934202D289688C45F9
:101BB000F7D1D1F80CC07A68C4F80CC0A160CCF899
:101BC0000840CC6088E6631942F0010745F0010542
:101BD000656030464B610B61C3F80CE0C3F808E068
:101BE0005F609A50083400F07BF9D5E64A6873E6E6
:101BF00008F1010818F0030F0CF1080C7FF47FAE18
:101C000030E0DC68A34208BF02303FF435AEB3E6F3
